:020000040800F2
:1000000000040020A51F0008F71F0008F71F0008C4
:10001000F71F0008F71F0008F71F00080000000086
:10002000000000000000000000000000F71F0008B2
:10003000F71F000800000000F71F000839BC010886
:10004000D1BD0108D3BD0108D5BD0108D9BD010846
:10005000F9BD0108FBBD0108FDBD010821BE010875
:1000600045BE010869BE01088DBE0108B1BE010888
:10007000B3BE0108B5BE0108B7BE0108B9BE01088C
:10008000BBBE0108BDBE0108BFBE0108F71F0008C6
:10009000F71F0008F71F0008F71F0008C1BE01087E
:1000A0000DBF01080FBF010811BF010813BF0108F0
:1000B00015BF010819BF010845BF0108A5BF010808
:1000C000A7BF0108A9BF0108ABBF0108ADBF010868
:1000D000B1BF010819C1010849C00108DDC101080B
:1000E000A1C2010865C3010867C3010869C301080B
:1000F0006DC30108C9C30108CBC30108CDC3010802
:10010000CFC30108D1C30108D3C30108D5C3010877
:10011000D9C30108ADC40108AFC40108B1C40108C6
:10012000B3C40108B5C40108B7C40108B9C40108C3
:1001300000000000000000000000000000000000BF
:1001400000000000000000000000000000000000AF
:10015000000000000000000000000000000000009F
:10016000000000000000000000000000000000008F
:10017000000000000000000000000000000000007F
:10018000000000000000000000000000000000006F
:10019000000000000000000000000000000000005F
:1001A000000000000000000000000000000000004F
:1001B000000000000000000000000000000000003F
:1001C000000000000000000000000000000000002F
:1001D000000000000000000000000000000000001F
:0401E0005FF8E0F1F3
:1001E800032A70B404460D4626D941EA000313F0E9
:1001F800030F13D020782B78984208BF294606D0E1
:100208001EE014F8010F11F8013F984218D1012A95
:1002180002F1FF32F5D1002070BC70470B4604464E
:1002280051F8045B50F8046BAE4204D1043A04461A
:10023800032A0B46F2D81D461046002ADAD1EBE70E
:10024800C01AE9E7032A2DE9F00109D82AB10023E9
:10025800CC5CC45401339342FAD1BDE8F001704735
:100268000B468218014603E02478013301F8014B5C
:1002780011F0030F1C46F7D113F003055DD06E4251
:10028800C5F1040CED009B594FEACC0C08E004348E
:10029800A7593B4607FA0CF748EA070741F8047BD9
:1002A800571A23FA05F8032FF1DC03E014F8013B91
:1002B80001F8013B8A42F9D8CFE753F8404C41F89E
:1002C800404C53F83C4C41F83C4C53F8384C41F8FE
:1002D800384C53F8344C41F8344C53F8304C41F80E
:1002E800304C53F82C4C41F82C4C53F8284C41F81E
:1002F800284C53F8244C41F8244C53F8204C41F82E
:10030800204C53F81C4C41F81C4C53F8184C41F83D
:10031800184C53F8144C41F8144C53F8104C41F84D
:10032800104C53F80C4C41F80C4C53F8084C41F85D
:10033800084C53F8044C41F8044C561A1D460C4618
:10034800403340313F2EB8DC2B460FE053F8101CE9
:1003580044F8101C53F80C1C44F80C1C53F8081CE7
:1003680044F8081C53F8041C44F8041C161B2146C6
:100378001D46103410330F2EE8DC2B4602E02468AB
:1003880041F8044B551A1C46032D03F10403F6DC0F
:1003980090E700BF032AC9B270B408D82AB103464F
:1003A800121803F8011B9342FBD170BC70478218E6
:1003B800044601E004F8011B14F0030FFAD14FF0D2
:1003C800013303FB01F31FE044F8403C44F83C3C94
:1003D80044F8383C44F8343C44F8303C44F82C3C6D
:1003E80044F8283C44F8243C44F8203C44F81C3C9D
:1003F80044F8183C44F8143C44F8103C44F80C3CCD
:1004080044F8083C44F8043C161B254640343F2E6B
:10041800DADC2C4607E044F8103C44F80C3C44F87D
:10042800083C44F8043C161B254610340F2EF2DC19
:1004380001E045F8043B541B032CFADC01E005F805
:10044800011B9542FBD3B0E710F0030F38B5044603
:1004580012D10368A3F1013222EA030313F0803FAB
:100468000AD1031D184653F8042BA2F1013525EAD9
:10047800020212F0803FF5D003782BB1431C1846D6
:1004880013F8012B002AFAD100F076F9204638BD7E
:10049800C9B2F0B4002950D010F0030F10D003787F
:1004A800002B79D0994246D0431C05E013F8012B64
:1004B800002A3FD091423ED013F0030F1846F5D1E1
:1004C800036841EA01270646A3F1013247EA0747D4
:1004D80022EA030212F0803F1DD187EA0303A3F149
:1004E800013222EA030313F0803F14D1043002E002
:1004F80012F0803F0FD1064650F8043BA3F10135B6
:1005080087EA030225EA0303A2F1013413F0803FCE
:1005180024EA0202ECD033783046002B3CD09942D2
:1005280009D0731C01E0914205D0184613F8012B3D
:10053800002AF8D11046F0BC704710F0030F0CD019
:100548000378002BF7D0431C03E013F8012B002A93
:10055800F1D013F0030F1846F7D102680346A2F151
:10056800013121EA020212F0803F0AD10430034629
:1005780050F8042BA2F1013121EA020212F0803F67
:10058800F5D01A781846002AD5D00133184613F842
:10059800012B002AFAD1CEE71846CCE780EA0102FF
:1005A80012F0030F3AD110F0030220F0030021F0FB
:1005B800030150F804CB08BF51F8043B0DD082F07A
:1005C80003024FEAC2026FF07F4323FA02F251F8A6
:1005D800043B4CEA020C43EA020300BFACF10132CF
:1005E8009C4501BF22EA0C0212F0803F50F804CB70
:1005F80051F8043BF2D04FEA0C604FEA1C2C01285A
:1006080028BFB0EB036F08BF1B0AF4D003F0FF0349
:100618004FEA1060A0EB0300704700BF10F0030F13
:100628000AD010F8012B11F8013B012A28BF9A4281
:10063800F4D0A2EB030070474DF8045D4DF8044D6B
:100648004FF0010242EA022242EA024201F0030CA0
:1006580021F0030150F8044B51F8045BBCF1020F80
:1006680026D04BD824F07F4CBCEB152FA4EB02030B
:1006780023EA04030DD113EAC21308BF51F8045B3F
:100688000AD18CEA040CBCEB056F0CD150F8044B72
:10069800E8E74FEA15255CE033F07F4352D10D7847
:1006A8004FEA146C55E04FEA146C05F0FF0550E072
:1006B8004FEA044CA4EB02034FEA1C4C23EA040360
:1006C800BCEB154F17D113EAC21308BF51F8045BEE
:1006D80007D18CEA040CBCEB054F08D150F8044B49
:1006E800E6E71B042ED10D884FEA144C31E04FEA9F
:1006F80005454FEA144C4FEA15452AE004F0FF0C73
:10070800BCEB156FA4EB020323EA04030DD113EA33
:10071800C21308BF51F8045B0AD18CEA040CBCEB85
:10072800052F0AD150F8044BE8E74FEA156510E0A9
:1007380014F0FF0F06D051F8045B4FEA142C25F093
:100748007F4506E04FF000005DF8044B5DF8045B60
:1007580070470CF0FF0205F0FF00012828BF904207
:1007680004BF4FEA1C2C2D0AF3D0A2EB00005DF861
:10077800044B5DF8045B704780EA0102844612F07E
:10078800030F4FD111F0030F32D14DF8044D11F082
:10079800040F51F8043B0BD0A3F101329A4312F035
:1007A800803F04BF4CF8043B51F8043B16D100BF0E
:1007B80051F8044BA3F101329A4312F0803FA4F19F
:1007C80001320BD14CF8043BA24312F0803F04BF26
:1007D80051F8043B4CF8044BEAD023460CF8013B93
:1007E80013F0FF0F4FEA3323F8D15DF8044B70473D
:1007F80011F0010F06D011F8012B0CF8012B002A7B
:1008080008BF704711F0020FBFD031F8022B12F069
:10081800FF0F16BF2CF8022B8CF8002012F47F4F24
:10082800B3D1704711F8012B0CF8012B002AF9D12C
:10083800704700BF20F0030110F00300C0F1000072
:1008480051F8043B00F1040C4FEACC0C6FF00002A5
:100858001CBF22FA0CF213434FF0010C4CEA0C2C8B
:100868004CEA0C4CA3EB0C0222EA030212EACC126B
:1008780004BF51F8043B0430F4D013F0FF0F1FBF3E
:10088800013013F47F4F013013F47F0F18BF01308C
:10089800704700BFF0B4002A46D041EA000313F0C5
:1008A80003032CD1032A07460E4643D904680D6872
:1008B800AC423FD1043A37D0A4F1013525EA04040B
:1008C80014F0803F18BF18462CD1041D0D1D0EE0F2
:1008D80054F8043B55F8041BA3F101308B4220EA7D
:1008E800030027D1043A1FD010F0803F1ED1032AFD
:1008F80027462E46ECD820462946002A1DD00478E3
:10090800013A0D78AC420CD172B18CB1002302E0EF
:1009180093420BD064B1013310F8014FCD5CAC4267
:10092800F6D0601BF0BC70471046FBE70020F9E7E3
:100938002046F7E738463146E1E724782D78F0E796
:1009480041EA000313F0030F0B4670B414BF0024F0
:100958000124032A94BF002404F001040546D4B9F5
:10096800BAB10E782B46013A03F8016B56B1AC1CAC
:100978007AB111F8015F2346013A04F8015C0134A9
:10098800002DF5D12AB19A18002103F8011B9342D2
:10099800FBD170BC7047194653F8044BA4F10136DB
:1009A80026EA040616F0803FDAD1043A45F8044BEB
:1009B800032A1946EFD8D3E701232DE9F0071D468E
:1009C80000264FF0FF37AC1900EB070C8C420DD214
:1009D8001CF805C010F80480E0452ED201252646F3
:1009E800E31BAC198C4200EB070CF1D34FF0010963
:1009F80000264D464FF0FF3C1360AC1900EB0C0885
:100A0800A1420ED918F8058010F804A0C2451AD9D9
:100A180001252646CCEB0409AC19A14200EB0C08D1
:100A2800F0D80CF101000137B8423CBF994638466E
:100A3800C2F80090BDE8F00770470BD00123374695
:100A48001D46F618BFE709D04FF00109B4464D46D8
:100A58004E44D2E79D4205D00135B4E74D4505D057
:100A68000135CAE72B4626460125ACE7A9462646A6
:100A78000125C2E72DE9F04FADF5826D81B014462E
:100A8800074610460DF580628B460C3219461D4606
:100A9800FFF792FF03AE04A901F57E72331F0090A1
:100AA80043F8045F9342FBD14DB1681E0023E25C1A
:100AB800C11A013303AEAB4246F82210F7D1DDF874
:100AC8000C142046009A6118FFF78AFB002877D19A
:100AD8000099814605F1FF380646C1F101020192ED
:100AE8005A46AB4609EB0B0501F1FF3AB81800214D
:100AF800AA1A00F0E5F900284FD1002D00F0C080B7
:100B08007B1903A913F8013C51F82330002B4CD171
:100B1800009B9E4228BF334698450FD903EB090135
:100B2800E05C7A18795C884205D038E012F8011F39
:100B3800E05C884233D101339845F7D8009A964251
:100B480080F0A48007EB090214F80A10534612F843
:100B58000A20914204BF0AEB0901791807D095E0F1
:100B680014F802C011F8010D844503D113465A1E2A
:100B7800B342F5D101369E4200F28D80DDF80C6457
:100B88002A46B144C6EB0B0609EB0B05B818002141
:100B9800AA1A00F095F90028AFD0002071E0019A58
:100BA8000026914499442A46EEE7002EFAD0DDF853
:100BB8000C2493423CBFC2EB0B0306469944F2E770
:100BC800009E4FF000080099AB1BB34238BF334674
:100BD800C1F101026E1E019201F1FF3A5A4689469F
:100BE800AB460133CDF80C3408EB0B05B8180021DF
:100BF800AA1A00F065F90028CFD1002D40D07B1942
:100C080003A913F8013C51F82330002B30D1B1452A
:100C180013D208EB090314F80910FA18FB5C99427F
:100C280018BF4B4627D14B4604E012F8011FE05C81
:100C3800884220D10133B342F7D3BAF1FF3F53467C
:100C48002CD007EB080C14F80A101CF80A20914263
:100C58000CD10AEB0802BA1804E0E05C12F8011D96
:100C6800884203D1013BF8D260460AE0DDF80C3433
:100C780098442A46B8E701992A4688449844B3E735
:100C8800284605B00DF5806DBDE8F08F009B013654
:100C98009E427FF673AF07EB0900F2E707EB080CFB
:100CA8006046EEE72DE9F04F8346037885B00C46A1
:100CB800002B00F0F9800A78A2B106460131012024
:100CC80002E011F8012B8AB1934214BF002000F012
:100CD800010016F8013F0D46002BF2D12B782BB1FD
:100CE8004FF0000B584605B0BDE8F08F0028F9D149
:100CF8000BF101002178FFF7CBFB2D1BA5F10102B9
:100D0800534243EB0203002808BF43F001030746A0
:100D180083B90BEB0508404594BFC0EB08084FF0BA
:100D280001081F2D08D9414622462B46FFF7A2FE8F
:100D38008346D7E78346D5E7294603AA2046FFF727
:100D48003BFE03996118814620464A46FFF748FA58
:100D580000284FD109F1FF33C9F10102064601927B
:100D680082464246C84699460AEB050BB818002148
:100D7800C2EB0B0200F0A4F80028B1D1BBF1000FC0
:100D8800B0D046452CBF334643469D420FD903EBAE
:100D98000A01E05C7A18795C884205D075E012F89F
:100DA800011FE05C884270D101339D42F7D1B04504
:100DB8007DD907EB0A0214F809104B4612F80920EE
:100DC800914202BF09EB0A01AC46791806D06EE0E1
:100DD800A55C11F8010D854203D113465A1EB34292
:100DE800F6D1654601369E4267D8039E5A46B244FC
:100DF800AE1BB9E7C9F10101C9EB0503424600265C
:100E080009F1FF3A88464B4538BF4B4601330393F7
:100E180006EB050BB8180021C2EB0B0200F050F8E6
:100E280000287FF45DAFBBF1000F3FF45BAF4D4589
:100E380012D906EB090314F80910FA18FB5C994259
:100E480008BF4B4605D026E012F8011FE05C884237
:100E580022D101339D42F7D1BAF1FF3F534628D042
:100E680007EB060C14F80A101CF80A20914217D157
:100E78000AEB0602BA1804E0E05C12F8011D884289
:100E88000ED1013BF8D2E3462CE7019A00269244A2
:100E98005A469A4468E74B4646445A46F618B7E716
:100EA800039B5A46F618B3E70D46012016E743465A
:100EB80098E707EB060CE34614E707EB0A0B11E784
:100EC80010F0030F034670B4C9B211D0002A22D023
:100ED80003788B421DD0013A013005E0DAB110F8F1
:100EE800014B013A8C4218D010F0030F0346F5D19C
:100EF800032A14D87AB1187888420ED0541E5D1C83
:100F080003E015F8016B8E4203D0013C2846F8D265
:100F1800002070BC70471046FBE71846F9E741EA25
:100F2800012646EA0646184653F8044B86EA0404A6
:100F3800A4F1013525EA040414F0803F03D1043AF2
:100F48001846032AEFD80346D4E700BF0000000084
:100F5800C1F30A5C0246ACF57E7C2DE9F84FACF192
:100F68000704132C0B4606460F468946804627DCA5
:100F7800002C52DB4FF6FF7CC0F20F0C4CFA04FA3F
:100F88000AEA0105054317D037A3D3E9002300F087
:100F980075F80022002300F0B3FC002856D0002F7B
:100FA80005DD4FF4801353FA04F407EB040929EA2A
:100FB8000A0900264B46324610461946BDE8F88F06
:100FC800332C07DDB4F5806FF6D100F057F80246F0
:100FD8000B46F1E74FF0FF3BACF11B0C2BFA0CFB77
:100FE8001BEA000FE8D020A3D3E9002300F046F85D
:100FF8000022002300F084FC40B3002F0ADD142CEB
:1010080006D00126C4F13404A64016EB080601D325
:1010180007F1010926EA0B0619E013A3D3E9002317
:1010280000F02CF80022002300F06AFC78B1002FB1
:1010380013DB46EA07054FF000094D45C3F6F07982
:101048000CBF2E46002608BFA94600E0B9464B460D
:10105800324610461946BDE8F88F00264FF0004981
:10106800F5E700BFAFF300809C7500883CE4377E4D
:1010780081F0004102E000BF83F0004330B54FEA41
:1010880041044FEA430594EA050F08BF90EA020FAE
:101098001FBF54EA000C55EA020C7FEA645C7FEA41
:1010A800655C00F0E2804FEA5454D4EB5555B8BF64
:1010B8006D420CDD2C4480EA020281EA030382EAD5
:1010C800000083EA010180EA020281EA0303362D67
:1010D80088BF30BD11F0004F4FEA01314FF4801C3A
:1010E8004CEA113102D0404261EB410113F0004F4C
:1010F8004FEA03334CEA133302D0524263EB430303
:1011080094EA050F00F0A780A4F10104D5F1200EA0
:101118000DDB02FA0EFC22FA05F2801841F10001FB
:1011280003FA0EF2801843FA05F359410EE0A5F1CF
:1011380020050EF1200E012A03FA0EFC28BF4CF000
:10114800020C43FA05F3C01851EBE37101F00045B6
:1011580007D54FF0000EDCF1000C7EEB00006EEBC3
:101168000101B1F5801F1BD3B1F5001F0CD349084D
:101178005FEA30004FEA3C0C04F101044FEA4452A4
:1011880012F5800F80F09A80BCF1004F08BF5FEA2B
:10119800500C50F1000041EB045141EA050130BD0B
:1011A8005FEA4C0C404141EB010111F4801FA4F1AE
:1011B8000104E9D191F0000F04BF01460020B1FA03
:1011C80081F308BF2033A3F10B03B3F120020CDA3B
:1011D8000C3208DD02F1140CC2F10C0201FA0CF019
:1011E80021FA02F10CE002F11402D8BFC2F1200C7E
:1011F80001FA02F120FA0CFCDCBF41EA0C01904034
:10120800E41AA2BF01EB0451294330BD6FEA04047C
:101218001F3C1CDA0C340EDC04F11404C4F1200267
:1012280020FA04F001FA02F340EA030021FA04F379
:1012380045EA030130BDC4F10C04C4F1200220FAD0
:1012480002F001FA04F340EA0300294630BD21FA0E
:1012580004F0294630BD94F0000F83F4801306BFD4
:1012680081F480110134013D4EE77FEA645C18BFC8
:101278007FEA655C29D094EA050F08BF90EA020F5F
:1012880005D054EA000C04BF1946104630BD91EA57
:10129800030F1EBF0021002030BD5FEA545C05D15A
:1012A8004000494128BF41F0004130BD14F5800499
:1012B8003CBF01F5801130BD01F0004545F0FE410D
:1012C80041F470014FF0000030BD7FEA645C1ABF42
:1012D800194610467FEA655C1CBF0B46024650EA79
:1012E800013406BF52EA033591EA030F41F40021A5
:1012F80030BD00BF90F0000F04BF0021704730B52B
:101308004FF4806404F132044FF000054FF00001FF
:1013180050E700BF90F0000F04BF0021704730B5C0
:101328004FF4806404F1320410F0004548BF404295
:101338004FF000013EE700BF42004FEAE2014FEAEA
:1013480031014FEA02701FBF12F07F4393F07F4FC5
:1013580081F06051704792F0000F14BF93F07F4FF7
:10136800704730B54FF4607401F0004521F000413A
:1013780020E700BF50EA010208BF704730B54FF0C0
:1013880000050AE050EA010208BF704730B511F0C5
:10139800004502D5404261EB41014FF4806404F1FD
:1013A80032045FEA915C3FF4DCAE4FF003025FEA7F
:1013B800DC0C18BF03325FEADC0C18BF033202EB07
:1013C800DC02C2F1200300FA03FC20FA02F001FA61
:1013D80003FE40EA0E0021FA02F11444C1E600BF00
:1013E80070B54FF0FF0C4CF4E06C1CEA11541DBFB3
:1013F8001CEA135594EA0C0F95EA0C0F00F0DEF87E
:101408002C4481EA030621EA4C5123EA4C5350EA62
:10141800013518BF52EA033541F4801143F48013B3
:1014280038D0A0FB02CE4FF00005E1FB02E506F044
:101438000042E0FB03E54FF00006E1FB03569CF099
:10144800000F18BF4EF0010EA4F1FF04B6F5007F9F
:1014580064F5407404D25FEA4E0E6D4146EB060611
:1014680042EAC62141EA55514FEAC52040EA5E509A
:101478004FEACE2EB4F1FD0C88BFBCF5E06F1ED844
:10148800BEF1004F08BF5FEA500E50F1000041EB7B
:10149800045170BD06F0004646EA010140EA020028
:1014A80081EA0301B4EB5C04C2BFD4EB0C0541EA4A
:1014B800045170BD41F480114FF0000E013C00F35F
:1014C800AB8014F1360FDEBF002001F0004170BD83
:1014D800C4F10004203C35DA0C341BDC04F114049C
:1014E800C4F1200500FA05F320FA04F001FA05F228
:1014F80040EA020001F0004221F0004110EBD370F5
:1015080021FA04F642EB06015EEA430E08BF20EA20
:10151800D37070BDC4F10C04C4F1200500FA04F3C3
:1015280020FA05F001FA04F240EA020001F0004155
:1015380010EBD37041F100015EEA430E08BF20EAC8
:10154800D37070BDC4F1200500FA05F24EEA020E10
:1015580020FA04F301FA05F243EA020321FA04F03F
:1015680001F0004121FA04F220EA020000EBD370F6
:101578005EEA430E08BF20EAD37070BD94F0000FF6
:101588000FD101F00046400041EB010111F4801F2A
:1015980008BF013CF7D041EA060195F0000F18BFDB
:1015A800704703F00046520043EB030313F4801F17
:1015B80008BF013DF7D043EA0603704794EA0C0FD1
:1015C8000CEA135518BF95EA0C0F0CD050EA4106E7
:1015D80018BF52EA4306D1D181EA030101F0004164
:1015E8004FF0000070BD50EA410606BF104619468C
:1015F80052EA430619D094EA0C0F02D150EA013698
:1016080013D195EA0C0F05D152EA03361CBF1046D8
:1016180019460AD181EA030101F0004141F0FE4177
:1016280041F470014FF0000070BD41F0FE4141F4FB
:10163800780170BD70B54FF0FF0C4CF4E06C1CEAFB
:1016480011541DBF1CEA135594EA0C0F95EA0C0FB0
:1016580000F0A7F8A4EB050481EA030E52EA03356B
:101668004FEA013100F088804FEA03334FF080558C
:1016780045EA131343EA12634FEA022245EA1115B9
:1016880045EA10654FEA00260EF000419D4208BF6A
:10169800964244F1FD0404F5407402D25B084FEA17
:1016A8003202B61A65EB03055B084FEA32024FF4C3
:1016B80080104FF4002CB6EB020E75EB030E22BF20
:1016C800B61A754640EA0C005B084FEA3202B6EBE0
:1016D800020E75EB030E22BFB61A754640EA5C008F
:1016E8005B084FEA3202B6EB020E75EB030E22BF1F
:1016F800B61A754640EA9C005B084FEA3202B6EB20
:10170800020E75EB030E22BFB61A754640EADC00DE
:1017180055EA060E18D04FEA051545EA16754FEA40
:1017280006164FEAC30343EA52734FEAC2025FEA5E
:101738001C1CC0D111F4801F0BD141EA00014FF0ED
:1017480000004FF0004CB6E711F4801F04BF0143BE
:101758000020B4F1FD0C88BFBCF5E06F3FF6AFAEDA
:10176800B5EB030C04BFB6EB020C5FEA500C50F16A
:10177800000041EB045170BD0EF0004E4EEA1131ED
:1017880014EB5C04C2BFD4EB0C0541EA045170BDF4
:1017980041F480114FF0000E013C90E645EA060E38
:1017A8008DE60CEA135594EA0C0F08BF95EA0C0F66
:1017B8003FF43BAF94EA0C0F0AD150EA01347FF4AE
:1017C80034AF95EA0C0F7FF425AF104619462CE785
:1017D80095EA0C0F06D152EA03353FF4FDAE1046E8
:1017E800194622E750EA410618BF52EA43067FF439
:1017F800C5AE50EA41047FF40DAF52EA43057FF4C9
:10180800EBAE12E74FF0FF3C06E000BF4FF0010CD3
:1018180002E000BF4FF0010C4DF804CD4FEA410C37
:101828007FEA6C5C4FEA430C18BF7FEA6C5C1BD004
:1018380001B050EA410C0CBF52EA430C91EA030F85
:1018480002BF90EA020F0020704710F1000F91EAE2
:10185800030F58BF994208BF90422CBFD8176FEAB0
:10186800E37040F0010070474FEA410C7FEA6C5C7E
:1018780002D150EA013C07D14FEA430C7FEA6C5C85
:10188800D6D152EA033CD3D05DF8040B704700BFB1
:101898008446104662468C461946634600E000BFFF
:1018A80001B5FFF7B7FF002848BF10F1000F01BDD1
:1018B8004DF808EDFFF7F4FF0CBF012000205DF89C
:1018C80008FB00BF4DF808EDFFF7EAFF34BF012021
:1018D80000205DF808FB00BF4DF808EDFFF7E0FFBA
:1018E80094BF012000205DF808FB00BF4DF808ED0B
:1018F800FFF7CEFF94BF012000205DF808FB00BF72
:101908004DF808EDFFF7C4FF34BF012000205DF853
:1019180008FB00BF4FEA4102B2F1E04324BFB3F530
:10192800001CDCF1FE5C0DD901F0004C4FEAC0024E
:101938004CEA5070B2F1004F40EB830008BF20F032
:101948000100704711F0804F21D113F13872BCBFEC
:1019580001F00040704741F480114FEA5252C2F141
:101968001802C2F1200C10FA0CF320FA02F018BF8A
:1019780040F001004FEAC1234FEAD32303FA0CFCDD
:1019880040EA0C0023FA02F34FEA4303CCE77FEA6C
:10199800625307D150EA01331EBF4FF0FE4040F4B6
:1019A8004000704701F0004040F0FE4040F4000065
:1019B800704700BF80F0004002E000BF81F00041A6
:1019C80042001FBF5FEA410392EA030F7FEA226CDD
:1019D8007FEA236C6AD04FEA1262D2EB1363C1BF6D
:1019E800D218414048404140B8BF5B42192B88BFDC
:1019F800704710F0004F40F4000020F07F4018BFFF
:101A0800404211F0004F41F4000121F07F4118BF1E
:101A1800494292EA030F3FD0A2F1010241FA03FCC6
:101A280010EB0C00C3F1200301FA03F100F00043AE
:101A380002D5494260EB4000B0F5000F13D3B0F176
:101A4800807F06D340084FEA310102F10102FE2AE5
:101A580051D2B1F1004F40EBC25008BF20F0010055
:101A680040EA03007047490040EB000010F4000F03
:101A7800A2F10102EDD1B0FA80FCACF1080CB2EB96
:101A88000C0200FA0CF0AABF00EBC25052421843F5
:101A9800BCBFD0401843704792F0000F81F400019A
:101AA80006BF80F400000132013BB5E74FEA41036D
:101AB8007FEA226C18BF7FEA236C21D092EA030FD9
:101AC80004D092F0000F08BF0846704790EA010F53
:101AD8001CBF0020704712F07F4F04D1400028BF80
:101AE80040F00040704712F100723CBF00F5000062
:101AF800704700F0004343F0FE4040F40000704798
:101B08007FEA226216BF08467FEA23630146420243
:101B180006BF5FEA412390EA010F40F48000704756
:101B28004FF0000304E000BF10F0004348BF4042FC
:101B38005FEA000C08BF704743F0964301464FF038
:101B480000001CE050EA010208BF70474FF0000394
:101B58000AE000BF50EA010208BF704711F00043D5
:101B680002D5404261EB41015FEA010C02BF8446A5
:101B78000146002043F0B64308BFA3F18053A3F504
:101B88000003BCFA8CF2083AA3EBC25310DB01FA4B
:101B980002FC634400FA02FCC2F12002BCF1004FCF
:101BA80020FA02F243EB020008BF20F00100704760
:101BB80002F1200201FA02FCC2F1200250EA4C00B4
:101BC80021FA02F243EB020008BF20EADC707047FA
:101BD8004FF0FF0C1CEAD0521EBF1CEAD15392EA08
:101BE8000C0F93EA0C0F6FD01A4480EA010C4002E4
:101BF80018BF5FEA41211ED04FF0006343EA50103E
:101C080043EA5111A0FB01310CF00040B1F5000F7F
:101C18003EBF490041EAD3715B0040EA010062F12E
:101C28007F02FD2A1DD8B3F1004F40EBC25008BF18
:101C380020F00100704790F0000F0CF0004C08BF36
:101C480049024CEA502040EA51207F3AC2BFD2F103
:101C5800FF0340EAC250704740F400004FF0000311
:101C6800013A5DDC12F1190FDCBF00F0004070474B
:101C7800C2F10002410021FA02F1C2F1200200FA89
:101C880002FC5FEA310040F1000053EA4C0308BF50
:101C980020EADC70704792F0000F00F0004C02BFA1
:101CA800400010F4000F013AF9D040EA0C0093F01C
:101CB800000F01F0004C02BF490011F4000F013B76
:101CC800F9D041EA0C018FE70CEAD15392EA0C0FE4
:101CD80018BF93EA0C0F0AD030F0004C18BF31F04F
:101CE800004CD8D180EA010000F00040704790F025
:101CF800000F17BF90F0004F084691F0000F91F0C9
:101D0800004F14D092EA0C0F01D142020FD193EA8E
:101D18000C0F03D14B0218BF084608D180EA010016
:101D280000F0004040F0FE4040F40000704740F0F2
:101D3800FE4040F4400070474FF0FF0C1CEAD052C0
:101D48001EBF1CEAD15392EA0C0F93EA0C0F69D01C
:101D5800A2EB030280EA010C49024FEA402037D087
:101D68004FF0805343EA111143EA10130CF000407E
:101D78008B4238BF5B0042F17D024FF4000C8B426E
:101D880024BF5B1A40EA0C00B3EB510F24BFA3EB4E
:101D9800510340EA5C00B3EB910F24BFA3EB91031E
:101DA80040EA9C00B3EBD10F24BFA3EBD10340EA78
:101DB800DC001B0118BF5FEA1C1CE0D1FD2A3FF6BE
:101DC80050AF8B4240EBC25008BF20F00100704773
:101DD8000CF0004C4CEA50207F32C2BFD2F1FF0316
:101DE80040EAC250704740F400004FF00003013A47
:101DF80037E792F0000F00F0004C02BF400010F4EB
:101E0800000F013AF9D040EA0C0093F0000F01F0FE
:101E1800004C02BF490011F4000F013BF9D041EA20
:101E28000C0195E70CEAD15392EA0C0F08D1420253
:101E38007FF47DAF93EA0C0F7FF470AF084676E726
:101E480093EA0C0F04D14B023FF44CAF08466EE7FF
:101E580030F0004C18BF31F0004CCAD130F00042CD
:101E68007FF45CAF31F000437FF43CAF5FE700BF25
:101E78004FF0FF3C06E000BF4FF0010C02E000BF4E
:101E88004FF0010C4DF804CD4FEA40024FEA4103F0
:101E98007FEA226C18BF7FEA236C11D001B052EAA6
:101EA800530C18BF90EA010F58BFB2EB030088BF6C
:101EB800C81738BF6FEAE17018BF40F001007047DB
:101EC8007FEA226C02D15FEA402C05D17FEA236CBD
:101ED800E4D15FEA412CE1D05DF8040B704700BF04
:101EE800844608466146FFE70FB5FFF7C9FF00289B
:101EF80048BF10F1000F0FBD4DF808EDFFF7F4FFD4
:101F08000CBF012000205DF808FB00BF4DF808ED6C
:101F1800FFF7EAFF34BF012000205DF808FB00BF8F
:101F28004DF808EDFFF7E0FF94BF012000205DF8B1
:101F380008FB00BF4DF808EDFFF7D2FF94BF012062
:101F480000205DF808FB00BF4DF808EDFFF7C8FF5B
:101F580034BF012000205DF808FB00BF42000ED20C
:101F6800B2F1FE4F0BD34FF09E03B3EB126209D4CC
:101F78004FEA002343F0004323FA02F070474FF082
:101F88000000704712F1610F01D1420202D14FF0F7
:101F9800FF3070474FF00000704700BF00F026F890
:101FA8000C4880F30888002103E00B4B5B58435032
:101FB80004310A480A4B42189A42F6D3094A02E009
:101FC800002342F8043B084B9A42F9D313F010FF60
:101FD8007047000000C000203CB402080000002048
:101FE800180E0020180E0020F83100207047FEE778
:101FF80010B586B0002301244FF46022114801A9CE
:1020080001938DF80930039204938DF808408DF8F8
:1020180014401CF09BF90B4821461CF0BDF90948F7
:102028001CF0C4F907481CF0C6F90028FAD1054885
:102038001CF0C5F903481CF0C7F90028FAD106B00E
:1020480010BD00BF00240140014610B50D48012213
:1020580003231CF0C7F90B4801211CF0B9F97F20B4
:102068001CF0F6FF074802211CF006FA0028F6D0FB
:10207800044802211CF006FA0248BDE810401CF092
:10208800F8B900BF002401400C4A0C2303FB0123CC
:1020980010B59C880CB9588010BD5B8803F11304F7
:1020A800844204DA142B07D9133B834204DC0C2343
:1020B80003FB012102238B8010BD00BFF81B002009
:1020C8000A4B10B500241C7021464FF48072084852
:1020D800FEF760F9074B43F6DE301C70064B1C70A8
:1020E8000DF060F9054B187010BD00BF8810002076
:1020F80090110020A71200209312002095120020B2
:10210800074B1978013101F01F011970054B1A7836
:102118008A4203D1013202F01F021A70704700BFD1
:1021280093120020A712002010B50A4B0A4A03EBAD
:10213800C0000A4B1978036802EBC10442F8313039
:102148004368002163600822FEF724F9BDE81040C7
:10215800FFF7D6BF8C1000209011002093120020AA
:102168002DE9F3479846474B1746DA78054602F0BB
:102178002002D2B20E46BDF82890002A7AD1B8F1D2
:10218800000F0AD19B7803F04003DBB2C3B900F01B
:102198007F0000F56E50633009E0B8F1010F09D1F6
:1021A8009B7803F04003DBB2BBB949F2D8400DF08D
:1021B800F9F8C4B2002C5FD0B8F1000F09D100E0E3
:1021C800012405F07F0149000DF1060001F5715168
:1021D8000CE0B8F1010F0CD100E04446E90101F52B
:1021E8000A41D8310DF1060001EB460102220DF03B
:1021F800EAF8BDF9063013B9B8F1000F3ED0B9F1CD
:10220800000F06D1204B93F800A0FFF779FF1F4B72
:1022180008E01F4B93F800A00AF1010202F01F0228
:102228001A701C4BB8F1000F12D1BDF8061040F619
:10223800B8326DB212EA250538BF4FF47A756D18B9
:1022480003EBCA0223F83A509470D670177109E06C
:10225800B8F1010F06D1BDF8061003EBCA0223F846
:102268003A10947003EBCA0383F80580A3F806902C
:10227800012004E0002002E0204600E04046BDE8DE
:10228800FC8700BFEC23002093120020901100204F
:10229800871000208C10002001228240094B0A4937
:1022A8001B78D2B2097808E0084800EBC3008078B0
:1022B800024205D1013303F01F038B42F4D1FF23FF
:1022C80018467047A7120020931200209011002092
:1022D800F0B500EB800101F56E51314F042285B055
:1022E800304836310DF06FF82F4C3B7804EBC302C1
:1022F80056791EBB2B4D31222A7107326A7134F987
:10230800331001A8343A05F0FFFD3B7802A804EB2E
:10231800C3031979022205F0F7FD3B780DF10A0095
:1023280004EBC304E178032205F0EEFDA81D01A922
:102338000922FEF705FB2E740F250CE0012E0AD1A9
:10234800184A322111710531517134F8333008259A
:10235800190AD1719371002314481A4612E010F833
:10236800011FA1F13004E4B2092C04D8E318302984
:10237800DBB203D004E037395B1800E00A33DBB284
:102388000132D2B2AA42EAD10F21B3FBF1F108011E
:10239800411A5B1A0348C3F10F03835405B0F0BD1B
:1023A8008D11002096120020901100209512002017
:1023B8002DE9F3415F4B04461B7843B15E4B1B7814
:1023C80003F02403042B02D1002900F0AF805B4BFB
:1023D8005B4F1B78002B00F093805A4821461BF076
:1023E80061F98046002840F08B803B1993F8303023
:1023F8002D2B01D0532B2DD1534E3578F5B10DF03F
:10240800D9FA611C034630B1337893201E33009308
:102418000122002302E0009001229320FFF7A0FE92
:102428000DF0C8FA014628B1337813201E33009303
:10243800002101E0009013200A465EE0611C0122A1
:1024480093202B460095FFF78BFE00951320294615
:102458002A4652E0542B05D10090611C9420012299
:1024680043464BE0462B384D11D12E7866B10DF01E
:10247800A1FA611C034620B12B789A201E330093E1
:1024880014E000909A2018E000969A202CE02E780C
:1024980026B30DF08FFA0346611C04F11C0043B10A
:1024A8002B7860F07F001E330093C0B201224346B0
:1024B80004E060F07F000093C0B20122FFF750FEF5
:1024C8000DF078FA21B2024628B12B7803201E338A
:1024D8000093002211E0009003200EE004F11C009C
:1024E80060F07F000096C0B2611C01223346FFF7FE
:1024F80037FE00960320214632460123FFF730FEBF
:10250800104821463F191BF0B7F897F83030542B84
:102518000CD8532B03D22D2B01D0462B06D10B48B8
:10252800214602B0BDE8F0411BF0B1B802B0BDE8E9
:10253800F08100BF8A100020E213002094120020CE
:102548002C1B0020EA1300200B140020E7130020A6
:1025580037B5114B04461B780D4693B10F482146F9
:102568001BF0A0F8034660B9012D04F1010103D165
:1025780000902A46812002E0009001229820FFF76F
:10258800EFFD214605481BF077F80548214603B0C2
:10259800BDE830401BF07BB894120020EA130020FD
:1025A800AE120020024B1A7842F001021A707047EE
:1025B800A914002008B50C4B1A780C4B03EBC20386
:1025C800597921B101290CBF0921002100E010210E
:1025D80040221346064805F0BBFA064B1A7842F02B
:1025E80002021A7008BD00BF8D1100209011002052
:1025F80096120020A9140020034B1A7802F0F80262
:102608006FF3C3021A707047A9140020024B1A789E
:1026180042F004021A707047A9140020024B1A787D
:1026280042F008021A707047A914002038B5114BFF
:102638001C7814F0010502D1FFF7B4FF05E004F09F
:102648000405EDB21DB9FFF7E1FF284638BD04F0D7
:102658000805EDB215B9FFF7E1FFF6E704F002044B
:10266800E4B21CB9FFF7A6FF204638BDFFF7C4FF48
:10267800012038BDA9140020014B1878704700BF0D
:102688008810002030B50F4B85B01B780546BBB9C4
:102698000D4C2278024112F0010F11D0FF22019354
:1026A8000121431C009202933C200B46FC3A0CF09B
:1026B800EDFE012313FA05F5237823EA05052570B5
:1026C80005B030BD95120020911200202DE9F84385
:1026D800134A00231370134A1678134A1178904648
:1026E800B14219D0114D2A78072A88BF2B7095F866
:1026F80000902C780D4F2046FFF7CEFDFF280CD117
:102708000134E4B2072C3C7001D900233B702B78CC
:102718004B45EED188F80060FF242046BDE8F883D9
:1027280088100020A7120020931200208E1100208C
:102738000121814010B5C943C9B20023094A9A183A
:102748009478083301EA0404B3F5807F9470F5D1D6
:10275800FFF798FF43F6DE300CF024FE024B1870AA
:1027680010BD00BF90110020951200202DE9F04106
:102778008B4E054633788B4C13B12378834204D0B3
:1027880043F6DE300CF00EFE30702570864C237850
:10279800072B00F2E680DFE813F008002000330082
:1027A80051005A0070008B00B500804B1E221A7031
:1027B8002846FFF771FD7E4BFF28187000F0D58082
:1027C8001AF0C2FA7B4B002093F8702042F0010205
:1027D80083F87020784B187065E0744B1B78002BD9
:1027E80000F0C3801AF0FCFB012840F00D8123782B
:1027F800142201332370714B01381A70BDE8F0813F
:102808006A4B1B78002B00F0B0806C4E307808B90A
:1028180001234AE01AF0E4FB022804D01AF0E0FB96
:10282800032840F0F1801AF08FFA2378042201334C
:1028380023701D233370624B1A70E5E05B4B1E2238
:102848001A702846FFF744FD237801332370574B4D
:102858001B78002B00F08980584B1D78002D40F024
:10286800D3801020FFF7E2FE002800F0D180237803
:10287800284601332370BDE8F0814C4B1B78002BB0
:1028880073D005F0CFF9002800F0C2804B4B7D22B1
:102898001A70494B00201870464B93F8702042F08C
:1028A800010283F87020237801332370BDE8F0819A
:1028B8003E4B1B78002B58D01AF092FB01283F4F53
:1028C80003D01AF08DFB03280DD1012212FA05F569
:1028D8003C4B1A7822EA05051D7064233B70237867
:1028E8000133237090E03878002840F08D80344A16
:1028F800032323701378013BDBB21370002B34D011
:10290800BDE8F0812B4B2D4F93F86A3013B13B781B
:10291800002B79D100233B700133AB40244A2A486D
:102928001178904600EBC10090F802E02EEA03030C
:1029380083703BB9254B1A788A4203D1013202F0E1
:102948001F021A702846FFF7A7FC1D4B0422FF2818
:1029580088F800001A703FD0032323701A333B70A5
:1029680052E000202070BDE8F081FFF745FE00230B
:1029780023701AF0E9F93378013BDBB2337033B1D5
:10298800134B9B7803F04003DBB2002B3FD0284663
:10299800FFF7CEFE0F4B1A7801321A7031E000BFF4
:1029A800951200208B100020881000209212002021
:1029B8008D1100200226002089100020861000209A
:1029C800901200209112002090110020A7120020E0
:1029D800EC2300208E1100200E4B9A7802F0400262
:1029E800D2B21AB11A6842F400021A60FFF704FE64
:1029F8001AF0AAF90023237043F6DE300CF0D2FC5B
:102A08003070FF20BDE8F0810020BDE8F081FF2094
:102A1800BDE8F081EC230020044B1A780AB1013A92
:102A28001A701B780BB9FFF783BE70479512002008
:102A3800044A054B10781B7803EA501000F0010097
:102A4800704700BFEC230020CF130020044B054A39
:102A58001B781078C3F3400303EA1010704700BFD7
:102A6800CF130020EC230020034B044A1B78D078B6
:102A7800C3F3800318407047CF130020EC230020D5
:102A8800044B054A1B78D078C3F3C00303EA50000F
:102A9800704700BFCF130020EC230020044B054AE9
:102AA8001B78D078C3F3001303EA9000704700BF87
:102AB800CF130020EC230020044B1878044BDB785C
:102AC8005B005BB2DB1103EAD0107047CF13002024
:102AD800EC2300202DE9F041154E0024B04620E0FB
:102AE8002046294617F07EFA90B1F35DFF2B0FD0F0
:102AF8004FF4A07363430A2202FB053318F803302E
:102B0800DB0905D00B4B1878C0F30010BDE8F08145
:102B180001350A37202DE3D10134022C06F5A076C1
:102B280002D000273D46DBE70020BDE8F08100BF6A
:102B38004E270020CF13002008B516F099FE034B4E
:102B48001B7800EA931000F0010008BDCF130020A5
:102B5800044B054A1B78D078C3F3401303EAD0002E
:102B6800704700BFCF130020EC2300202DE9F84F59
:102B7800FFF75EFF8146FFF769FF8246FFF774FFA4
:102B88008346FFF77DFF8046FFF788FF0446FFF77F
:102B9800A1FF0546FFF7DCFF0746FFF7CDFF064616
:102BA800FFF78AFF4FEA8B0343EA4A0343EA090324
:102BB80043EAC80343EA471343EA861345EA040491
:102BC80043EAC013E0B243EA0010BDE8F88F000002
:102BD800044B987800F00F00A0F10203584240EB34
:102BE80003007047D2120020044B987800F00F00C1
:102BF800A0F10102504240EB02007047D2120020BF
:102C0800044B987800F00F00A0F10301484240EB14
:102C180001007047D2120020054B987800F00F0091
:102C2800A0F1060CDCF1000040EB0C00704700BF7F
:102C3800D2120020514AF0B513781446012B29D03E
:102C480003D3022B40F098805EE04D484D4B04784A
:102C580019786FF3C304047001F0F80158786FF322
:102C6800C301197000F08001C9B2002900F0848006
:102C7800012111709C78062204F00F045443024687
:102C88004148005D60F306025A701A7861F3020247
:102C98001A70F0BD3B494D780B4625F07F0000289F
:102CA80038D00A7802F00802D2B222B9344A117830
:102CB80041F0080111709A7802F00F02012A04D13C
:102CC8002F4A117841F00101117015F07F0F53D18F
:102CD80019789E7801F00700062206F00F0602FB1D
:102CE8000606294F5D78BE5D013066F3060500F0E3
:102CF80007005D7090FBF2F502FB150262F302011A
:102D0800197002232370F0BD1E494D780B4625F03B
:102D18007F0028B98B7860F303038B701070F0BDC7
:102D2800174A11786FF3C3011170997801F00F01F8
:102D3800012903D111786FF30001117015F07F0F8D
:102D48001AD119789E7801F00700062206F00F06BE
:102D580002FB06060C4F5D78BE5D013066F3060582
:102D680000F007005D7090FBF2F502FB150262F3BC
:102D78000201197001232370F0BD00BFF412002076
:102D8800AD120020D2120020F8F0010808B543F671
:102D9800ED200CF007FB014B187008BDAC120020A9
:102DA800014B1870704700BFD3130020024B1A5C08
:102DB8006FF303021A5470471713002070B50C46BE
:102DC800C10001F5CC411248683103220CF0FBFA2E
:102DD80000250F482946EEB21AF064FC98B10D4B55
:102DE8002278EB5C1A420ED13046FFF7DFFF294606
:102DF80009481AF04CFCF608074B06F5CA40A830FB
:102E0800995D0CF0C5FA0135182DE2D170BD00BFEF
:102E1800D5130020FB120020D512002038B546F249
:102E2800F05540242046FFF7C1FFA5F5CA43094ADB
:102E3800B03BD15C11F0100F06D06FF30411D154E0
:102E4800284600210CF0A4FA0134E4B20135B82C6C
:102E5800E8D138BD171300207FB58F4B05461B7886
:102E6800002B00F011818D4E325C541C04F00F04CD
:102E780064F30302172832542AD8002C00F0098181
:102E880001339C4240F00281D3B26FF30303335401
:102E9800834BC4081B1993F8962000F0070352FAD5
:102EA80003F313F0010F40F0F38029467D481AF030
:102EB800E3FB7C4B04F5CA40195DA83001240CF0F3
:102EC80067FA2D1902230093019402951820C4E093
:102ED8003F2840F2DB80002C00F0DB8001339C426D
:102EE80040F0D480335C01216FF30303335400F5C1
:102EF800CA40B0300CF04CFA735D43F010037355C0
:102F0800A5F14003DBB2032B07D80422009201335A
:102F180002320192029319202FE0A5F14803DBB297
:102F2800032B07D804220092013303320192029343
:102F38001A205EE0A5F15003DBB2012B07D804226A
:102F4800009201330332019202931B2051E0572D66
:102F580007D1042300930124033301930294212011
:102F68007BE0A5F15B03DBB2012B09D804220092B8
:102F7800013302320192029322200121033A7FE0B9
:102F88005D2D04D1042300930193043B06E05E2DDC
:102F980007D10423009301330193053B029328468C
:102FA8006CE0A5F15F03DBB21F2B09D80422009265
:102FB800013392180192029333200121053A5FE010
:102FC80005F16103DBB2032B07D804220092013319
:102FD8000332019202935F200BE005F15903DBB243
:102FE800012B09D804220092013303320192029383
:102FF80060200121043A43E0AA2D07D1042300935D
:103008000124043B01940293612026E0A92D07D1F5
:1030180004230093023B0193023B029362202DE0BC
:10302800AC2D08D1042300930322043B01920293A0
:103038006320012124E0AB2D06D104230093043B37
:1030480001930293642019E0AD2D0CD10423009361
:103058000124023301930294682021460322234667
:103068000CF014FA15E04F35EDB2012D10D80423F9
:10307800009301350233019302956A20012103224E
:103088000B460CF003FA03E01C4602E0002400E0C3
:103098000124204604B070BD000000201713002052
:1030A8002C1B0020D5120020024B185CC0F3001026
:1030B800704700BF17130020F8B503220E46002101
:1030C8000746FDF767F946F268650024337823411F
:1030D80013F0010F08D02946064803220CF073F9B3
:1030E800384604491AF087FA01340835042CEDD122
:1030F800F8BD00BFDA130020024846F2A8510322A7
:103108000CF061B9D512002070B5044600F56A507C
:1031180044300CF047F90B4D06462B7813F0010F9D
:1031280002D1CC201BF0A8F82B8843F001032B8098
:10313800054B1E55054B13F8242042F0010203F8F5
:10314800242070BDE2130020C5120020B412002014
:10315800024B185C084100F001007047FB12002088
:1031680070B505460024094BE0B2E618E35C4BB1A4
:103178002946FFF7EDFF28B10023337004482146A4
:103188001AF085FA0134182CEDD170BDF013002027
:10319800CC12002038B5054600242846E1B2FFF7D6
:1031A800D7FF10B1044BE35C23B90134042CF4D1EC
:1031B800002038BD012038BDC512002038B50546AD
:1031C8000CF0F8FBA0B100242846E1B2FFF7C0FFDD
:1031D80040B1084B13F8243013F0010F02D0064B0E
:1031E800E35C23B10134042CEED1002038BD01206A
:1031F80038BD00BFB4120020C5120020F8B5114830
:1032080000211822FDF7C6F846F268650024012758
:103218000D4829460322A7400CF0D5F8FFB2002636
:10322800094831461AF03EFA20B1064BF25C47EAEB
:103238000202F2540136182EF2D101340835042C5A
:10324800E5D1F8BDFB120020DA1300202DE9FF417B
:1032580000263446B0461A4B1B78234113F001026E
:10326800184B23D0184F1D5D17F82430A84538BFD8
:10327800A84613F0010F1AD0CDB965F3000307F87B
:10328800243023B20122F71902935B2029462B46EA
:10329800009201950CF0FAF87B78B878F978184321
:1032A800621C2B460095FEF75BFF00E01A550134BF
:1032B8000436042CCFD1054B83F80080BDE8FF818C
:1032C800AC120020C5120020B4120020AB1200205E
:1032D80010B50C4B1B78A3B10B4B1B788BB100249A
:1032E8000A4821461AF0DEF940B1094821461AF089
:1032F800D9F918B920460121FFF75AF80134182CDA
:10330800EED110BD941200208A100020E71300208F
:10331800861800202DE9F043364D374A2B880026C1
:103328006FF386136FF3C4032B80344B344F85B08F
:1033380016701E709146984617F8013B5BB32A78C1
:10334800D20052B243EAA2122B88182E62F3C403A9
:1033580043F040032B801ED000243046E1B2FFF733
:10336800F7FEA8B117F8013C13F0010F06D00122AF
:10337800A24099F800100A4389F8002013F0020FC0
:1033880006D00123A34098F80020134388F80030A2
:103398000134042CE1D10136F6B2192ECCD12B78A8
:1033A80003F04004E4B20CBB03F02403042B12D155
:1033B800FFF78EFFFF23009340202146012223467A
:1033C800019402940CF062F88020214601222346E1
:1033D8000094FEF7C5FE2B8800226FF345136FF3A8
:1033E80082036FF3C4032B80064B1A7005B0BDE847
:1033F800F08300BFE2130020FC24002019250020E0
:10340800DB120020D413002010B500240548214603
:103418001AF048F908B9044BE0540134182CF5D1D6
:1034280010BD00BFD0130020DB12002070B5164677
:103438000D46317804469DF81020002925D0002B30
:1034480023D012B111491AF0CBF80121204609F016
:10345800FDFD20462946324609F0D0FDACB10322D5
:1034680046F2A8510A480BF0AEFF214608481AF068
:10347800C2F80749032246F2A8500BF09EFF054800
:103488000349BDE870401AF0D7B870BDC51B0020CD
:10349800A8120020D512002030B5064B04781D78FC
:1034A80024EA05040C7001781B7823EA01031370E1
:1034B80030BD00BFAC12002038B50A4D002415F805
:1034C800013F2D2B09D0532B07D0542B05D0462B69
:1034D80003D0054821461AF0DAF80134182CEED149
:1034E80038BD00BF5B1B0020E713002010B50D4856
:1034F8001AF06EF800240C4821461AF0D3F868B187
:103508000A4BE31893F83030462B03D0542B01D0E4
:103518002D2B03D1034821461AF0AEF80134182C9C
:10352800E9D110BDF5120020E71300202C1B002064
:10353800094A0A4B117831B1997801F00F0181429B
:1035480001D0002111709A7860F303029A705A78BA
:1035580042F080025A707047F4120020D212002004
:103568007FB5604B154604461A780E4600235E491F
:1035780011F8231011F0010F05D001219940C1F174
:103588000F0101EA02020133042BF0D1574B1A70E4
:10359800002C6FD014F0010F0AD0FF2301210093F3
:1035A800FF3B0193029352200A460B460BF06EFF35
:1035B80014F0020F0AD0FF2301210093FF3B01936F
:1035C800029353200A460B460BF060FF14F0040FD9
:1035D8000AD0FF2301210093FF3B0193029354205B
:1035E8000A460B460BF052FF14F0080F0AD0FF23CF
:1035F80001210093FF3B0193029355200A460B4695
:103608000BF044FF14F0100F0AD0FF2301210093A0
:10361800FF3B0193029356200A460B460BF036FFF8
:1036280014F0200F0AD0FF2301210093FF3B0193E0
:10363800029357200A460B460BF028FF14F0400F60
:103648000AD0FF2301210093FF3B019302935820E6
:103658000A460B460BF01AFF14F0800F0AD0FF231E
:1036680001210093FF3B0193029359200A460B4620
:103678000BF00CFFCEB10024284621461AF012F8B0
:1036880060B1FF230093FF3B0193631C1BB2012130
:1036980002935A200A460B460BF0F8FE21462846AC
:1036A800013419F0F4FF182CE6D110481049114ADA
:1036B800FFF7F2FE104B00221A7001320092063218
:1036C8000192083202920A490A4A084809F048FC5D
:1036D8000A4B3C2251201A7004B0BDE870400CF02F
:1036E8004FBA00BFAC120020B412002014150020FD
:1036F8007A1500206E150020D9140020C41200206D
:1037080010B5FFF733FA0446074819F09AFFD0F1CD
:10371800010138BF002104B929B1034A2046BDE898
:103728001040FFF71DBF10BD14130020054B03EB1D
:10373800D00393F8963000F0070053FA00F000F039
:10374800010070472C1B002010B50C4B04461B7859
:1037580013F001030FD0FFF71DFD68B10CF02AF933
:1037680018B92046FFF7E2FF30B10548214619F0A5
:1037780083FF012010BD184610BD00BFE2130020D2
:1037880014130020024B1878003818BF0120704726
:10379800C412002010B5034C04EB830358709970D1
:1037A800DA7010BDB412002010B5002409480021B9
:1037B800001908220834FCF7EDFDB4F5807FF5D137
:1037C800054A00231370054A002199520233AA2B97
:1037D800F9D110BD8C10002087100020EE150020B4
:1037E8007FB5444B04461B780E46AA2B74D042483A
:1037F800214619F057FF054600286DD12046FFF7EE
:10380800A3FF002869D13D48214619F04BFF50B964
:103818003B48214619F046FF054620B92046FFF7E8
:103828001BFB002859D1374B1B7823B9364B1B7823
:1038380013F0010F08D1354BDB7803F02003DBB21E
:1038480013B9334B03221A76012E05D82B4821468B
:1038580019F028FF40B13FE0022E07D12848214641
:1038680019F020FF10B137E0244800E02448214631
:1038780019F002FF2748214619F009FF022E12D13C
:10388800012564194A20294603222B4600960195F2
:1038980002940BF0FBFD0023182021462A460093D2
:1038A800FEF75EFC19E0012E09D102230093631C88
:1038B80002930196122031460322334609E07EB96D
:1038C800012102230093631802930191112003221E
:1038D8000B460BF0DBFD03E00025284604B070BD65
:1038E800012000232118024600930125FEF738FC29
:1038F800F3E700BFD3130020D5120020AE1200203A
:1039080008140020AC120020EA150020EC23002047
:10391800DB120020EA1300202DE9FF4704460D467C
:103928006148214619F0BEFE8046002840F0B88064
:1039380021465D4819F0A0FE5C48214619F0A7FE13
:103948005B4E0DBB012708F10208E31902934246BA
:10395800032039463B46CDF8008001970BF096FDD1
:10396800327862B10CF026F8024630B1337840461E
:103978001E33009321462A4604E0009000E000929E
:10398800404621463B461CE0012D1FD1631C022204
:1039980002930E2029462B46009201950BF076FDE6
:1039A80032788AB10CF006F8024630B133780D202F
:1039B8001E3300932146424602E000900D20214626
:1039C8002B46FEF7CDFB50E00092F7E7022D0AD117
:1039D80001216318029314202A4643460095019159
:1039E8000BF054FD41E0032D3FD101272A464FF04B
:1039F800020904EB070A4D2039463B46CDF80090F2
:103A08000197CDF808A00BF041FD3578EDB10BF02A
:103A1800D1FF024630B1337848461E330093214621
:103A2800424602E00090214648463B46FEF798FB96
:103A38000BF0C0FF611C034620B133781A201E33F7
:103A480000931FE000901A2020E021462A463B46BA
:103A580048460095FEF784FB1A2051463A462B4605
:103A68000095FEF77DFB38461BE033789BB10BF0E1
:103A7800A1FF0346611C04F11C0033B10C4B1B78F9
:103A88001E3300930122002301E000930122FEF778
:103A980067FB012005E0009304F11C00611CF5E7B9
:103AA800002004B0BDE8F087E7130020EA130020E7
:103AB8000B140020064B1B1893F87800492804D0F3
:103AC800452814BF0320022070470120704700BF1B
:103AD8002C1B00202DE9F041244F00243C70244881
:103AE800214619F0DFFDE5B2224B002837D01E5DD4
:103AF8003B789E4200D303B93E70002E30D1314648
:103B08001C481822FCF746FC1B4B1C4803EBD5034A
:103B180093F8938004F0070348FA03F8214608F065
:103B2800010819F0BFFD68B9B8F1000F02D02846A6
:103B3800022101E028463146FFF7EEFE28460CF048
:103B48001FF80DE0B8F1000F0AD12846FFF7B2FFC1
:103B58000B4BDB7803F02003DBB20BB9094B18558C
:103B68000134182CBBD1BDE8F08100BF0B14002034
:103B7800CC120020F01300202C1B0020E71300209B
:103B8800EC230020DB1200202DE9F04F8F4B89B089
:103B98001B7813F0010F06D08D4B1A786FF386123D
:103BA8001A7001F034BA8B498B4A0B7810788B4D18
:103BB800984218BF8A49137018BF0B706B7803F0CE
:103BC8000803DBB24BB143F6CF200BF0EBFB844B81
:103BD80018702B886FF3CB232B80824B1B78AA2B72
:103BE80008D18149AA3B0B702B8843F080032B80B6
:103BF80000F088BE6A78794B02F01002D2B27B4C92
:103C08009AB11A886FF30C321A80794B1B7823B952
:103C1800784B1B7813F0010F07D1E37803F02003EA
:103C2800DBB213B9744B03221A762368734F6FF310
:103C3800186323603A7802F00202D2B232B96A49B4
:103C48004A781AB1694A43F080731360E67816F02F
:103C5800010647D05D20FFF727FA002859D16B7875
:103C6800DFF8788103F00203DBB22BBB5D30FFF78E
:103C7800F3F8064600BBB8F80030012143F400739E
:103C8800A8F80030042303220093019302900B4606
:103C98000D200BF0FBFB45200BF072FF3146012293
:103CA80033460D200096FEF75BFA0920314632466E
:103CB80001230096FEF754FA6B7803F00203DBB297
:103CC8003BB34B4B1B7823B94A4B1B7813F0010FBE
:103CD8001FD1E37803F02003DBB2D3B9464B0322AC
:103CE8001A7616E06B7803F00203DBB26BB131464B
:103CF800324601230A200096FEF732FA8D2031461B
:103D0800012233460096FEF72BFA2B886FF34923DE
:103D18002B802368344A6FF35963236093787BB10F
:103D2800D37823B93B7813F00C0F05D108E03B7822
:103D380003F00C03042B03D0236843F000732360C3
:103D4800E17801F00201C9B2002959D05E20FFF7DD
:103D5800ABF9002863D16B78204F03F00403DBB282
:103D6800EBB95E30FFF778F80646C0B93B88012109
:103D780043F480633B8004230093013303220193BF
:103D880002900B4617200BF081FB45200BF0F8FE44
:103D98000D203146012233460096FEF7E1F96B7893
:103DA80003F00403DBB2002B39D0114B1B7823B985
:103DB800104B1B7813F0010F31D1E37803F0200387
:103DC800DBB263BB0C4B03221A7628E015150020E2
:103DD80060250020D8130020D9130020E21300200A
:103DE8000C140020D3130020180E0020EC23002010
:103DF800AC120020EA150020DB120020271B00204F
:103E08006B7803F00403DBB22BB18D2001220B4643
:103E18000091FEF7A5F92B886FF38A232B8023687E
:103E2800DFF8CCB26FF3DF7323605F2306930026BD
:103E3800D94695E03046394616F0D4F8002870D0B7
:103E48001BF80A30FF2B6CD04FF4A0727243A8F114
:103E58005E03DBB207930A2303FB072219F802E08B
:103E680009EB02035FEADE1E4FD02268404642F0AB
:103E7800004222600593FFF717F9059B00285BD1E4
:103E88001A7912F0040F24D14046FEF7E5FF059B8E
:103E98008446F0B91A79322042F004021A7107995F
:103EA800042300930291DB180121032201930B469E
:103EB800CDF814C00BF0EAFA4A200BF061FEDDF8E9
:103EC80014C00C20079901226346CDF800C0FEF704
:103ED80047F94FF4A07373430A2202FB07334B449C
:103EE8001B7913F0040F27D07C4B1B7823B97C4B2C
:103EF8001B7813F0010F1FD1E37803F02003DBB226
:103F0800D3B9784B03221A7616E01B7913F0040F05
:103F180007D08C20079901227346CDF800E0FEF700
:103F28001FF94FF4A07373430A2202FB07334B4473
:103F38001A796FF382021A71013708F10108202FEC
:103F48005FFA88F80AF10A0A7FF474AF069A013614
:103F580002F12003DBB2022E0BF5A07B069305D0FD
:103F68004FF0000ADDF81880574663E723685E497A
:103F780023F080636FF39E7323600B79002B00F0AE
:103F88001384DFF870A1DFF870B14FF09F080027A5
:103F98001AF8011F3E46013700294FD02368A8F1BF
:103FA8005F0943F080635FFA89F923604846FFF7A9
:103FB8007BF8002858D14D4A122303FB0623997831
:103FC80011F0200F21D148460593FEF745FF059BC8
:103FD8008146D0B99A78012142F020029A700423D0
:103FE8000093023301933BB2032202930F200B4646
:103FF8000BF04CFA45200BF0C3FD0D204946012279
:104008004B46CDF80090FEF7ABF83849122303FB76
:1040180006139B7813F0200F26D0304B1B7823B95A
:104028002F4B1B7813F0010F1ED1E37803F0200308
:10403800DBB2CBB92B4B03221A7615E02B4B12229D
:1040480002FB06329278994612F0200F05D08D2097
:1040580001220B460091FEF783F8122303FB069317
:104068009A786FF345129A701BF8011F002945D002
:104078002368404643F080432360FFF715F8002883
:1040880052D11A4B4FF0120909FB063999F8023040
:1040980013F0400F48D14046FEF7DEFE06460028E2
:1040A80042D199F80230012143F0400389F80230E7
:1040B80004230093033301933BB2032202934B2062
:1040C8000B460BF0E3F950200BF05AFD192031464E
:1040D800012233460096FEF743F825E0AC12002093
:1040E800EA150020DB120020180E0020AF24002063
:1040F8004E270020A7240020822400209B4B122258
:1041080002FB06329278994612F0400F05D09920AA
:1041180001220B460091FEF723F8122303FB0696B3
:10412800B3786FF38613B37008F10108042F5FFAB0
:1041380088F87FF42DAF8E4BDFF84CB206934FF022
:104148005008043F1BF8011F3E460137002951D093
:10415800236808F1610A43F080635FFA8AFA2360F2
:104168005046FEF7A1FF00285BD13301DFF81C920F
:104178009B1B19F8032012F0400F23D150460593DA
:10418800FEF76AFE059B8246E0B919F80320012173
:1041980042F0400209F803200423009302330193FC
:1041A8003BB20322029369200B460BF06FF94520BE
:1041B8000BF0E6FC0D20514601225346CDF800A035
:1041C800FDF7CEFF33019B1B19F8033013F0400FA6
:1041D80027D0684B1B7823B9674B1B7813F0010F66
:1041E8001FD1E37803F02003DBB2D3B9634B03227A
:1041F8001A7616E03301DFF894919B1B19F8033007
:1042080013F0400F05D08D2001220B460091FDF7D9
:10421800A7FF33019B1B19F803206FF3861209F8D7
:104228000320069A12F8011F0692002935D0236848
:10423800404643F080432360FEF736FF002843D111
:10424800DFF848A14FEA0619C6EB09091AF8093040
:1042580013F0200F38D14046FEF7FEFD064698BB06
:104268001AF80930012143F020030AF80930042321
:104278000093033301933BB20322029310200B46B1
:104288000BF004F950200BF07BFC19203146012279
:1042980033460096FDF764FF16E03301DFF8EC9033
:1042A8009B1B19F8033013F0200F05D09920012229
:1042B8000B460091FDF754FF33019E1B19F8063099
:1042C8006FF3451309F8063008F10108022F5FFA69
:1042D80088F87FF437AF2A4B1978002958D023681B
:1042E800AD2043F080632360FEF7DEFE00285ED138
:1042F800244B1A78984612F0400F20D1AD30FEF7C3
:10430800ABFD0746D8B998F80030012643F04003C2
:1043180088F80030042300930233314603220193C6
:104328006720334602960BF0B1F845200BF028FCC5
:104338000D20394632463B460097FDF711FF98F8A5
:10434800003013F0400F32D00A4B1B7823B90A4BC8
:104358001B7813F0010F2AD1E37803F02003DBB2B6
:104368002BBB064B03221A7621E000BFAF240020A6
:10437800EF230020AC120020EA150020DB120020F9
:1043880024240020382400207224002055240020F2
:104398009E4E337813F0400F05D08D2001220B4636
:1043A8000091FDF7DDFE33786FF386133370984B79
:1043B800197800292DD02368572043F080432360C3
:1043C800FEF772FE002833D1904E337813F0200F99
:1043D8002ED15730FEF740FD074648BB33780322FD
:1043E80043F020033370042301260093033331463E
:1043F80001931F20334602960BF048F850200BF02B
:10440800BFFB1920394632463B460097FDF7A8FE08
:104418000EE07E4E337813F0200F05D0992001224C
:104428000B460091FDF79CFE33786FF3451333700C
:104438004FF000094FF0A70AC8464E46754B08F1E1
:104448000108F15C00294DD02368AAF14C0B43F018
:1044580080635FFA8BFB23605846FEF725FE002831
:1044680053D1162373436C4FFA5C12F0200F22D1FC
:1044780058460593FEF7F0FC059B8346D8B9FA5CCD
:10448800012142F02002FA540423009302330193DD
:104498000FFA88F30322029320200B460AF0F6FF56
:1044A80045200BF06DFB0D20594601225B46CDF8E7
:1044B80000B0FDF755FE16237343FB5C13F0200F85
:1044C80023D0564B1B7823B9554B1B7813F0010F9B
:1044D8001BD1E37803F02003DBB2B3B9514B0322BD
:1044E8001A7612E0162373434B4FFB5C13F0200F30
:1044F80005D08D2001220B460091FDF731FE1623D1
:104508007343FA5C6FF34512FA54474BF15C002988
:1045180036D02368504643F080432360FEF7C4FD3D
:10452800002842D13C4B4FF0160B0BFB063B9BF887
:10453800013013F0200F38D15046FEF78DFC0746A6
:10454800002832D19BF80130012143F020038BF879
:10455800013004230093033301930FFA88F30322F5
:1045680002934C200B460AF091FF50200BF008FBF9
:104578001920394601223B460097FDF7F1FD14E06A
:10458800254F162303FB06735B7813F0200F05D025
:10459800992001220B460091FDF7E2FD162303FB4B
:1045A80006777B786FF345137B70204B1B78002BC5
:1045B80000F091801E4B184FF35C1622002B78D028
:1045C80002FB06F3FA5C07EB0901C2F3801BBBF19F
:1045D800000F2FD142F04002FA54782204234A8077
:1045E8000093DB18012101930FFA88F30322029349
:1045F8002E200B460AF04AFF46200BF0C1FACDF8F0
:1046080000B00920414601225B4662E038240020C0
:104618002924002080240020F8230020AC12002048
:10462800EA150020DB120020762400203124002027
:104638002B240020B1F9021029BB5FEAD21B22D13A
:1046480043F6DE2005930AF0ADFE059BD8B1FA5C6F
:10465800012142F08002FA5404230093DB180193ED
:104668000FFA88F3032202932F200B460AF00EFF5D
:1046780047200BF085FA0920414601225B46CDF818
:1046880000B0FDF76DFD16237343FB5CDB0922D0F8
:10469800794B1B7823B9794B1B7813F0010F1AD18A
:1046A800E37803F02003DBB2ABB9754B03221A762B
:1046B80011E07243B95C11F0400F0CD063F386111E
:1046C80063F3C711B9544F447B8089200093414656
:1046D8000122FDF745FD01360AF1010A022E09F112
:1046E80016095FFA8AFA7FF4A9AEDFF8B4A1482761
:1046F800023E1AF8011FB0460136002937D0236858
:10470800384643F080432360FEF7CEFC002847D1AB
:104718004FF01C0909FB08F9DFF888B11BF80930CC
:1047280013F0200F3CD13846FEF796FB8046002850
:1047380036D11BF80930012143F020030BF809306A
:10474800042300930333019333B20322029313200B
:104758000B460AF09BFE50200BF012FA1920414636
:1047680001224346CDF80080FDF7FAFC18E01C232F
:1047780003FB08F3DFF82C9119F8033013F0200F2E
:1047880005D0992001220B460091FDF7E9FC1C2376
:1047980003FB08F819F808306FF3451309F80830D7
:1047A8000137042EFFB2A4D1A37803F00803DBB2CB
:1047B800002B40F0A78048F68E24A4F50A478E3FC8
:1047C8003048394618F06EFF30B92F48394618F08E
:1047D80069FF002800F090802C48394618F062FFE5
:1047E800002840F089803946284818F045FF2046BF
:1047F8000AF0D8FD264EC0B2307000287CD00138AF
:10480800C0B2307009F046FF002875D13078214ECB
:1048180000F56A506E300AF0C5FD1F4BC0B2E318B0
:1048280013F8468C307000EA08083946154818F025
:1048380039FFDFF844A0DFF8649038B112483946F0
:1048480018F030FF10B99AF800302DE00E483946BC
:1048580018F028FF38B10B48394618F023FF10B973
:104868009AF8003004E09AF8003018EA030F1BD0D9
:1048780023EA08081AE000BFAC120020EA1500205D
:10488800DB1200201C1B00201F1B0020221B002005
:1048980013130020391500202C91FF1F1415002038
:1048A800502400207825002048EA03089F48A049A2
:1048B80089F800809F4AFEF7EFFD9D489E490FF05A
:1048C80083FB68B10BF076F850B99B4808F000FC00
:1048D80030B9012398489949954A0093FEF7A6FDF7
:1048E8000023009301330193337890480293904951
:1048F800904A924B08F034FB013448F6A6239C42B8
:104908007FF45BAF8E4E73786FF3C71373702B7899
:1049180003F08002D2B2002A00F0C08089490C78E6
:10492800002C40F0BB8003F02403042B12D1FEF7C7
:10493800CFFCFF2300934020214601222346019407
:1049480002940AF0A3FD8020214601222346009408
:10495800FDF706FC2B8800246FF3C7136FF382035F
:1049680064F3451364F3410364F30003764A64F384
:10497800492364F38A2314702B80744B1A7842F00D
:10498800C0021A705A7864F3C3025A70FEF794FD95
:104998006F4818F01DFE6F4818F01AFE6E4818F0A0
:1049A80017FE19226D482146FBF7F4FC6C4B9A78E8
:1049B80002F0BF0264F345129A701A7D02F0BF023A
:1049C80064F345121A7593F8262002F0BF0264F3C7
:1049D800451283F8262093F8382002F0BF0264F3CA
:1049E800451283F838205F4B1A7802F0DF0264F32F
:1049F80086121A70DA7B02F0DF0264F38612DA7329
:104A0800594B1A7864F345121A701A7F64F34512E9
:104A18001A7793F8382064F3451283F8382093F80E
:104A2800542064F3451283F85420504B1A7802F04E
:104A3800DF0264F386121A704D4B5A7864F34512FC
:104A48005A701A7802F07F0264F345121A70DA7D00
:104A580064F34512DA759A7D02F07F0264F3451219
:104A68009A7511E04FF4A07262430A2101FB0322F8
:104A7800404901338A181179202B6FF38201117193
:104A8800F0D10134022C01D00023EBE704223A488C
:104A98000021FBF77FFC394B00221A70384F387819
:104AA80000287DD12A78374B02F00202D2B2B2B187
:104AB800264A517860F3C30151701A88CA3042F00F
:104AC80080021A8019F0D8FBC62019F0D5FB19F01E
:104AD8001FFC0BF0E1F8FEF7A1F9FEF765FE2A4A84
:104AE8002B8811786FF341036FF300016FF3000314
:104AF80011702648002118222B80FBF74BFC244814
:104B080018F066FD234818F063FD134818F060FD9F
:104B1800214818F061FD042217480021FBF73AFCF0
:104B2800164A002313701D4A1370A1E014150020C3
:104B38007A1500206E150020B1120020D91400202B
:104B4800D2120020180E0020D41300206025002067
:104B580008140020AE120020CC120020DB12002026
:104B6800AF24002055240020782500203824002078
:104B7800F82300204E270020C5120020AB12002089
:104B8800AC120020E2130020AD120020F013002028
:104B9800891D0020D0130020ED1300200B140020E5
:104BA8002C7804F00203DBB293B914F001040FD19E
:104BB800774818F00DFD3B78E0B2234113F0010F60
:104BC80003D0FEF7A1FA0AF0EBFE0134042CF2D16F
:104BD8002B78704C13F0010F22D0FEF791FD23883B
:104BE80043F002032380FEF731FB6B4B1F78A7B914
:104BF800CA2019F041FBCD2019F03EFB23886748F5
:104C080067F300032380664B1A7842F001021A709A
:104C180018F0DEFCFEF702F902E00120FEF788FC3E
:104C28002B7803F00202D2B212B35E4A12782AB18C
:104C380013F0010F02D10220FEF77AFCFEF74AFFBB
:104C480059495A4818F0E2FC5849594818F0C8FC24
:104C5800FEF74CFC5549574818F0C2FC56495548D0
:104C680018F0C9FCFEF7D0FB5448504918F0E4FC92
:104C780053484D4918F0B4FC524A13780BB9FEF763
:104C880049FB737803F08003DBB2DBB92B7803F0C0
:104C98002403042B06D143F6EC200AF083FB08B169
:104CA80006200DE0FEF76EFD08B1052008E00BF0C8
:104CB800C7F808B1032003E001F044F810B104205C
:104CC800FEF736FC404B1B781BB173786FF3C713A4
:104CD80073703E490B7813B13D4B1B780BB32B789F
:104CE8002C4E03F04403402B1BD100242146012203
:104CF800234620460094FDF733FAFF2300933F2014
:104D0800214602222346019402940AF0BFFB33880D
:104D180043F6CE2043F0040333800AF043FB2D4BC7
:104D280018702A4A2C4E13789BB1294B197881B9EF
:104D38002A78184B02F04002D2B252B11A8861F3B5
:104D480082021A80337823B943F6CE200AF02AFB70
:104D580030702A780F4902F00400C0B21F4B0028B7
:104D680000F09F8002F02000C0B21A4C002837D013
:104D78001A7842F0C0021A702378002B40F0958010
:104D88000A8863F3820263F345120A808DE000BF4C
:104D9800891D0020E2130020AB120020141300200C
:104DA800AD1200200B140020D5120020D0130020D3
:104DB800CC120020E7130020F5120020ED1300208C
:104DC800C9120020180E0020662C0020D8130020DD
:104DD8000C140020D4130020DA12002060250020D3
:104DE800D20052B219789211D2B241F0C00112F039
:104DF800010F197003D0C9B260F3C711197012F00E
:104E0800020F03D01A786FF386121A701B78814A42
:104E180003F04003DBB21BB9537843F00803537027
:104E280043F6CD200AF0BEFAC0B20128307002D194
:104E3800794B02221A702478002C36D1FEF748FAF2
:104E480021460122234680200094FDF789F9FF239B
:104E580001220093402021462346019402940AF03F
:104E680015FB2B8843F6CD2043F020032B800AF056
:104E780099FA6A4B18706A4B1C706A4B1A780AB117
:104E8800013A1A70197881B9674A13786BB1FF2310
:104E98000093412002220B46019102910AF0F6FA92
:104EA80003E01A7842F0C0021A700AF079FF5F48EE
:104EB80018F0C7FB5E4B18B91A7860F3820202E05B
:104EC8001A7842F004021A706A785A4812F00101FE
:104ED8001A780CBF61F3410242F002021A70564977
:104EE80018F0AAFB5549534818F085FB5148544916
:104EF80018F081FB3378012B40F089802B8800243F
:104F08006FF349236FF38A232B80434B19221C70BC
:104F180021464C48FBF73EFA4B4818F059FBFEF780
:104F2800CBFA464818F054FB454818F051FB474B5C
:104F38009A7802F0BF0264F345129A701A7D02F063
:104F4800BF0264F345121A7593F8262002F0BF02D7
:104F580064F3451283F8262093F8382002F0BF0244
:104F680064F3451283F83820394B1A7802F0DF02CF
:104F780064F386121A70DA7B02F0DF0264F3861299
:104F8800DA73344B1A7864F345121A701A7F64F393
:104F980045121A7793F8382064F3451283F83820BD
:104FA80093F8542064F3451283F854202A4B1A7856
:104FB80002F0DF0264F386121A70284B5A7864F301
:104FC80045125A701A7802F07F0264F345121A707B
:104FD800DA7D64F34512DA759A7D02F07F0264F394
:104FE80045129A7511E04FF4A07262430A2101FB41
:104FF80003221B4901338A181179202B6FF3820190
:105008001171F0D10134022C01D00023EBE709B073
:10501800BDE8F08F60250020DA120020D4130020AC
:10502800180E00200C140020D8130020F8120020BD
:10503800AD120020E2200020E7130020AE1200206D
:1050480008140020DB120020CC120020AF2400201E
:10505800552400207825002038240020F82300203B
:105068004E2700202DE9FF4104460D460AF0C2FEF6
:105078009C4B1A1992F830709B4A98461278AA2AC3
:105088000AD1A7F14F03DAB20B2A00F2AC81974A92
:105098005BB29A4040F1A781954B0C2202FB043386
:1050A8005A7A0833AA42C0F09E81FF2A00F09B81F9
:1050B800FF229A7008EBD40393F8935004F0070387
:1050C8001D41502F05F0010500F0268114D8462F08
:1050D80000F0F08009D8412F00F08F80452F00F0B4
:1050E8001B812D2F40F07D8130E0482F00F0BD80DE
:1050F8004F2F40F076810DE0542F5BD005D8522F0A
:105108007BD0532F40F06D8118E0A7F15903012B94
:1051180000F267817748214618F0C4FA064600284D
:1051280040F061815A2F01D1734808E1592F03D00B
:105138007148214618F0A0FA704800E170482146ED
:1051480018F0B0FA0646002800F054816D48214650
:1051580018F0A8FA002840F046812146694818F05E
:105168008BFA6948214618F092FA012602224DB1BD
:10517800A4191420314600230092019602940AF0E3
:1051880085F937E101340A20294633460092019611
:1051980002940AF07BF9214632462B4613200095EB
:1051A800FCF7DEFF122029462A4633460095FCF715
:1051B800D7FF1FE15348214618F074FA0546002826
:1051C80040F0118101260222A7193E2031463346BC
:1051D8000092019602970AF059F9394632462B4651
:1051E80014200095FCF7BCFF2146464818F044FA05
:1051F8002146454818F04BFAFCE04148214618F092
:1052080051FA0646002800F0F5804048214618F07B
:1052180049FA002840F0E7803A48214618F042FA57
:10522800064628B92046FDF717FE002840F0E28020
:10523800002D40F09D802046FEF786FA002840F0B9
:10524800D4802046FEF736FC314BDB7803F0200390
:10525800DBB20BB92F4B1855412F00F09780522F16
:1052680040F0BF802046012192E02848214618F0EE
:1052780019FA002840F0B7802248214618F012FA9F
:1052880028B92046FDF7E8FD002840F0AC80002D45
:105298006ED12046FEF758FA002840F0A6801C4B35
:1052A800DB7803F02003DBB2002B6FD1194B03220C
:1052B8001A766BE01548214618F0F4F9002840F0FA
:1052C80092801048214618F0EDF9064628B9204684
:1052D800FDF7C2FD002840F08D80002D48D1204602
:1052E800032155E02C1B0020D31300200000308040
:1052F800F81B0020221B00201C1B00201F1B002065
:10530800D0130020E7130020EA130020D512002054
:10531800EC230020DB1200203848214618F0C2F99F
:105328000646002866D03648214618F0BBF90646DE
:10533800002858D12046FDF741FF20B131482146C9
:1053480018F09AF956E0502F28D12F4B1B782BBB19
:105358002046FDF71FFF08BB2C48214618F0A2F98C
:10536800064620B92046FDF777FD002842D115B141
:10537800204602210CE02046FEF79CFB244BDB78FC
:1053880003F02003DBB20BB9224B1855204600214D
:10539800FEF7C2FA061E18BF01262BE02046FDF7CD
:1053A800F9FE0546F8B91C48214618F07BF906466F
:1053B800D8B92046FDF750FD0746D8B9164821460A
:1053C80018F05AF9154A135D8BB911494E7806F051
:1053D8002006F6B26EB908EB040393F86030135553
:1053E80008E0012606E0002604E02E4602E03E46DC
:1053F80000E01E46304604B0BDE8F081D01300201E
:10540800D5120020141300200B140020E7130020ED
:10541800EC230020DB120020CC120020F013002027
:10542800032210B505490648FBF78AFA05480649DC
:105438000222BDE81040FBF783BA00BF3E190020E6
:1054480002020020070200203C19002070B5804CA1
:10545800237813F0010F0AD00AF0B4FA38B100200B
:105468007C4902F02BFD7C4B7C48197849E07C4D47
:105478002B78002B4AD00AF0ABFA002846D0794B9B
:105488001B7873B9784B5B7813F0010F09D00AF0D9
:1054980091FA30B9237803F02403042B01D10330A7
:1054A800B6E0724C207870B10020714902F006FD18
:1054B800217801226F4802F027FD00201021621C8C
:1054C80007F0D0F902E06C4902F0F8FC6B4C644834
:1054D80007F018FA2378002B00F00A810AF072FA14
:1054E800002800F00581664966481022FBF728FA73
:1054F80064485B21FAF7CCFF002800F0F980217896
:1055080001308322BDE8704002F0FEBC5E4C237877
:1055180003F00503012B5DD100205C4902F0CEFCAD
:10552800202110225A48FAF735FF601D59490322F5
:10553800FBF7B0F940BBE01C57490222FBF7AAF978
:1055480030B95648FBF776F95449024650480BE003
:10555800E01C53490222FBF79DF940B95148FBF77B
:1055680069F9504902464A48FBF7EAF90EE0E01C9F
:105578004D490222FBF78EF930B94C48FBF75AF92E
:105588004A4902464248EFE7FFF74AFF6278303A55
:10559800D3B2092B00F2AC803B4B9B78303BDBB29B
:1055A800092B00F2A5800A2101FB0231C9B20029AA
:1055B80000F09E80334BFF220C291A7740F2988026
:1055C80010295A7740F2948013299A7740F29080F4
:1055D800DA7770BD234E3378F3B9234B5B7813F039
:1055E800010F19D00AF0E6F9B0B9314818F029F8D6
:1055F80068B1304C304B226802EA03033BB914F01F
:1056080037F920B9E37803F04003DBB223B1002077
:10561800BDE8704008F038BC337863B90AF0CAF9BD
:1056280048B1264B1B7803F00603042B03D02B78D4
:105638000BB90120ECE7FEF7A5F810B100202049CE
:1056480052E0204B1C78002C40D01F494CE000BF92
:10565800E2130020ED670208AB120020FE010020D3
:10566800AC12002037150020EA150020F91400209C
:10567800C445020803020020824502080B140020DA
:10568800A3450208F201002039190020CB4A02087C
:105698000202002030B2020834B202082E4B02087F
:1056A80037B202080D4B02083AB20208EC4A020867
:1056B800F8120020EC2300203000000FAD1200206B
:1056C800F15702081D0E0020E545020802F09AFB7A
:1056D80002F08CFB17F0B6FA064BDB7803F02003D8
:1056E800DBB22BB104492046BDE8704002F0E6BBAE
:1056F80070BD00BFEC230020DD440208054B1B7879
:10570800D8019B015BB2DB1140B243EAE070C0B242
:10571800704700BFE213002070B50E4686B0410006
:105728000122054601F5E97105A809F04CFE0021A2
:10573800012E8DF815104FF0FF0205F1010305D178
:105748000092019102930920FB3A04E00092019132
:1057580002931E2004220B4609F098FE05A83F4933
:10576800FAF71CFF50B105A83D49FAF717FF28B111
:1057780005A83C49FAF712FF00286BD105A839495A
:10578800FAF70CFF384B0446C0B95A78214642F064
:1057980010025A70FF23022200930190FE3B0290F0
:1057A8003D2009F073FE4D200AF0EAF91220691C29
:1057B800012223460094FCF7D3FC03E05A786FF3E8
:1057C80004125A700024294BE35C552B07D1284654
:1057D800214611F0AEFF10B1204611F099FF0134B7
:1057E800082CF0D1002E32D121482249224AFDF757
:1057F80053FE204821490EF0E7FBC0B10AF0DAF861
:10580800A8B91E4807F064FC88B905A81349FAF737
:10581800C5FE012320B9009318481949154A04E028
:1058280016481749134A00933346FDF7FFFD154BF9
:1058380010491D700023009305330193124B0E4A43
:105848001B780B4802930E4B07F08AFB02E00F4BC4
:1058580000221A7005A806B070BD00BF6BB202081E
:105868003DB2020828B4020860250020FD2400206B
:10587800141500207A1500206E150020B1120020A2
:10588800D9140020E825002039150020C412002072
:1058980007B54100012201A801F5E97109F093FD5E
:1058A800002301A804498DF80530FAF777FED0F1F6
:1058B800010038BF00200EBD6BB2020807B54100D9
:1058C800012201A801F5E97109F07DFD002301A875
:1058D80004498DF80530FAF761FED0F1010038BFB0
:1058E80000200EBDFAB3020870B5134B04461B180E
:1058F80093F8305089B11148214617F0BDFEA5F143
:105908005903DBB2012B0CD94F2D0AD0542D08D0E6
:1059180021460B4817F0B0FE07E00848214617F06B
:10592800B6FE0748214617F0B2FE04480549BDE80F
:10593800704017F055BE00BF2C1B0020F812002045
:10594800CF120020ED130020024B1878C0F380001E
:10595800704700BFAD120020024B1A8860F308227E
:105968001A807047E2130020034B5878C00140B2F8
:10597800C011C0B2704700BFE2130020014B187875
:10598800704700BFAC12002030B5457800230021D5
:10599800C218917055FA03F111F0010F08D00649A9
:1059A80059188C7C017804EA0101A14208BF917062
:1059B8000133042BEBD130BDF914002046F65221F7
:1059C800042209F000BD000070B5104C05461022F5
:1059D80020460021FAF7DEFC002004F8010C2A78A2
:1059E800103414F8011FC3B291420BD152B10849C7
:1059F800013301F8013B112246F6A243BDE870408D
:105A080002F09AB901300428EBD170BDFA140020D5
:105A1800F91400202DE9F3412D4C0722E37848F6CC
:105A2800242702FB0030C0B200F50A40453009F0D7
:105A3800B9FC257964795FFA80F8002648FA06F3FC
:105A480013F0010F3AD03946042201A809F0BBFC33
:105A58009DF804009DF805309DF806109DF8072074
:105A680000282BD0002929D0002B27D0002A25D0A8
:105A7800934204D19C4221D185421FD30FE09A4220
:105A880010D99C421AD3944218D89C4201D9944206
:105A98001AD39C4201D1854216D294420ED18D422E
:105AA8000CD811E09C4201D185420DD2944201D11B
:105AB8008D4209D99C4207D8944205D30136043750
:105AC800082EBBD1002000E00120BDE8FC8100BF0A
:105AD800D429002010B50446C00800F50A407D30DE
:105AE80009F060FC04F00704C0B2204100F0010096
:105AF80010BD70B5C50805F50A457D35044628462C
:105B08000E4609F04FFC04F00704C0B2012126B983
:105B1800A14040EA0101C9B202E0A14020EA010126
:105B28002846BDE8704009F033BC0000F0B57C4B56
:105B38008DB0DE78042200EBC606F6B2F10001F55E
:105B4800EC4104A8AC3109F03EFC764B764C1A784F
:105B5800002304A9C95C312905D13039994041EAAB
:105B68000202D2B205E0302903D12F39994022EA46
:105B780001020133042BECD122706B486B496C4A4B
:105B8800FDF78AFC694B1B7813B9694B1B78F3B195
:105B9800664868490EF018FA68B109F00BFF50B969
:105BA800644807F095FA30B90123624862495F4AB0
:105BB8000093FDF73BFC0023009302330193FD3370
:105BC8000293594859495A4A5B4B07F0C9F906EB01
:105BD8000611002501F5F041257004A86C31082252
:105BE80009F0F1FB2C462F46544B0135E35C542B4E
:105BF80036D104AB1B5D312B03D1204611F090FC4C
:105C080038B104AB1B5D302B2AD1204611F088FC3B
:105C180030B34FB9FF2300933420394604223B4662
:105C28000197029709F032FC04AF385D21463038FD
:105C380011F084FC3B5D0127312B4FF0030305D1A4
:105C480000932BB201970293352004E000932BB206
:105C5800019702933620002104220B4609F016FC16
:105C68000134082CC0D1B10101F5F84104A8243150
:105C7800202209F0A8FB083C04AD274615F8013B93
:105C8800E6B20134302B03D13046FFF723FF38B199
:105C980015F8013C312B2CD13046FFF71BFF40B3E0
:105CA8004FB9FF2300933420394604223B4601971D
:105CB800029709F0EBFB15F8011C30463039C9B2E0
:105CC800FFF717FF15F8013C0021302B4FF0FF03B9
:105CD80005D1009323B201910293372004E0009389
:105CE80023B201910293382004220B4609F0CEFB1F
:105CF8000127202CC2D1124D6B7803F00403DBB2CC
:105D080063B1203C2046FFF7E5FE38B90134E4B220
:105D1800202CF7D16B7860F382036B700DB0F0BD67
:105D2800D4290020AC120020141500207A15002078
:105D38006E150020B1120020D9140020FD24002087
:105D480060250020014B1878704700BF1D0E002009
:105D58002DE9F04F4A4B00221A704A4A85B016784E
:105D6800002E40F08A80484B4FF4B468DA7899786E
:105D780008FB02F24FF03C0808FB01285A78434F11
:105D880090441FFA88F8BA4665E03AF815303C2482
:105D9800DAB2544304EB13244C44A4B2042CEEB2FC
:105DA80007D842F25A73984503D904F51C54603455
:105DB800A4B2444511D948F6442009F0F3FAC8EBD7
:105DC8000403834209DC324B1A787B1993F8383084
:105DD800934302D02A4901230B702B4AD378B3424C
:105DE8002BD142F26073B4FBF3F203FB12439BB274
:105DF80043451CD1274B9B7813F0090F3DD1264B07
:105E08005B7803F02003DBB2002B36D1234B1A78E2
:105E18001BEA020F11D10199009841EA02021A7097
:105E2800FFF7F8FD48B90098FFF780FE05E01B4B27
:105E380002991A7801EA02021A70013509F5B46963
:105E4800072D1FFA89F9A0D1039E07370136042EC2
:105E58000AF10E0A11D04FF0010B0BFA06FB5FFA9C
:105E68008BF301936FEA0B03F2B2DBB24FF0000938
:105E7800009202934D46039687E705B0BDE8F08F80
:105E88001D0E00200F140020D4290020101400201B
:105E9800AC120020EC2300206E2500200E140020F8
:105EA80073B50C4601EBC001C9B2C90001F5EC415C
:105EB8000546042201A8AC3109F085FA104B0020F0
:105EC80003EBC402121B521982F8380001AA125CB3
:105ED800312A0AD10121814003EBC402121B521955
:105EE80092F83860314382F8381001300428EDD137
:105EF80001A93122302317F0DDFBC0B27CBD00BF01
:105F08001014002000B501EBC001C9B2890189B0A5
:105F180001F5F84124312022684609F054FA20207E
:105F280069463122302317F0C5FBC0B209B000BD65
:105F380007B501EBC001C9B201EB011101F5F04150
:105F48006C310822684609F03EFA08206946312279
:105F5800302317F0AFFBC0B20EBD00002DE9F843A7
:105F6800002634462BE021462846FFF799FF2146B4
:105F780081462846FFF7C6FF214640EA0909284618
:105F8800FFF7D6FF5FFA89F949EA000010F0FF0F22
:105F980005D040463946022209F015FA03E04FF0D1
:105FA800FF33A8F800300135EDB20237072D08F1AC
:105FB8000208D8D10134E4B20E3E042C07D0054BB8
:105FC800C6F5EC47C6EB03083C370025CBE7BDE830
:105FD800F88300BF1014002010B518F0CDFB4FF463
:105FE800803018F0E9FB18F001FD0128044628D19B
:105FF800102018F0E3FA022018F0D4FA002018F064
:106008001BFC002018F02CFC4FF4806018F01EFCDC
:106018004FF4404018F02EFC4FF480304FF4E0115C
:1060280018F0E6FB204618F0EFFB392018F0CAFC00
:106038000028FAD0022018F0EDFB18F0F5FB08282C
:10604800FBD17C20012118F087FC46F601200121B4
:1060580018F082FC0C48012118F08AFC0B48012139
:1060680018F086FC0420012118F082FC7E2018F02C
:10607800A9FC38B118F0D0FC054B04211A7861F35B
:1060880044021A7010BD00BF03400600000808183B
:10609800492C002010B50C46014620B110220C48AE
:1060A800FAF74EFC04E00A4820211022FAF772F9A8
:1060B80034B1084821461022BDE81040FAF740BC28
:1060C800044820211022BDE81040FAF763B900BF48
:1060D800F20100200202002010B5FF2B1446029A9C
:1060E80003D0421802F8013C08E06FF07F439A425F
:1060F80004D01314437013128370C27015F082FD1C
:1061080002E07F2018F0A4FF15F068FD0028F8D100
:10611800ACB10B4890F82010163001F00F0115F0C3
:1061280071FD02E07F2018F093FF15F057FD00285D
:10613800F8D1044B93F8693013F0010FE9D110BD81
:106148004C0C0020642B002010B50A4B002203EBF6
:10615800C003013B1046084951184C7813F8011F39
:106168008C4205D10130C0B20C320828F3D1F73087
:1061780010BD00BF22F10108F81B002070B50D4CBE
:1061880005460E464FF4807200212046FAF702F9C0
:106198002A46314604F58070FAF754F8642004F86A
:1061A800025C16F0ADFF002384F8F131024B642243
:1061B8001A6070BDCC2C00204419002010B5054C85
:1061C800002120464FF48072FAF7E4F8002384F89F
:1061D800F13110BDCC2C0020164B2DE9F0415D8A21
:1061E80007462846FBF79CFC1349FBF7A5FD134B14
:1061F800134E1860D723B5FBF3F5EDB2822229467A
:106208000446F01901F080FE2846FBF78DFC014694
:106218002046FBF7D3FB0B49FBF7DAFCFBF79EFEA6
:106228000337BE19C1B281223046BDE8F04101F002
:106238006BBE00BF541D00200000574364140020AB
:10624800F20100200000204170B54B4D2868FBF793
:1062580073F845A3D3E90023FAF70EFFFBF75AFBBF
:10626800FBF76AF842A3D3E90023FBF7B9F83EA38A
:10627800D3E90023FBF7DEF9FBF74CFBFBF75CF8EF
:10628800FAF766FEFBF746FB3C4906462860FBF733
:1062980047FE20B13046FBF761FEC4B25EE03046EF
:1062A8003649FBF751FE50B130463549FBF738FE09
:1062B80028B13046FBF752FEC0B2441C4EE03046CF
:1062C8002F49FBF741FE50B130462E49FBF728FE17
:1062D80028B13046FBF742FEC0B2841C3EE030468F
:1062E8002849FBF731FE50B130462749FBF718FE25
:1062F80028B13046FBF732FEC0B2C41C2EE030464F
:106308002149FBF721FE50B130462049FBF708FE32
:1063180028B13046FBF722FEC0B2041D1EE030460D
:106328001A49FBF711FE50B130461949FBF7F8FD41
:1063380028B13046FBF712FEC0B2441D0EE03046CD
:106348001349FBF701FE48B130461249FBF7E8FD57
:1063580020B13046FBF702FEC0B2841D0A20214658
:10636800BDE8704009F014B8736891ED7CFF7F4078
:106378000000000080842E416814002000001041B5
:106388000000F0410000484200008E420000B84280
:106398000000E0420000F2422DE9F04F9DB015F0F8
:1063A800C7FB092016F0D8FF16F02EFE4FF4614007
:1063B80017F00EF8092017F08BF80022A3484FF4C5
:1063C800804118F060F9A248002118F029FDA14980
:1063D80004224B78DFF8A0E26FF300034B709E4B6A
:1063E8009E4C1A705A709A70DA701A715A719A71B2
:1063F800DA719B4B033A1A709A4B00201F328EF8C1
:10640800000020705A7005900546069006467F20C9
:1064180018F01EFE23780E2B01F2B281DFE813F08C
:106428000F004F009500E0007902DE033004850478
:10643800E806DA07ED075608AF08CE087E098A4E47
:106448008A48317801F00F01013149014118FFF7FD
:1064580021FE337813F00F0308D1854A92F82121E1
:10646800012A41F08D81834A138024E0012B03D156
:106478007F4B93F839310BE0022B04D17C4B93F816
:106488002D31032B05E0032B06D1794B93F82D31E1
:10649800012B41F075810EE0774901220A70774897
:1064A8004FF4007118F0EFF8754BC8221A60337872
:1064B8006FF30303BFE333785A1C01F05DB8704BE8
:1064C8001A6822B96D484FF4007118F0DCF8DFF84B
:1064D80098816C4898F8001001F00F0101314901CA
:1064E8004118FFF7D7FD36B198F800305A1C62F30F
:1064F800030388F800305F4B00221A8098F80010D8
:1065080001F00F02022A03D11A7842F010020AE0C1
:10651800042A03D11A7842F0040204E0052A05D1BE
:106528001A7842F040021A7001F02AB9062A04D1FA
:106538004D4B6FF3030119707EE301F00F01012247
:1065480012FA01F1198001F01BB9474E4E48317813
:1065580001F00F01013149014118FFF79BFD96F841
:10656800008008F00F08B8F1070F27DC18F0010FBA
:10657800464B02D00020588002E04FF0FF3159808E
:106588004FEA6809062209F1010902FB09394FF0AF
:10659800FF32A9F802204046FFF7D6FDFF2806D0B3
:1065A8003B4B03EB40005823437401F0E9B8002348
:1065B800A9F8023008F1010801F088B8002110227A
:1065C80013A8F9F7E7FE0FA800211022F9F7E2FE59
:1065D80023780133237033786FF3030301F079B81C
:1065E800DFF884A09AF8008018F00F0840F03F8187
:1065F800284E337803F04003DBB2F3B926486FF036
:106608007F43817A0122009301F00F01FF23FFF7F6
:1066180063FD224B93F8692012F0400F08D093F8DD
:106628006C3013F0040F03D0337843F04003337019
:106638007378142262F3C7037370737813F0F80F3A
:1066480030D0174800F12001A5E300BF0018014031
:10665800002C0140761D00202C1B00206E14002009
:106668001B0E0020AF2400206D14002062F10108E9
:10667800F81B00206025002074190020000C014040
:106688004419002002F20108E2F201081A2500204C
:10669800F2010020D72300204C0C0020642B00209E
:1066A80002F40108BC4B1B7803F04003DBB2002B5B
:1066B80000F0D980DFF80483DFF8049398F80030FD
:1066C80013F00C0B30D1B54E6FF07F4396F82B10BA
:1066D80006F12100009301F00F0101220523FFF7C5
:1066E800FBFC96F84C104FF4860A06F1420001F0C4
:1066F8000F010122FF23CDF800A0FFF7EDFC96F86B
:106708004110FF2306F1370001F00F015A46CDF87A
:1067180000A0FFF7E1FC042389F8003098F8003066
:1067280043F0080301F02AB803F00803DBB2002B9A
:1067380039D099F800A0BAF1000F03D0984800F1B9
:10674800400138E0954E6FF07F4B717D06F10B00EC
:1067580001F00F010122FF23CDF800B0FFF7BCFCC8
:1067680096F82B1006F1210001F00F0101220723F2
:10677800CDF800B0FFF7B0FC96F836104FF486035A
:10678800009306F12C00FF2301F00F015246FFF79A
:10679800A3FC98F800306AF3C303DBB243F00403A8
:1067A80088F800305AE099F800C0BCF1000F08D012
:1067B8007B4800F16001FFF76DFC99F8002030324A
:1067C80008E2764E6FF07F40717DFF23009001F064
:1067D8000F0106F10B000122CDF80CC0FFF77CFC7D
:1067E8009AF80030DFF8C4B103F0100A5FFA8AFAA9
:1067F800DDF80CC0BAF1000F0CD098F800206CF34B
:10680800820288F800205A1C62F303038BF80030D8
:1068180000F0B6BF96F82B106FF07F42009206F199
:10682800210001F00F0101220C23FFF755FC96F817
:1068380036104FF4860300935246FF2306F12C00CE
:1068480001F00F01FFF748FC9BF8003083F01002BD
:10685800C2F3001262F304138BF80030042389F8A2
:10686800003000F08DBF4E4800F1800193E2B8F18E
:10687800010F3CD14A4800F1A001FFF70BFC002EA4
:1068880000F07E879AF80030444E5A1C62F30303E6
:106898008AF8003096F82B106FF07F4906F1210036
:1068A80042460F2301F00F01CDF80090FFF714FCCA
:1068B80096F82B1006F1210042460E2301F00F0135
:1068C800CDF80090FFF708FC96F82B1006F1210090
:1068D800424601F00F010F23CDF80090FFF7FCFBB3
:1068E80030488021424617F0CEFE00F049BF2C48C0
:1068F80000F1C001FFF7CEFB002E00F041872A4BC4
:1069080096221A609AF800306FF303038AF8003071
:1069180092E1264E317811F00F0A16D1244800F181
:106928002001FFF7B7FB204B1B68002B40F028879E
:1069380013A8F9F77FFF40221346014613A801F078
:1069480007F93378012200F017BEBAF1010F39D1E7
:1069580012486FF07F4390F8201000220093163001
:1069680001F00F01FF23FFF7B7FB01F05BF90028E7
:1069780000F006873378022262F3030333700D4B6D
:106988001A7842F080021A700B4B5A7842F00202D1
:106998005A7000F0F5BE00BFD72300204C0C002031
:1069A80002F4010800100140441900206D14002071
:1069B800E2F40108DC230020742600206031002066
:1069C800F731002001F00F0101F10E0303F00F036E
:1069D800012B44D89B4849014118FFF75BFB9A48B3
:1069E8006FF07F4390F8201000221630009301F0DA
:1069F8000F01FF23FFF770FB16F0BEF9337803F0A1
:106A08000F03022B13D112F007FF002800F0B886FD
:106A18008E4B1A7842F040026FF304121A705A78BB
:106A28006FF345125A703378032200F0A5BD12F0B7
:106A3800DDFE78B112F088FF12F054FE844B00207E
:106A48001A7858816FF3C7121A703378042262F3E8
:106A5800030333707F4B1A786FF3000263E5BAF1D2
:106A6800040F4DD1DFF8DC914901DFF81082494469
:106A78004846FFF70FFB98F80010774B01F0040227
:106A8800D2B27AB941F004016F4883F800A088F8BF
:106A9800001090F836104FF4860300932C3001F064
:106AA8000F01ECE293F800A0BAF1000F40F06886FD
:106AB80065486FF07F45417D01220B3001F00F01E1
:106AC800FF230095FFF708FB64480122817AFF2322
:106AD80001F00F010095FFF7FFFA98F80030052242
:106AE8006AF3820388F800303378484662F3030378
:106AF800337009F1A001FFF7CDFA554600F040BE0A
:106B0800DFF84481FF2398F8201000226FF07F49B6
:106B180008F1160001F00F01CDF80090FFF7DCFA3C
:106B28002BB2072B18D1337808F121006FF3030338
:106B38003370237801220133237098F82B100E2329
:106B480001F00F01CDF80090FFF7C6FA4448802104
:106B5800002217F098FD0025424E96F86B3013F08E
:106B6800040F00F00D8698F857106FF07F4300224D
:106B780000933D48FF2301F00F01FFF7ADFA96F8A7
:106B88006B303A4A03F00F03012B137003D1002D29
:106B980008BF01250CE0022B04D12BB2012B08BF42
:106BA800032505E0032B03D12BB2032B08BF0725D0
:106BB800ABB213F0010F02D02D4A3121517713F0F7
:106BC800020F02D02A4A3221917713F0040F00F005
:106BD800D7853322264BDA7700F0D2BD1948254EE7
:106BE80000F1C001FFF756FA96F80090DFF85C80D4
:106BF80019F00F090CD112F08FFC98F8003069F3E6
:106C0800000388F8003033785A1C62F303033370AA
:106C180012F014FD98F8003013F0010F00F0B08561
:106C280000221548802117F02EFD0A4B00225A70C9
:106C3800337862F30303337023780133237000F051
:106C48009FBD00BFE2F401084C0C00207426002010
:106C5800DC230020F0250020F7310020010000206F
:106C680000100140642B0020990C0020D62300203E
:106C7800F20100206D14002000180140603100204E
:106C88008548864E00F1E001FFF704FA0FA8F9F7EE
:106C9800D1FD0FA902468248F9F752FE002181482A
:106CA800B18090F8C5106FF07F4300220093BB308D
:106CB800FF2301F00F01FFF70FFA7B4A92F86B10E0
:106CC80092F86C30327843EA012312F0010FB38056
:106CD80010D0A3F1EB0292B20A2A04D9A3F5E67305
:106CE8009BB2282B02D8F3880133F38033786FF3F3
:106CF800000333707378002B40F04285674AD288CE
:106D08007AB16A4A1BA8117863F3030111702278DB
:106D18008DF86F300132227028228DF86C2017F020
:106D2800D1FC0022F28000F02BBD614EDFF8A8A153
:106D3800337803F00408B8F1000F15D109A84146CB
:106D48001522F9F727FB5B4BCAF800801B684546FC
:106D5800CDF827303368474643F004033360564B79
:106D680083F8F98100F00CBD03F08003DBB2002B3F
:106D780067D1DAF80010002940F002854F48FFF784
:106D880089F94F484FF4805117F073FC012806D059
:106D98004A4800F1A001FFF77DF900F0F1BC46492F
:106DA80091F8F921002A43D008314648013AF9F709
:106DB800C7FD444B03F1100113F8012B0D2A01D034
:106DC8000A2A02D1202203F8012C8B42F4D13E4B2F
:106DD8004FF03C0808FB073808F11E084046F9F751
:106DE80029FD414602463948F9F754FDD8B9022F22
:106DF80003D1336843F0100304E0032F03D1336851
:106E080043F040033360327853005BB203EAC26355
:106E1800DB173268DBB263F3C71232601BB1FFF7CE
:106E2800CDF900F0ADBC0137FFB2042F08BF02272F
:106E3800254B3C2606FB07363046F9F7FBFC314666
:106E480026E0DAF80080B8F1000F40F099847378F2
:106E580003F02002D2B2002A40D11D4B09A81A889B
:106E68009B781C498DF82630ADF82420F9F7ECFA08
:106E7800114B1B7A302B07D1FFF7A0F9336843F485
:106E88000053336000F07CBC09A8F9F7D3FC09A9CA
:106E9800FFF774F900F074BCE2F40108F025002053
:106EA800060200204C0C0020642B00206D140020EA
:106EB800481900203FB20208C42C0020E2F501085E
:106EC80000080140020200200C000020CC2C002009
:106ED80044B2020848B202084419002003F04003F3
:106EE800DBB2002B40F08980B14800F16001FFF768
:106EF800D1F8B048F9F79EFC8046AE49AE48424604
:106F0800F9F7C8FC002873D1AC4B43441B7A302BEB
:106F18006ED1FFF753F93368DFF8D09243F480431A
:106F2800336099F82B106FF07F43009309F121002B
:106F3800082301F00F010122FFF7CEF86423CAF8F5
:106F480000307F2018F084F8DAF80030002BF8D1F0
:106F5800984699F88E10D633994E89F886304B3B6F
:106F68006FF07F4A89F88730964801F00F01424652
:106F78007433CDF800A0FFF7AFF896F8B91106F50D
:106F8800D670033001F00F014246FF23CDF800A070
:106F9800FFF7A2F896F8C41106F5DD7001F00F01AD
:106FA8004246FF23CDF800A0FFF796F896F8CF11D8
:106FB80006F5E270013001F00F014246FF23CDF8DB
:106FC80000A0FFF789F896F8DA1106F5E87001F0E5
:106FD8000F014246FF23CDF800A0FFF77DF899F88E
:106FE80099107948CDF800A001F00F01424646E01B
:106FF8007648F9F71FFC75494AE796F802B0DFF8BA
:10700800EC910BF0020B5FFA8BFBBBF1000F3AD14E
:1070180099F82010FF236FF07F4809F1160001F05E
:107028000F015A46CDF80080FFF756F8684B93F8E1
:107038006B3003F00803DBB2002B00F0A18399F852
:107048002B10012209F1210001F00F010323CDF8D3
:107058000080FFF741F83368554843F4003300F1E6
:1070680080013360FFF716F855485A4690F8E51145
:1070780000F5EC70CDF80080033001F00F01FF231C
:10708800FFF72AF87CE3CAF8008099F820106FF01F
:107098007F4300934246FF2309F1160001F00F01D8
:1070A800FFF71AF82AB241F211139A421DD1434B45
:1070B8001B7A302B13D1FFF781F83368454668F304
:1070C800514368F38E3368F34D333360414B1A787C
:1070D80068F303021A7023780133237050E33E48A3
:1070E800F9F7A8FB3C49FFF749F8394E96F86B3099
:1070F80013F0040F00F0448325B9384820211022EA
:10710800F9F748F97F2017F0A3FF99F857106FF0A7
:107118007F43002200933248FF2301F00F01FEF75E
:10712800DBFF96F86B202F4B02F00F020D2A1A7026
:1071380005D125B92C4A412191754FF480551A780B
:10714800062A08D12AB2B2F5805F04D1264A362130
:10715800D1754FF488551A78082A08D12AB2B2F5A1
:10716800885F04D1204A3821117641F210151B7826
:107178000B2B09D12AB241F210139A4204D11A4BAF
:107188002A225A7641F211150D486FF07F4390F884
:10719800F0110022009300F5F370FF2301F00F01B6
:1071A800FEF79AFF96F86B3013F0010FAAD0E7E2CA
:1071B800E2F501081A010020CC2C0020C42C002084
:1071C80001000020D00C0020DB0C0020FC00002077
:1071D800642B00206D1400203801002002020020DA
:1071E800990C0020D6230020F20100204C0C00202E
:1071F800A34B1A7842B300221A700F20FAF724FF23
:1072080006460A20FAF720FF9E4B9F4958824A7883
:1072180012F0010F18D06436301A58839B4B1A7835
:10722800642A01D19B321A701B78984EFF2B0BD021
:107238000A21B3FBF1F1964B23311980954817F0D9
:10724800EFFD337801333370DFF8648298F800304B
:1072580013F00F0612D18E4B23228B481A804378E5
:10726800232143F0010343708A4817F0D9FD8A4867
:1072780000F12001FEF70EFF04967AE2012E68D194
:10728800804B5A8BA2F1690189B2112908D8049957
:1072980011F0010F04D141F00101C9B20491059226
:1072A800049A12F0020F0DD15B8A7C4A1380A3F571
:1072B800AE630B3B9BB2D72B04D8049840F0020373
:1072C800DBB204931B20FEF787FF0599744B0AB2C3
:1072D800632A05DD642192FBF1F230321A7401E071
:1072E800092A0CDD059A11B2642291FBF2F002FB27
:1072F80010120A2012B292FBF0F230325A7405983A
:1073080002B2642092FBF0F100FB11210A2209B2BB
:1073180091FBF2F002FB101230329A745B4B1B782F
:10732800FF2B08D158495B484B786FF300034B702B
:10733800002117F075FD049A032A40F02182524873
:10734800002143786FF300034370524817F068FD3B
:107358000FE2022E03D1534BC8221A6009E2032E12
:1073680016D1504B1B68002B40F00A824A4800F1A6
:107378004001FEF78FFE1B20FEF72EFF414B5B8A74
:10738800A3F51E630F3B9BB2542B00F2F981F0E189
:10739800042E0CD13B4B988A0CF00EFA002840F0D2
:1073A800EF813D4800F16001FEF774FEE1E1052E32
:1073B80007D1344B988A0CF0FFF9032840F0E0819C
:1073C800D7E1062E40F0D58122786FF3030301320E
:1073D8002270D3E1344800F12001FEF75BFE334B05
:1073E8001B78002B00F0CC81237801332370304BBD
:1073F8001A786FF30302FFF796B82D4EDFF8A480D2
:10740800337813F00F021AD12A4800F12001FEF751
:1074180041FE2948F9F70EFA274902462748F8F7A6
:1074280011FF2548F9F706FA254BA3F81602337819
:107438005A1C62F30303337016F074F891E0012AC2
:1074480016D1D8F80030002B40F09A8116F096F843
:10745800012840F095811B48F9F7ECF919490246D3
:107468001948F9F717FA002840F08A8111486FE0A7
:10747800D8F80020002A40F083810B217BE000BF70
:107488001E0E0020541D0020761D00207C140020B4
:10749800480C0020002C0140A2F6010870140020BE
:1074A800F20100204419002022F701086C14002082
:1074B8006D14002062F7010874010020C421002027
:1074C800282F002092010020292F0020864E337893
:1074D80013F00F080CD185484146FEF7DBFD3378E1
:1074E8005A1C62F303033370814BA3F8028047E10F
:1074F800B8F1010F18D17F48042117F0BAF8002815
:1075080000F03E81794800F12001FEF7C3FD337891
:107518004FF0FF315A1C62F303033370764B642239
:107528001A60734B59802BE1B8F1020FDFF8C8815C
:107538001BD1D8F80030002B40F022816D4804217F
:1075480017F097F8002840F01B81694B588067486E
:1075580000F14001FEF79EFD33785A1C62F30303E5
:1075680033706423C8F800300AE1D8F80020002AF4
:1075780040F006810C21217062F30303A9E05F4902
:1075880010234FF40052CB700D3B8B700A805C487F
:1075980017F020F80A2200215A48F8F7FBFE80204D
:1075A80016F07CFF2378013323704F4B1A786FF362
:1075B80003021A70504BC8221A60E1E05248DFF803
:1075C80044A100F12001FEF765FD9AF80030002B78
:1075D80000F0D6804D48DAF80020434E0260BAF831
:1075E800042082809AF806208271317811F00F0108
:1075F80059D1DFF80481D8F80010002940F0C08084
:107608009AF80410A2F5A6524FF0640B103A0BFB3F
:1076180001229AF805004FF00A0909FB002003939C
:10762800FAF77EFA3A49FAF787FB02469AF8020017
:10763800039BA0F5A65010380BFB030B9AF801002A
:10764800344B09FB00B018600392FAF769FA039A01
:1076580001461046FAF7B4F92F4B1860F9F76CFE9B
:107668001DA3D3E9002382468B46FAF73FF9002889
:1076780000F086805046594619A3D3E90023FAF74B
:107688002BF900287CD0FEF7DFFD337848465A1CDA
:1076980062F303033370C823C8F8003007F082FE92
:1076A800C0B207906CE001296AD10D300799832296
:1076B80000F02AFC104BD3F80080B8F1000F5FD11E
:1076C800404616F0EBFE237801332370337868F3D5
:1076D8000303337054E000BF736891ED7CFF7F4073
:1076E8000AD7A3703D0080406D140020C2F701083E
:1076F8001A250020000C014044190020721D0020AA
:10770800001001408414002022F801080202002021
:1077180000007A4480140020681400208448854EB4
:1077280000F12001FEF7B6FCF37913F0010F27D022
:10773800DFF8488298F8009019F00F0920D17E4BA5
:107748000A2259781878103902FB0011B17019799A
:10775800D878103902FB00117170D9799B791039EA
:1077680002FB0312327013F04DFBF37969F3000347
:10777800F37198F800305A1C62F3030388F800305C
:10778800DFF8FC9199F8006016F001063EF43FAE70
:107798006A4B01221A7014F0A1FF2378092B01D03B
:1077A8000D2B28D1012066490EF07CFC654B664AFA
:1077B8005B7803F01F03D35C644A522B137002D129
:1077C800634B01221A70634B634A03F1200153F89B
:1077D800040B8B4242F8040BF9D1002117A80EF0D4
:1077E8007DFC17A80D2115F039FE5C4B1A78013283
:1077F80002F003021A7099F8006006F00206F6B269
:10780800002E00F08B800CF033FA0FF021FE069862
:107818000322431C93FBF2F202EB42029B1ADBB2F7
:107828000693002B79D1DFF8488198F84960C24661
:10783800002E4DD0022E03D198F80130312B49D0BB
:1078480023780E2B13D1464846490522F9F722F82A
:107858008246002840D1B21F37484349F9F770F8EB
:10786800344B5646DA7942F00102DA7135E00D2BD5
:1078780003D13E483A49072227E0032B22D13C4B4B
:10788800002713F8012F2C2A03D00137FFB2B74283
:10789800F7D113A832493A46F9F752F87B1C07E0AA
:1078A8000AEB03025278303AD2B2092A03D80133DC
:1078B800DBB2B342F4D30AEB0701FA430FA8023153
:1078C800D21802E0264909A8721EF9F739F803E030
:1078D800069E02E0012600E000261E4B204A03F126
:1078E800100153F8040B8B4242F8040BF9D1214BD9
:1078F800214A03F1100153F8040B8B4242F8040BA0
:10790800F9D1402388F811301C3B88F82230023B1B
:1079180088F84B3015F09AFB00E0002699F8003003
:1079280003F0F5036FF3000389F80030FEF76FBD2D
:1079380062F80108D4290020721400201E0E0020CD
:10794800C52E0020C42E0020E02602084A2400206C
:107958006C140020F201002088240020F22300206B
:10796800732C00204BB20208782C002084140020CD
:10797800722C002002020020842C00206D140020AC
:107988004C2C0020AFF30080084B187800F004005E
:10799800C0B250B11A6822F004026FF341021A60B3
:1079A800034B00221A70034B18787047EC23002011
:1079B800A814002090140020084B1B7813F0010F26
:1079C8000AD1074B1B783BB1064B1B6823B9064A03
:1079D800136843F002031360704700BFA914002026
:1079E800A8140020A4140020EC230020064B00213A
:1079F8001970064B06481A6822F0020261F38202E7
:107A08001A601222F8F7C6BCA8140020EC23002044
:107A18009014002038B5094C094922780546F8F732
:107A280011FC23780021E954064B1A6822F004025D
:107A380061F341021A60207838BD00BFA814002005
:107A480090140020EC2300200D4B1B7813F0010F3D
:107A580014D10C490C4A0818137810F8010C0B497A
:107A6800112BC85401D801331370094B4FF4967287
:107A78001A60084A136843F004031360704700BF94
:107A8800A9140020A2F80108A814002090140020CE
:107A9800A4140020EC23002070B5294C002384F89E
:107AA800293084F8283014F8103094F82A2003F08C
:107AB8000F0363F3030284F82A202A2604EB40000C
:107AC800417873431F4D61F3071284F82A20628CB2
:107AD800E95A1D48E28417F0A1F994F82A301A48A7
:107AE80003F00F0306FB03535988013989B217F0D5
:107AF80099F901210A46144817F060F90121124842
:107B080017F04DF994F82A3010481B097343E95AC5
:107B180017F084F994F82A300C481B0906FB035522
:107B28006988013989B217F07BF901210A460748AB
:107B380017F044F905480121BDE8704017F02FB946
:107B4800AA140020AEF801080008004000340140E3
:107B580030B5164C94F82B50A38445F0010500234A
:107B680084F82B50628484F8211084F8203019E0BE
:107B7800C55CA5F13002D2B2092A08D9A5F14102A3
:107B8800D2B2052A9ABFA5F13702D2B22A46084DC9
:107B9800013305EB420292F8515192F850212570B9
:107BA80062700234DAB28A42E2D330BDAA140020ED
:107BB800AEF80108124B10B59A8C0024DA8483F8C9
:107BC800294083F82840224601210E4817F0F6F88C
:107BD80064210C4817F022F932210A4817F022F9DB
:107BE80001212246084817F0E9F86421064817F0F1
:107BF80015F905483221BDE8104017F011B900BF4A
:107C0800AA140020000800400034014010B50021EB
:107C18002C220348F8F7BEFBBDE81040FFF7CABFA7
:107C2800AA14002070B5204C2378042B37D8DFE83D
:107C380003F0030D152A30001C4B012093F82B305C
:107C480013F0010F2ED02070013870BD174B93F838
:107C58002000FFF721FF0223237020E0134DEE8C54
:107C6800EEB9FFF7A7FF95F8203095F821200133EA
:107C7800DBB29A4285F8203001D8042300E00323C0
:107C88002370304670BD094BD88C50B9012323703E
:107C980070BDFFF7BBFF00232370012070BD0020DB
:107CA80070BD002070BD00BFD6140020AA140020AB
:107CB800202102480A46F8F76DBB00BFF2010020F8
:107CC80038B5044608460D46F8F7B4FD98B10319CF
:107CD800202B094BC8BFC4F120001C19002308E061
:107CE80014F8012BE02A14BFEA5C202204F8012CC6
:107CF80001338342F4DB38BDF20100200D4B46F618
:107D080012221B689B6893420FD043F6EE229342DF
:107D18000BD0122B09D0B3F5E97F08D046F6B62070
:107D28001B1A584240EB030070470120704701209E
:107D3800704700BF10150020F0B51F4687B00646F3
:107D48000C46084600211546F8F724FB244B07B1DA
:107D58009F80B3F9041005A801EB8601042207F0FF
:107D680032FB002605AB9B5D013BDBB2B92B34D857
:107D78001D2B4FEA031208D8D31803F5144168469F
:107D8800EE31112207F01FFB0BE01649D3185B18E0
:107D98006A4603F11007186859680833BB4203C2E2
:107DA800F9D12046F8F746FDC7B26846F8F742FD14
:107DB8003818A84203D8E0196946F8F7DDFC684688
:107DC800F8F738FD7B1C1B18AB4203D8E0190649AD
:107DD800F8F73AFB0136042EC4D107B0F0BD00BF56
:107DE8007C150020139C02085FB2020810B5044CF1
:107DF800002120466C22F8F7CDFA0123A37010BDAC
:107E08007C150020044B00225A701A709A7842F0B0
:107E180001029A70704700BF7C1500202DE9F843D5
:107E2800244C8046A3780D4613F0010F3FD06FF322
:107E38000003A37015F0E2F86378002B37D123789C
:107E48000BB90A336370A3781B4F6FF30003A37059
:107E580015F0D4F8217807EB080661180731304689
:107E68002A46F8F76DFD3046F8F7E4FCC6B2AE4294
:107E7800DFF840900FD80CD2002306EB080089F8F1
:107E8800003038180A332021AA1B89F80130F8F786
:107E980081FAAE420BD12178064B6418227A1AB1C6
:107EA80001311970BDE8F8831A700A225A70BDE8CA
:107EB800F88300BF7C150020F2010020054B1A78DA
:107EC8000AB100221A701B7845F6551202FB0311FD
:107ED800FFF7F6BEF6140020F8B505460C4608185C
:107EE800002107F055FA013CE4B26719384607F05B
:107EF80059FAC6B2202E03D83846002107F048FAAE
:107F08000CB1202EEFD9F8BD02F00F03032B22F09D
:107F18007F0230B5D2B20CD94FF47A7491FBF4F4E5
:107F28002025E4B2057002B114B130340470002287
:107F38000130B1F57A7F05DB4FF47A7491FBF4F5E3
:107F480004FB1511022B0BD9642491FBF4F42025B2
:107F5800E4B2057002B114B130340470002201306B
:107F6800632904DD642491FBF4F504FB1511012B4E
:107F78000AD90A2391FBF3F32024DBB2047002B17F
:107F88000BB1303303700130092904DD0A2391FB5A
:107F9800F3F203FB12113031017030BD13B5104BF1
:107FA80001461B689A899C7B12F0100214BF0220BC
:107FB800012034B10B4C9B7C2478634303FB0011F4
:107FC80009B23AB10DF10600022207F0FCF9BDF83A
:107FD800060002E0084607F0E5F900B21CBD00BF44
:107FE800101500202C15002010B50F4B1B689A891E
:107FF8009C7B12F0100214BF0221012134B10B4CFA
:108008009B7C2478634303FB010000B22AB1084932
:108018000222BDE8104007F0D0B9054B1968BDE849
:10802800104007F0B5B900BF101500202C1500202E
:10803800441500203038C0B2092894BFFF20002022
:1080480070470000044B1A786FF300021A70034B54
:1080580000221A70704700BF6D150020F31400202D
:1080680070B58B4CFFF7EEFF2578264605F0F00536
:10807800202D6BD107F09EFC002867D1854B1B781B
:108088003BB92378C3F30312013262F30713237059
:1080980070BD814B1B7803F08003DBB2002B51D0FD
:1080A8007E48F8F7C7FBC4B2C4B17D4E7D4930465F
:1080B8002A46F8F745FC0A2C0BD822463046774961
:1080C800F8F73EFC30192946C4F10A02F8F762F9BC
:1080D80004E0304671490A22F8F732FC704C042259
:1080E80004F10C00A521F8F755F96F4B1A7852B135
:1080F800FF23012A237306D9022A637303D0032AB4
:10810800A37318BFE373694C94F8A33013B9684894
:10811800684902E0664804F1A3010622F8F710FC5A
:10812800654B1B78452B40F06881237813F00C0FC2
:1081380040F06381022243F0100362F301035B4ABB
:10814800137070BD56485D492A464BE1347804F0F7
:10815800F004102C3FD107F02DFC00283BD1202241
:1081680057494F48F8F7ECFB4D4855492246F8F770
:10817800E7FB544B1B7813F0010F06D05248F8F771
:1081880059FB51490246514805E05148F8F752FB5E
:108198004F4902464D48F8F7D3FB3E4B1B781BB9B5
:1081A8004C484D4910221DE14A484C491022F8F725
:1081B800C7FB394B1B7803F08003DBB22BB1424875
:1081C800F8F738FB024646484FE04148F8F732FBDB
:1081D8000246434842E0337803F0F003302B46D19F
:1081E80007F0E8FB002842D12D4C20223D492046CB
:1081F800F8F7A6FBA521052204F10B00F8F7CAF849
:10820800394B1B78042B02D9FF23E37300E002D11A
:10821800FF23A37301E0032B02D1FF23637301E063
:10822800022B02D1FF23237300E00BB1FF23E3727B
:108238002E4B5B7813F0600F05D03F23E372237356
:108248006373A373E3732A4B1B7803F02003DBB239
:1082580033B11F48F8F7EEFA024626481C49C1E038
:108268001948F8F7E7FA024622481749BAE033787E
:1082780013F0F00344D120221F490948F8F760FBA6
:108288001E4B074819888322BDE87040FFF73CBEA3
:108298006D15002074190020481900204C19002081
:1082A800F2010020E46A0208411A00207C1900202B
:1082B8000C0200204F4B0208D8140020A26A0208C2
:1082C8004498020874260020AF990208FF01002094
:1082D800D099020802020020F09D02086598020861
:1082E8000F020020F44B0208281B00207C1D0020F0
:1082F800EC2300200D020020914B0208F01400200E
:10830800502B1ED107F056FBD8B93C4920223C48D7
:10831800F8F716FB3B48F8F78DFA3A4902463A480F
:10832800F8F70EFB3948F8F785FA38490246384815
:10833800F8F706FB3748F8F77DFA3649024636481B
:1083480050E0337803F0F003102B06D107F032FB2E
:1083580018B12B483149202244E0337803F0F00269
:10836800402A43D126482E49203AF8F7E9FA2D4BFE
:108378001B78002B28D02C4B5C7834B92B48F8F7A5
:1083880059FA2A4902462A4824E01B78022B06D1CA
:108398002848F8F74FFA2749024625481AE02648A0
:1083A800F8F748FA244902462148F8F7C9FA012C97
:1083B80003D022D3052C20D80EE02048F8F73AFA4B
:1083C8001E4902461E480DE01E48F8F733FA1D49BB
:1083D80002461748F8F7B4FA1B48F8F72BFA1A4977
:1083E80002461748BDE87040F8F7AABA174A6FF373
:1083F80007131370164B00221A6070BD704B0208E9
:10840800F201002070440208F60100207A440208B4
:1084180006020020754402080D020020D34B020812
:1084280086980208D4230020E5200020D09902086D
:10843800FB010020E9980208AF990208A7980208F2
:108448000B020020F1990208C89802086D15002057
:1084580010150020204B70B5F022204D1A702B7893
:1084680013F0010F0BD01E4C207810F0010006D13C
:108478001C49FFF723FD237843F0010323701A4EAC
:108488003378532B0ED1164C237813F0010F07D0F5
:1084980000201649FFF712FD23786FF300032370BD
:1084A800FFF7D0FD3378232B14D10D4B1B7813F035
:1084B800010F0FD1FFF7C6FD2B780D4A43F00603D5
:1084C8002B701378013BDBB213700A4A52F8232051
:1084D800094B1A6070BD00BF791500206D1500208A
:1084E800151500201D8F0208D8140020FC8E0208E4
:1084F8005B1500205C150020101500202DE9F041C7
:108508005B4BF0225B4D1A702A7802F01003DBB245
:10851800002B2DD1584963F347120B601C462A7073
:10852800564A9A5C2D2A01D00134E4B20133082B53
:10853800F6D1534E3A213046F7F7AAFF38B1801BDF
:10854800C0B20130301821460222FFF7DDFC4D4B46
:108558001B78452B40F089800024204601340EF01A
:10856800CFFF082CF9D12B7843F010032B7036E09D
:10857800454C237813F0010F16D13F4EFFF736FC18
:108588003F4F3168384601310222FFF7BDFC2D23E9
:10859800BB70307846F63E433C496522FFF7CCFB7A
:1085A800237843F00103237003200D21FFF736FCE5
:1085B8002D78304E15F0E00541D110203449FFF7F1
:1085C8007DFC304B1B78442B0DD12B4A13680133AB
:1085D8002A4903F00703C95C2D29F8D01360BDE8C8
:1085E800F041FFF72FBD532B0DD132784E3B63F38B
:1085F80047123270204A27491268062000FB0212EF
:108608005380BDE8F081232B2FD11B4B1D6033789D
:1086180003F0EF0365F347133370FFF713FD237877
:108628001D4A43F0060323701378013BDBB2137035
:108638001A4A52F823201A4B1A60BDE8F081104CF0
:1086480010201849FFF73AFC04F110002821F7F729
:108658001FFF50B1001B3178C0B201302018490902
:108668008022BDE8F041FFF74FBCBDE8F08100BFB4
:10867800791500201515002044150020FD24002040
:10868800F2010020D81400206D1500208315002069
:10869800998E02081A2500205B1500205C15002021
:1086A80010150020BA8E0208434B2DE9F041F02244
:1086B800424E1A703378424D43F0010333702B68F1
:1086C800404C9B7C33B9404B1B7803F04003DBB232
:1086D8002BB10DE0012B0BD111F0E2F840B907F0F6
:1086E800DBFA236800206FF355532360374943E0D2
:1086F800A778DFF8D08007F02003DFB2B7B907F01A
:10870800CBFA2968324B897C1A78384661F3010222
:108718001A70D8F800302D4943F40013C8F8003017
:10872800FFF7CCFB2B4B802283F843200AF0F4FBA5
:10873800804678B12B689B7C012B08D1264B5B784F
:1087480003F01003DBB213B10020244914E0002029
:10875800234911E00AF010FC074610B140462149B0
:108768000AE00AF051FC10B138461F4904E0194BE1
:1087780093F8433013B91D49FFF7A0FB1C4B1B7836
:10878800232B16D1FFF75EFC337843F006033370D2
:1087980007F082FA23686FF35553236009F02EFC23
:1087A800144A1378013BDBB21370134A52F8233092
:1087B8002B60BDE8F08100BF791500206D15002001
:1087C80010150020EC230020481900203E8F0208D5
:1087D8007A260020B117002074260020808F020816
:1087E8005F8F0208C28F0208A18F0208E38F020878
:1087F800D81400205B1500205C150020614B2DE982
:10880800F341F022604E1A703378604D43F0010353
:1088180033702B685E4C9B7C8BB95E4B1B7803F0E6
:108828004003DBB283B15C4B1B7803F00403DBB27B
:10883800ABB1A37803F04003DBB22BB10FE0012BFF
:108848000DD111F02DF850B9F9F73AFC2368002042
:1088580023F480036FF3D7532360504964E0A7786B
:10886800DFF82C8107F04003DFB22FBBF9F728FCB3
:1088780029684B4B897C1A78384661F301021A70D3
:10888800D8F80030454943F4800367F3D753C8F854
:108898000030FFF713FB2B68198A21B900910820D3
:1088A80001220B4606E00BB2012B05D100970E20E2
:1088B80039463A46F9F754FC0AF02EFB074678B1D8
:1088C8002B689B7C012B08D1364B5B7803F0100397
:1088D800DBB213B10020344926E00020334923E0FD
:1088E800F9F7DAFCFF2809D1A07800F08000C0B2BF
:1088F80010B138462E4917E02E4915E00AF03CFB26
:10890800804660B1F9F7B8FEC0B2022802D83846EE
:10891800294909E0062809D83846284904E00AF018
:1089280073FB18B126494046FFF7C8FA254B1B7858
:10893800232B23D1FFF786FB337843F006033370EC
:10894800F9F7BEFB2368204A23F480036FF3D7535B
:1089580023601378013BDBB213701C4A52F82330B2
:108968002B600F4B1B7813F0030F02D10AF0AAFA01
:1089780020B102B0BDE8F04109F040BB02B0BDE84B
:10898800F08100BF791500206D150020101500201A
:10899800EC230020481900207C1900203E8F020893
:1089A8007A26002074260020808F02085F8F020834
:1089B8004690020867900208049002082590020871
:1089C800A18F0208D81400205B1500205C15002038
:1089D80010B5FFF737FB124B2522DA77114B124CF3
:1089E8001B6816219A7C01FB0242517801F00F00A6
:1089F8000F2814D00A2803DD0A2060F30301517000
:108A08009B7C162202FB034463780A2103F00F03C0
:108A1800594306486D32BDE81040FFF775BA10BDDE
:108A2800F201002010150020F82300200E0200207B
:108A38002DE9F74F984BDFF8B0A2F0221A70DAF858
:108A48000030D0469C6847F27803E11A4C4244EB68
:108A58000104DA3A6243914B9D5C9F18C5F3000507
:108A6800EEB29946002E29D130468D49FFF726FAF5
:108A78008C4B1B78232B40F035857B7866F30413E9
:108A88007B70FFF7DFFA884B1A7842F006021A70FB
:108A9800864A1378013BDBB21370854A52F82330BB
:108AA800CAF80030834B1D70834B1D70834B1D70BB
:108AB800834B1E60834B1D7000F014BD824E814DA8
:108AC800337893B1814A4FF4A071137803F01F00F3
:108AD8005B0959430A2303FB00137D49CB18DB7854
:108AE800002B40F06682137084E06E4B1B78532B8A
:108AF80040F0FC8095F80080B8F1000F2ED1404678
:108B0800214611F0AAFC5FFA80FABAF1000F25D0CD
:108B18007B7868F304137B706E4F3A781AB9204655
:108B280011F0B2FB13E0531E6B49002B184603EA01
:108B38000101B8BF02F11E004011002903DA013912
:108B480061F01F01013111F0EBFB00233B7011F0C4
:108B580017FD85F800A00022594BE2E02B78002B86
:108B680000F0278256490A680F460B2A01D10C23C8
:108B780016E00C2A11D1013B6101544A59181170B1
:108B8800554903EA0101002903DA013961F01F019F
:108B98000131204611F0C4FB1CE0092A02D10A2346
:108BA8000B60D0E10A2A27D14B49013B03EA0101B6
:108BB800002903DA013961F01F010131204611F063
:108BC800F1FB2B786201D318DBB2404A591E1170B1
:108BD800404A13704FF00008C7F80080FFF732FAD8
:108BE800162303FB04935A7842F010025A7085F852
:108BF800008014233370DCE1043A042A3FD8374953
:108C0800D2B20878364F60B300200870397841B185
:108C18003448401810F8010C032802D0002840F00E
:108C2800C881013B0A2058434FF4A07E0EFB040084
:108C3800DFF89CE070448018417160011B18D8B2BD
:108C480000EB800000F5E840FC30801806F0A0FB3F
:108C5800387818B1013811F0FBFCAAE10BF0B4F830
:108C6800A7E101200870013B0A214B434FF4A07192
:108C780001FB04331649CB189A1853790AE00F4FB1
:108C88003B7823B901223A700A4A137091E1FFF741
:108C9800D9F900233B708CE179150020F8230020D6
:108CA8005C590208D81400206D1500205B150020BF
:108CB8005C150020F8140020191500202C15002040
:108CC8004415002036150020EE1400202D15002034
:108CD8004E270020E91500201F00008042150020C3
:108CE800E81500202C1B002010150020432B1AD15A
:108CF800964A1278002A40F043812B78002B00F026
:108D08005881934B1A78002A40F05381914B196887
:108D18000C2903D00A2903D02A7014E10B2200E0A1
:108D280009221A600FE1232B7ED1884A1278002A83
:108D380040F026812978DFF818A2002935D09AF862
:108D4800003053B184490F2B0A7084490A7000F22D
:108D5800308101338AF800302BE17E4A1368082BF2
:108D68001ED84FF4A077674301394FF00A0E0EFB67
:108D780001717B4F181F7918C9780627013907FB3D
:108D88000101784800EB810151F8040F01330028F4
:108D980040F0D880032B40F2D580082BF4D9D1E0DD
:108DA800092B40F006810233CCE07B786E4E61F3EC
:108DB80004137B7032781AB9204611F065FA13E073
:108DC800531E6A49002B184603EA0101B8BF02F195
:108DD8001E004011002903DA013961F01F01013139
:108DE80011F09EFA0023337011F0CAFB0AF0ECFF71
:108DF800FFF728F95E4B1A7842F006021A705D4AAE
:108E08001378013BDBB213705B4A52F82330524AA5
:108E1800C8F8003000231370504A8AF800301370E5
:108E28004C4A2B7013605DE32A2B3CD1474A1278D9
:108E3800002A40F0A58046490B784BB14648012BE3
:108E480002704648027040F2B480013B0B70B0E0FB
:108E58002878002800F0AD803E4A1368002B00F007
:108E6800A880092B1AD84FF4A071614301384FF03C
:108E78000A0E0EFB00103A491F1F0818C178062079
:108E8800013900FB0171374800EB810151F8040DED
:108E9800013B002856D1032BF8D853E00B2B40F0A8
:108EA8008880023B4EE0442B1AD1284A1278002AC7
:108EB80066D1274B1B78002B7BD12878431EDBB269
:108EC8001E2B76D8214611F0C8FAC0B2002870D0FF
:108ED800204A13680C2B6CD00A2B6AD028701BE030
:108EE800552B4DD1194A1278002A49D1184B1B78B5
:108EF800002B5ED1287801285BD90238214611F071
:108F0800BDFAC0B2002854D0124A13680C2B50D0B6
:108F18000A2B4ED019490870043B042B13D84FF480
:108F2800A071614301380A2707FB00100C49081893
:108F3800C1780620013900FB01330A4951F8233072
:108F48000BB904331360FFF77DF832E042150020B7
:108F58002C15002044150020F814002019150020B5
:108F68004E270020400D0020E91500201F0000803A
:108F78006D1500205B1500205C15002036150020BB
:108F8800303BDBB2092B14D89B4A1268043A042AF6
:108F98000FD89A4A117861B9994A12784AB1994A10
:108FA8000A27107807FB0033DBB2182B137088BF31
:108FB80011702F78DFF8B082002F5FD198F8000089
:108FC80010F0010012D114B920468F4900E08F49F2
:108FD800FEF774FF98F8003043F6DF2043F00103F2
:108FE80088F8003006F0DEF9894B1870337813B929
:108FF8008848894901E0874888490A22F7F7A0FC90
:10900800204611F019FA864D0146022205F1190091
:10901800FEF77AFF834B1B7803F08003DBB22BB398
:10902800814B1B88EB81337803BB804B18781A4639
:1090380018B9204611F0F4F818E07D4B411E01EAFA
:109048000303002B03DA013B63F01F0301334FF4E2
:10905800A07161430A2505FB03137649CB18DB7819
:1090680013B911F0BBF901E000231370162303FBB9
:109078000494637843F01003637033E24FF4A073F1
:109088006343013F0A2202FB07336A4EF31893F841
:1090980003B06301FF1898F80030FFB213F0010F16
:1090A80045D1FEF7A3FE07EB071101F5E0417C313E
:1090B8001022614806F087F9604B594811229A71CD
:1090C80044230370173BC370791C01300F3AFEF735
:1090D8001BFF494B1B6813B9102059491FE0012B8E
:1090E80002D1102057491AE0022B02D1102056490C
:1090F80015E0092B02D11020544910E00A2B02D1A7
:10910800102053490BE00B2B02D11020514906E0E7
:109118000C2B02D11020504901E050491620FEF7CF
:10912800CDFE98F8003043F0010388F80030334B47
:109138001A789846002A00F0EA8007EB071707F527
:10914800E0477C3710223648394606F03CF90022C1
:109158009146334B995C9A4641B109F101095FFA8E
:1091680089F90132B9F1100FF3D106E003EB0900D8
:109178002021C2F11002F7F70DF998F800004845D0
:109188000BD90138C01906F00DF930B91B4B202155
:1091980018780138C01906F0FBF8DFF8D09099F874
:1091A800003018460193FEF745FF4A46019BDFF859
:1091B800C09018B9432B40F0848001E0432B04D1C0
:1091C800002389F80030202172E0DFF8A8E0244964
:1091D8009EF800C023489C454ED10B78ACF1300C6A
:1091E8000133DBB24FF00A0E0B700EFB0C33C35C7D
:1091F800002B53D10B7051E0441500202C15002092
:1092080042150020E8150020BF590208435A0208F9
:1092180075240020F8010020855A0208A65A020881
:10922800F2010020EC2300205EB20208E9150020BC
:109238001F0000804E270020831500207C15002089
:10924800AE5B02088D5B0208CF5B0208745C020803
:10925800955C0208B65C0208D75C0208F85C020854
:109268001915002020FA01086D150020D8140020D7
:10927800F8140020F51400208EF8003099F800301A
:109288004FF0000C81F800C043B198F800300F2B64
:1092980004D803F1010E954B83F800E0402389F8C8
:1092A800003013780978303B0A2202FB0313C15CB3
:1092B80098F8000001380AF80010381806F068F825
:1092C8000EE08B4B1B7803F08003DBB243B199F8B7
:1092D80000302BB998F80030FF22534403F8012CD2
:1092E80099F8003013B1834A013B137099F80030A4
:1092F800012B10D198F800300F2B02D87B4A01338C
:1093080013707D4A002389F80030137003E00420AD
:109318000C21FEF783FD794B1F681FBB4FF4A07229
:1093280054432B780A22013B02FB03443619757813
:109338002D090F2D00F0D680714CA52104F11C00D9
:10934800063AF7F727F8FF232377002D00F0CA80A5
:10935800012D637700F0C680022DA37700F0C2804C
:10936800E377BFE0012F18D14FF4A07254432B7854
:109378000A21013B01FB03443619737803F00F03FC
:109388000F2B00F0AF80092B04DC01335D485943F3
:10939800BD3AA2E05B4859436AE0022F38D10BF18D
:1093A800FF3B5FFA8BFBBBF1070F98BF564BDFF80B
:1093B80050819CBF5B4493F8647008F11B0088BF20
:1093C800002720210522F6F7E5FF2878C7EB0808D3
:1093D8000138002318E04FF4A07262430A2101FB10
:1093E8000022B25C08EB07011A4112F0010FC7F125
:1093F800000202D08A18DB2101E08A18A52182F830
:109408002010013308F10108DAB2BA42E3D369E067
:10941800032F2FD14FF4A07254432B780A25013B18
:1094280005FB0343F218F35C13F0400F02D0102041
:10943800364906E093785A1ED2B2FD2A06D9344935
:10944800102003B0BDE8F04FFEF738BDFE2B02D167
:1094580010203049F5E710202F49FEF72FFD2F4B3C
:109468002F481B78013B05FB03442E4D2C19A1788E
:10947800832232E0043F042F34D80622FFB20BF1D6
:10948800FF3B02FB0B7B284B284853F82B100A3173
:10949800F7F756FA264B1B7893B1154B1B7803F058
:1094A8008003DBB23BB123482021022203B0BDE890
:1094B800F04FF6F76FBF204B1E48197882220CE058
:1094C8002B780A22013B53434FF4A07202FB043469
:1094D8003619F71917487979BE3A03B0BDE8F04F45
:1094E800FEF712BD03B0BDE8F08F00BF2C150020B9
:1094F800EC230020F8140020191500204415002042
:10950800F20100200D02002020FA0108325C020856
:10951800F05B0208115C0208535C02083615002053
:109528000F0200204E270020400D002002020020DC
:109538004215002010020020E81500202DE9F04710
:109548004C4C4D4F2378F02243F0010323704B4BD2
:10955800DFF85C911A703B68494A9E6847F27803C5
:10956800F01A464246EB000616217143555C531823
:10957800C5F300055FFA85F89246B8F1000F23D1CC
:1095880040464049FEF79AFC99F80030232B6FD1EA
:10959800FEF758FD23783C4A43F0060323701378FE
:1095A800013BDBB21370394A52F823303B60384B29
:1095B8001D70384B1D70384B1D70384BC3F8008038
:1095C800374B1D70BDE8F08799F80020232A23D176
:1095D8005A786FF304125A7010F0D2FF0AF0F4FBB5
:1095E800FEF730FD2378284A43F0060323701378EA
:1095F800013BDBB21370254A52F82330244A3B6002
:1096080000231370234A1370234A1370234A1360EC
:10961800234A1370BDE8F087532A0DD15A78C2F354
:1096280000144CB942F010025A70214630460134F9
:1096380010F076FE202CF8D1304610F0FDFE1623EF
:1096480003FB06A67378C1B213F0100F0AD02029C5
:1096580002D10020134901E013490020BDE8F0477A
:10966800FEF72CBC11480222BDE8F047FEF74CBCBF
:10967800BDE8F0876D150020101500207915002031
:10968800F82300205C5902085B1500205C150020B7
:10969800F8140020191500202C150020441500206E
:1096A8003615002035920208569202080B02002057
:1096B800D81400202DE9F0412D4E2E4F307800F5BA
:1096C800E0405A3005F06EFE3B78C4B213F0010F4B
:1096D80026D0294D2B78552B0AD1EC2C01D0013CF2
:1096E800E4B23078214600F5E0405A3005F050FEEB
:1096F8002B78442B0DD1A4F11403DBB2D72B01D95D
:109708000134E4B23078214600F5E0405A3005F0E3
:109718003FFE2B78532B03D1FEF794FC0AF054FB41
:10972800164B1B7803F08003DBB253B13B7813F080
:10973800010F06D0124820210422BDE8F041F6F7B7
:1097480029BE14F0800F0F4805D12B230A2103747A
:109758006143113006E02D230374373B5C4311301D
:1097680004F520610322BDE8F041FEF7CDBB00BF40
:109778002C1500206D150020D8140020EC230020A3
:1097880002020020F20100201FB5204B20491A7860
:109798001AB1087840F00100087009781C4C11F0E3
:1097A800010F31D01B490978532901D00AB103E0D0
:1097B80082B901221A700DE023290BD100201870FC
:1097C8001549FEF77BFBFEF73DFC237843F00603C3
:1097D800237019E01B78012B16D120210A460F4867
:1097E800F6F7D8FD0E4B68461B681022996805F0FD
:1097F800EAFD002409491DF8040001EB4401013485
:1098080013F06BFF102CF5D11FBD00BF2C150020E5
:109818006D150020D81400202C950208F2010020B4
:1098280010150020034B1B78532B01D1FEF70ABCFF
:10983800704700BFD8140020084BFF281A689368A7
:1098480007D1917B41B10649927C097801FB02332B
:1098580002E0927C02FB0033184670471015002086
:109868002C1500204328F8B504460D46174608D1A4
:10987800114B0A261A7891FBF6F66FF3C3021A7099
:1098880000E00E462046FEF7D5FB90B10A4B303C6F
:109898001A780A2602F00801C9B2002918BF002563
:1098A80006FB05466FF3C30236B21A70BE42A8BF64
:1098B8003E4630B2F8BD00BF6D150020634B2DE960
:1098C800F3411A689846157C977C614C2DB1614824
:1098D80021780222FEF718FB00E02570FF012378AB
:1098E80007F50A47D83707EB43075B4E0BB90DB1AD
:1098F8000FE015B901A8394601E001A8B91E0222F6
:1099080005F061FD9DF80430F3759DF80530337658
:1099180005E006F117003F210222F6F73BFD5B2325
:10992800B375023373764D4B1B7813F0010F61D07A
:109938004B4B1B78A3F13002D2B2092A35D82278D2
:109948000AB9002D40D1474A117814469942464A2F
:1099580001D000211170DFF814E10DF1080C9EF818
:1099680000E0A3F13000E644DFF80CC1117800EB09
:109978008000604400EB010C0131C9B240189CF82A
:109988006CC090F86C000EF804CC117008B1032973
:1099980001D90021117023700DB9384600E0B81EB6
:1099A80001A9022205F009FD17E0232B04D12F4B52
:1099B8001A7892B9013205E02A2B05D12B4B1A7877
:1099C8005AB1013A1A7008E0532B06D1284A533B82
:1099D8001370264A1370FFF725FF264B1B7803F0F8
:1099E8008003DBB2002B2FD0204B1B78F6182023E6
:1099F800F37529E045B31A4B1878A0F13003DBB2B0
:109A0800092B10D81A4A137803B92370013303F0CD
:109A180001031370D8F800302178B3F91020FFF74C
:109A280021FF207005E0432803D1114B1B7803B9AF
:109A38002370104B1B7803F08003DBB223B1054879
:109A480020210222F6F7A6FCBDE8FC8110150020B3
:109A58001A15002000020020F20100206D150020D8
:109A6800D8140020F514002019150020F214002045
:109A780036150020EC23002020FA0108F7B5364EF1
:109A8800364D3378364C6FF34103337013F01CF9BD
:109A9800FFF7C8FE02238DF807302B788BB1314AC7
:109AA800D17941F00101D1712F4A207802EBC3032B
:109AB800D3F8A07093F8A5203978FFF7D3FE387053
:109AC8000DE0337813F0010F06D02378303BDBB27A
:109AD800062B9CBF234AD37003238DF807303378B5
:109AE80013F0010F12D0214B1B7803F08003DBB277
:109AF80063B129781C4B1E4803EBC10393F8A430CB
:109B08009DF80720C0182021F6F744FC2378232B62
:109B180009D1184A2B781268927C013A934202DAEA
:109B28000E4A0133137023782A2B04D12B7813B1F2
:109B38000A4A013B13702378532B0AD111F062F9BA
:109B48000021084B2970DA7961F30002DA71FFF716
:109B580069FE00232370FEBD6D1500203615002018
:109B6800D8140020D429002020FA0108EC23002072
:109B7800F2010020101500202DE9F14F914E924C72
:109B88003378924D232BDFF888820BD12368B3F901
:109B98000800FEF703FA286098F8003043F008033D
:109BA80088F800303378532B40F0E280236848F679
:109BB80085229B68934202D12A68854B05E04AF2C8
:109BC8001422934203D12A68824B1A700EE043F69E
:109BD800DD2293420AD1804B29681A7861F300028A
:109BE8001A7005F0E7FE08B105F002FF236843F696
:109BF800E0229B68934206D1774B29681A7861F373
:109C0800C7121A7019E043F6EA22934206D1724B42
:109C180029685A7861F300025A700EE043F6E72289
:109C280093420AD129686D4B19B11A6842F0005263
:109C380002E01A6861F35D721A60236843F6DA225B
:109C48009B68934202D12A68654B05E043F6E822F7
:109C5800934203D12A68634B1A7008E048F68E22B3
:109C6800934204D12B6813B9584B01221A60236818
:109C7800986848F6CF23984202D12A685A4B05E0E3
:109C880048F6D023984203D12A68584B1A7016E038
:109C980048F6CE23984203D12A68554B1A7015E02E
:109CA80048F6D123984203D12A68524B1A701BE018
:109CB80048F6D223984202D12A684F4B1AE048F658
:109CC800D423984202D12A684C4B13E048F6D52396
:109CD800984202D12A684A4B0CE043F6E233984294
:109CE80002D12A68474B05E049F2DC43984202D189
:109CF8002A68454B1A7000B2FEF776F923689A680D
:109D080043F698139A4231D12968DFF80CB1DFF88D
:109D1800BCA00BEBC1031B793C4FC3F34113012BD0
:109D2800DFF8F8901EDD387800F56650203005F031
:109D38002FFB3B78DAF8001009EB030211720BEBEA
:109D4800C1021279C2F34112032A0BD11E4A1268CA
:109D580090681030C01805F01BFB3B78DAF800203B
:109D68004B441A743B782A6809F80320FFF75AFD18
:109D780098F80030264F13F0010F00F0B1802368E7
:109D8800114F9A6843F698139A4267D13378442B57
:109D98004ED12F7844E01F4B01371B78FFB233B107
:109DA80009EBC7031B79C3F34113012B40DC05F012
:109DB80001FE28B109EBC7031B7913F0100F2FD050
:109DC8002F6035E0D814002010150020441500201D
:109DD80074190020D4230020EA150020EC23002069
:109DE800622C0020312400207626002046270020FF
:109DF800492700204727002078260020EF2500204B
:109E0800A41600208A1000200F1400202C15002012
:109E18006D1500203E0D0020080400202C1B00209A
:109E2800914B03EBC7021279994612F0080FB2D092
:109E38003378552B5ED12E780DE0013EF6B205F051
:109E4800B9FD30B1884B03EBC6031B7913F0100F33
:109E580001D02E604EE0002EEFD14BE005F0AAFDB8
:109E680000282CD03B6843F6C4219A688A4203D064
:109E780046F6AA718A4204D13078B5F900102D222D
:109E880019E0A2F56A516139052903D943F6E92198
:109E98008A4201D1012307E043F6E0218A4202D039
:109EA8000A318A4202D100232B6023E03078B5F9C9
:109EB8000010B3F91020FFF7D5FC28601AE03B68C2
:109EC8006A4A99688A18012AF0D832782F2A11D953
:109ED800B3F9103030339A420CDC303A2A6009E08A
:109EE8002368B3F90800FEF759F828603B7843F077
:109EF80008033B70FFF796FC216843F6D2228B6873
:109F080093420BD12B6813B959485A4901E0584874
:109F180059490222F6F714FD0226D2E0534A9A184C
:109F2800012A17D82B6813B95448554908E0012B62
:109F380002D15248534903E0022B05D14F485249F8
:109F48001022F6F7FDFCBBE0032B40F0B9804B482C
:109F58004E49F5E748F6D32293424D4F0DD1296873
:109F68000A22B1FBF2F302FB13123032FA773033D4
:109F78002E22BA777B770326A3E043F69812934202
:109F88005ED12E68384D102255F8361007F11000B2
:109F980005EBC605F6F7D4FC2D7905F00705012D6C
:109FA80002DC781D3B4910E0022D0AD13A490B2208
:109FB800781DF6F7C5FC394BB81D19782A460131CA
:109FC8003BE0032D09D13649781D0B22F6F7B8FC82
:109FD800324BB81D197801312EE0042D02D1781DBD
:109FE800304903E0052D10D12F49781D2B4D0B2248
:109FF800F6F7A6FC2978B81D01310222FDF784FF87
:10A00800297807F10A00093116E0062D58D1234DA9
:10A0180026490B222648F6F793FC29782548013172
:10A028000222FDF771FF2978234809310222FDF742
:10A038006BFF2978214811310222FDF765FF3FE0C7
:10A04800B1F91060092E04DD632ECCBF0326022669
:10A0580000E00126C6F120003818296846F0800281
:10A06800FDF752FF2DE000BF080400203175FFFF07
:10A0780010020020F0FA0108F2FA0108020200209A
:10A088000A9902082B9902084C9902086D9902084E
:10A09800F2010020B79A0208129A02082C15002033
:10A0A800969A0208549A0208339A0208759A020886
:10A0B800F7010020F8010020FC0100200002002028
:10A0C800102698F8003013F0010F0BD0264B1B78A0
:10A0D80003F08003DBB22BB124482021801B3246D9
:10A0E800F6F758F9224EB37803F00203DBB2002BDF
:10A0F80036D0FDF703FE1F4D034628B92878F11D19
:10A108006522FDF719FE08E0B2792978B388F01DB9
:10A1180001FB023109B205F056F9236846F6AA7226
:10A128009B6893420FD006DC43F6C42293420AD0C0
:10A1380043F6784205E046F6EA72934203D048F6C1
:10A148008E2293420CD105200B21FDF767FE29785A
:10A1580009480131022201B0BDE8F04FFDF7D4BE35
:10A1680001B0BDE8F08F00BFEC23002012020020F0
:10A178007C1500202C150020F3010020F0B5114BB0
:10A188001F78114B303F1E680DE0D6F814C01CF83C
:10A1980003C00133644501D112E00023DAB28242E0
:10A1A800F3D301350D70094B0622094902FB073329
:10A1B8000D785B1993F8D440002CEED10C70F9326D
:10A1C8001046F0BDD81400201015002020FA010810
:10A1D800191500202DE9F74F984C994925680878FA
:10A1E800AB682E8A9AB200FB0626074647F2AC6097
:10A1F8008342B6B288460BD1924B1A785B7802F04C
:10A208000702C3F3420303EBC20306EBC3062CE0C9
:10A2180047F66C018B4212D18A4B8B481A785978D1
:10A2280002F0070288235A43C1F34201773B03FB3C
:10A23800012320210822F618F6F7ACF815E047F6B6
:10A2480024418B420BD17F4B1A785B7802F00702CE
:10A25800C3F3420303EBC2039B01F61805E0B3F511
:10A26800E97F04BF3B4602EB4306784F784D3B78C5
:10A2780013F0010F54D123689A6846F6B2639A42E4
:10A2880004D046F6B2439A4240F04681714B1B789F
:10A298002A2B3CD1704B93F8009009F1010909F081
:10A2A800010983F80090B9F1000F1BD046F6B243BC
:10A2B8009A4208D1694B46F63E329A809A7842F023
:10A2C80002029A7028E1202110226548F6F762F808
:10A2D80098F8003000205901C918624BC918FDF7D9
:10A2E800EDFD19E1FDF782FD236848469A6846F6B8
:10A2F800B2439A420CBF5C495C49FDF7DFFD98F810
:10A3080000105B4801310222FDF7FEFD04E1552BE8
:10A3180002D0442B40F000814F4B00221A70FBE022
:10A3280023685869F6F786FA4A4B834693F800A0E3
:10A338009946BAF1450F02D14E4B00221A70504689
:10A34800FDF778FE00284ED04B4B5FFA8BFB1A784E
:10A3580052450ED15846FFF711FFFF2804D1584641
:10A36800FFF70CFFFF283ED0444B1A7801321A70D1
:10A3780015E0DFF808A100228AF80020584601936A
:10A38800FFF7FCFEFF28019B04D09AF80020013259
:10A398008AF8002099F80020FF281A7023D0216835
:10A3A800374A4B6910601B5C886846F6B261884280
:10A3B8001360924610D1562B01D0542B0CD198F82B
:10A3C8000030123BDBB2022B06D82B7830B2C01813
:10A3D80004F0E8FFCAF800002B7830B2C018DAF8A9
:10A3E800001004F0D5FF99F80030552B17D12368D9
:10A3F800997C0F2913D92A7808398A42144B01DA33
:10A40800083200E000221A70144B9B7803F0020314
:10A41800DBB20BB1FDF7F6FC184B00221A7099F865
:10A428000030442B3BD123689A7C0F2A37D92978EE
:10A43800074B072926D90839197025E0101500207F
:10A448002C15002031150020020200206D15002077
:10A4580036150020D8140020781500207C1500201F
:10A46800F2010020B5810208C67F020808800208B0
:10A47800F3010020F2140020F51400201915002023
:10A4880044150020083A1A70914B9B7803F0020398
:10A49800DBB20BB1FDF7B6FC8E4B00221A7099F8AF
:10A4A8000030432B0CD1236830B25B6919788A4B92
:10A4B80019602B78C01804F06BFF864B00221A70C5
:10A4C80099F80030232B13D122682B78927C013A1B
:10A4D80093420DDA814A013313707E4B00221A70C1
:10A4E8007B4B9B7803F00203DBB20BB1FDF78AFCD0
:10A4F80099F800302A2B0FD12B786BB1774A013BA2
:10A508001370744B00221A70714B9B7803F002038E
:10A51800DBB20BB1FDF776FCFFF784F9704A2B78B4
:10A5280011789246994288BF137012780F3293427D
:10A5380002DD6B4A0F3B137023684FF0000B93F852
:10A548001290B9F10F0F9ABFC9F120095FFA89F982
:10A558004FF010099AF8003030B2C018584404F08F
:10A5680021FF604B03F8090009F101095FFA89F935
:10A57800B9F11F0F05D822680BF1010B927C9345A6
:10A58800E8DB3A7812F0010F16D022685649927C1F
:10A5980009780F2A01F0800198BFC2F11002C9B2F0
:10A5A80094BFD2B2002239B129789AF8000010314C
:10A5B8009A18091A5F2353542368986849F2DA43B2
:10A5C800984209D1494B1B78532B05D104F0EAFE78
:10A5D800474B187004F0D6FF3D4EB37803F00203E2
:10A5E800DBB2002B55D0FDF789FB034688B92268FA
:10A5F80047F6244192688A420BD046F6B2418A4215
:10A6080014BF287898F80000F11D6522FDF794FB27
:10A6180010E02368B2799B683648B3F5E97F0CBF30
:10A6280098F800102978B38801FB0231B27909B291
:10A6380004F0C9FE23689A7C032A08D99A6847F26D
:10A64800AC618A4203D046F6B2418A4213D19B6874
:10A6580047F2AC6293420BD13B7813F0010F01D063
:10A66800102013E0202107222348F5F793FE10E07D
:10A67800B3F5E97F02D105200B2108E046F6B24286
:10A68800934202D10020102101E000200721FDF7AC
:10A69800C5FB23689A7C032A16D9B27802F0020215
:10A6A800D2B28AB19B6847F2AC6293420CD046F6AC
:10A6B800B242934208D0297810480131022203B0EF
:10A6C800BDE8F04FFDF720BC03B0BDE8F08F00BF38
:10A6D8007C1500201915002044150020361500208F
:10A6E8002E150020F2010020EC230020D8140020B1
:10A6F800F71400208315002002020020F301002037
:10A708002DE9F74F874C884F2368884E9968B3F92D
:10A7180010303A78B3F1010848BF03F106084FEA50
:10A72800E808337808F1010812F0010F03FB081854
:10A738007F4D00F0AD807F4B1A789946432A4DD162
:10A7480028780FFA88FA0AEBD00004F02BFE22686A
:10A75800794B916846F2A2529142186001D12A7849
:10A768003AB12A78012102F0070211FA02F25040A8
:10A778001860287819780AEBD00004F009FE2368DD
:10A7880047F24A029B68934209D1694B1A786B4B8E
:10A7980003EBD203684A126883F89C201EE046F651
:10A7A8005222934205D13178002001310AF08CFB06
:10A7B80014E046F2686A4FF0000B23689B68534523
:10A7C80004D101200BEB00010AF07EFB0AF1080A14
:10A7D80046F288639A450BF1010BEED199F80030E7
:10A7E800232B10D122682B78927C013A93420ADA03
:10A7F8004F4A01331370524B9B7803F00203DBB2CC
:10A808000BB1FDF7FFFA99F800302A2B0CD12B7801
:10A8180053B1474A013B1370494B9B7803F002033D
:10A82800DBB20BB1FDF7EEFA99F80030552B14D1D5
:10A838002368997C0F2910D92A7808398A423C4B19
:10A8480001DA083200E000221A703D4B9B7803F0D1
:10A858000203DBB20BB1FDF7D5FA99F80030442BAF
:10A868007FD123689A7C0F2A7BD92978304B072916
:10A8780002D90839197001E0083A1A70304B9B78F0
:10A8880003F00203DBB2002B6BD0FDF7BBFA68E0E4
:10A8980048F6452399420DD1264B1B78A3F1310187
:10A8A800C9B2032906D842F006023A700722534378
:10A8B800573B337023689A6843F6E3339A4250D182
:10A8C8001C4B1B782A2B45D11E4B93F8009009F19D
:10A8D800010909F0010983F80090B9F1000F13D0BC
:10A8E80033781B2B08D9164B46F63E329A809A7855
:10A8F80042F002029A7034E05A011349D31800203A
:10A90800C918FDF7DBFA2CE0FDF770FA48460F4945
:10A91800FDF7D4FA31780E4801310222FDF7F4FA36
:10A928001FE000BF101500206D1500202C15002019
:10A9380036150020D8140020441500202C1B0020B8
:10A948007C15002038150020B4850208728502089D
:10A95800F3010020552B01D0442B02D17D4B00225E
:10A968001A70FEF75FFF7C4A2B781178934699425C
:10A9780088BF137012780F32934202DD764A0F3B7C
:10A98800137023684FF0000A93F81290B9F10F0F73
:10A998009ABFC9F120095FFA89F94FF010099BF8AD
:10A9A80000004FFA8AF318180FFA88F202EBE00059
:10A9B800019304F0F7FC9BF80020019B5FFA80FCF0
:10A9C8009B1803F0070316E04CFA03F063490133C0
:10A9D80000F0010000280CBFA520DB20DBB201F845
:10A9E80009000AF1010A09F10109082B5FFA8AFA3C
:10A9F8005FFA89F903D0B9F1200FE5D109E0B9F17F
:10AA0800200F06D023684FFA8AF19B7C8918994257
:10AA1800C5DB3B7813F0010F15D0236850499B7CA8
:10AA280009780F2B01F0800198BFC3F11003C9B258
:10AA380094BFDBB2002331B1297810318A1A474913
:10AA4800CB185F219954DFF8248198F802304746E3
:10AA580003F00203DBB2002B63D0FDF74FF9034686
:10AA680000BB226846F6522192688A4206D02431F9
:10AA78008A4203D043F6E5118A4204D13078394935
:10AA88006522002309E043F6E3318A4208D1307891
:10AA98001C38C0B208F107016522FDF74DF918E02E
:10AAA8002878F7E7236846F612229B68934203D07A
:10AAB80043F6EE22934202D1BA79317801E0BA79AD
:10AAC8002978BB88274801FB0231BA7909B204F01A
:10AAD8007AFC23689A7C102A02D905200B211EE0F3
:10AAE8009B6846F6122293420ED006DC43F6E51226
:10AAF800934209D043F6EE2204E046F652229342EE
:10AB080002D02432934201D1102007E043F6E33209
:10AB1800934202D10020102101E000200721FDF717
:10AB28007DF9236846F6B6219A688A420FD046F620
:10AB380070118A420BD09B7C102B08D929780A48BF
:10AB48000131022203B0BDE8F04FFDF7DDB903B0D3
:10AB5800BDE8F08F381500202E150020F2010020E6
:10AB6800EC23002083150020F30100207C15002031
:10AB78002DE9F04F714E89B033689C689F7C122C88
:10AB880001D00B2C0DD16E4A1778303F122CFFB232
:10AB980009D19B7B3BB96B4BD879FEF74DFE054637
:10ABA80015E0013FFFB2FF20FEF746FE4AF24813C8
:10ABB8009C4205460BD14AF2152004F0F3FBC0B2C3
:10ABC800069020B15F4B9B790BB1FDF73BFA3368D8
:10ABD8009A68122A17D19B7BC3B1594B1878313820
:10ABE800401904F0DFFB574B5FFA80FA9B7973B189
:10ABF800AAF13003DBB2092B09D8534B1B7833B9C0
:10AC0800FDF720FA03E04FF0000A00E09A464F4CA7
:10AC1800DFF84C812178DFF84C9111F0010100F048
:10AC28006B8198F80030DFF840B100218BF80010F4
:10AC3800184605910493FDF7FDF9DFF830B1059941
:10AC4800049B002800F0B5804148DFF824E101703A
:10AC58009EF800003F4A984213603B4940F08A80C2
:10AC680033689B8903F00F03032B21D1A0F1300C2B
:10AC78000A2000FB0CF0384BDFF8E0C093F800E046
:10AC88000390704407900EF1010E1CF80000DDF8E7
:10AC98000CC05FFA8EFE106083F800E00CEB0E002B
:10ACA800DFF8B8E01EF80000002870D118706EE0D8
:10ACB800082B2CD1A0F1300C27480CEB8C0E037814
:10ACC8000793264B9E44079B734493F86CE00793C5
:10ACD800224BBEF1000F01D180F800E090F800E0AF
:10ACE8000CEB8C0C634403EB0E0C0EF1010E5FFAB7
:10ACF8008EFE73449CF86CC093F86C30C2F800C0A8
:10AD080080F800E0002B42D1134803703FE0072B86
:10AD18000ED130280ED1DFF840E09EF8003003B1A4
:10AD28000538013303F0010310608EF800302EE07F
:10AD3800062B2CD10B78013328E000BF101500201A
:10AD4800F714002039150020361500206D15002055
:10AD5800672C0020441500201915002020FA01084E
:10AD6800D81400201B150020F3140020F81400202C
:10AD7800F514002099488EF800309BF800304FF009
:10AD8800010C80F800C013B10B7863440B704023AA
:10AD98008BF800300B78BB4202D3914B781E1870A9
:10ADA80008781168281804F0F3FA237843F00403AC
:10ADB800237098F80030232B1ED1894B7A1E1878FF
:10ADC800904219DA0130C0B218702818049304F0C0
:10ADD800E9FA049B20B918782021281804F0D8FA39
:10ADE800804B40221A7023787C4A43F00403237076
:10ADF80000238BF80030137098F800302A2B10D1FC
:10AE0800774B1A786AB1013A1A70764B40221A7059
:10AE18002378724A43F00403237000238BF8003030
:10AE2800137098F80030432B1ED16D4B1878B84238
:10AE380005D228182021049304F0AAFA049B9BF851
:10AE4800002032B91B787A1E934202DA644A013331
:10AE580013702378634A43F00403237000231370AC
:10AE68005E4A8BF8003013709BF8003013B15E4ACD
:10AE7800013B13709BF80030012B0ED1584B1A7808
:10AE8800BA4201D201321A70544A00231370227850
:10AE980042F0040222708BF80030237803F0040299
:10AEA800D2B2002A3BD0514A6FF3820313700021BB
:10AEB80011224F48F5F76EFA4E4A494B11781B7824
:10AEC800994288BF137011780F318B4202DD4949CE
:10AED8000F3B0B704848137801781022C91849199C
:10AEE800434804F070FA4248F5F7A4FCC2B20F2AAE
:10AEF80015D809EB02000DE011224846F5F74AFA89
:10AF080010222946484604F05EFA4846F5F792FCB6
:10AF1800024648442021C2F11002F5F73BFA98F89E
:10AF28000030532B20D133689A684AF248139A426A
:10AF380008D1284604F036FA20B14AF2152001213A
:10AF480004F026FA28463946FCF7C6FF264A0023AD
:10AF58001370294A01201370264A01461370009382
:10AF68000246034609F0DCFFFEF75CFC204B234A4F
:10AF780003F1100153F8040B8B4242F8040BF9D18A
:10AF880033689A68122A50D19B7B002B4DD0AAF1C6
:10AF9800300A5FFA8AFABAF1090F46D8237813F013
:10AFA8000107174B08D09A7932B10D4A1178154A22
:10AFB8001278313A914238DA9B792BB9104BDA7909
:10AFC800114B1B789A4230D00E4B054A18781178ED
:10AFD800054A30381278002325E000BF19150020F3
:10AFE80036150020672C0020F81400206D1500206D
:10AFF8001B1500202E150020F3140020020200204B
:10B0080039150020F71400202C15002017B199429B
:10B0180000D132B9DFF8F4C04FF02A089C448CF80C
:10B0280010800133DBB28342F0DB326893680B2B6C
:10B0380001D0122B0AD1334B991D13F8010B20288C
:10B0480002D10D3003F8010C8B42F6D192684AF216
:10B0580048139A4210D12C4B9B796BB1069B5BB17C
:10B068000027781904F09EF918B1284B2A22DB1919
:10B078001A740137102FF4D1237813F0010F0ED072
:10B08800234B1B7803F08003DBB243B1214B224AE8
:10B098001B78127810339B1A1C4A5F21D1541F4C1D
:10B0A800A37803F00203DBB2002B28D0FCF726FEBE
:10B0B8001B49034628B908786522E11DFCF73CFEC8
:10B0C80012E03068B4F90430A27984680978122C47
:10B0D80001FB023105D1807B18B90B49C97902FB04
:10B0E8000131104804F06FF933689B68122B06D1C0
:10B0F8000820014609B0BDE8F04FFCF78FBE09B043
:10B10800BDE8F08F0202002039150020F20100206E
:10B11800EC230020361500202E1500207C15002079
:10B128002C1500208315002024282DE9F041144611
:10B1380009D15C4B5C481978801801310222FCF770
:10B14800E3FE0234AAE0E72809D1564B564819789D
:10B15800801801310322FCF7D7FE03349EE0A328B0
:10B168002AD1504D2B78172B15D810464F49FCF78C
:10B17800A5FE4E48F5F75EFB2A2124184A48E4B29A
:10B18800F5F786F9002800F08A8029780222013133
:10B19800FCF7BAFE83E05901C918454D01F566511F
:10B1A800613110466918FCF789FE05F57250583070
:10B1B800F5F740FB241871E0F22821D1394F3A4DB8
:10B1C8003978072605EB0208B1FBF6F14046013154
:10B1D8000222FCF799FE39782D23B1FBF6F688F8A0
:10B1E8000230F3009E1B8B1B324FDBB207EB83034D
:10B1F8001988E21CA9529B78A818837006344DE080
:10B2080025280BD12C4B46F63E329A8045229A715E
:10B218009A78053842F002029A703CE05E280BD119
:10B22800254B46F63E429A8045229A719A783E38D6
:10B2380042F002029A702EE07C280BD11E4B46F297
:10B2480022029A8011229A719A785C3842F002029E
:10B258009A7020E0EC280BD1174B46F682429A8070
:10B2680045229A719A78CC3842F002029A7012E01C
:10B27800A7280BD1104B46F6A2429A8045229A7114
:10B288009A78873842F002029A7004E0E02801D1E7
:10B29800541C03E018B1044B18550134E4B220469D
:10B2A800BDE8F0812C150020F201002094810208ED
:10B2B800BC440208716802087C15002038B50A4BA6
:10B2C80045F655151B78002405FB030507E0074BD9
:10B2D80022461978FFF728FF041B2D190446287801
:10B2E80008B11F2CF3D938BDF61400202C15002006
:10B2F80070B5002543F6FA44204604F053F8064694
:10B3080004F1080004F04EF816F0FF0F06D020F004
:10B318007F0010F0FF0F01D00135ADB246F21903DE
:10B328009C4201D00934E7E7284670BD38B5B0F92A
:10B3380000500B4C05EBC50505F57455023528463C
:10B3480004F030F8C1B211F0800F07D023882846E6
:10B35800013B01F07F01238004F01AF8208838BDF2
:10B36800F0140020454B2DE9F74F1B88444A04464A
:10B3780089461788DFF80C8123B14FF0000A0AE0EC
:10B388009A4608E00529FBD198F8003043F00403F9
:10B3980088F8003070E098F8003013F0030F0BD0F5
:10B3A80013F0010F02D0B4F1FF3F05D103F00203FF
:10B3B800DBB21BB1012C01D03F19BFB23BB2B3F1D4
:10B3C800FF3F04D0B3F57A7F08BF002701E040F2C1
:10B3D800E7370FFA87FB0BEBCB0303F5725303F147
:10B3E8007A00019303F0DEFF10F0FF0F019B16D0E7
:10B3F800B9F1050F09D103F1820003F0D3FF20F062
:10B408007F0010F0FF0FC6D022E0B9F1000F1FD067
:10B4180003F1820003F0C6FF00F07F0618E00AF18E
:10B42800010AB4F1FF3F1FFA8AFA04D198F80030F4
:10B4380043F0010305E0012C05D198F8003043F0F2
:10B44800020388F80030BAF57A7F0DD03D46A2E7AE
:10B458004E4505D0B9F1000F02D0B9F1050F9AD1C8
:10B46800BAF1000F05D000E03D46054A2DB215603F
:10B4780002E0034BC3F800B0BDE8FE8FF0140020D3
:10B488004415002048150020F0B503789BB05A1EDB
:10B49800D2B26B2A0F4600F2C8805E01644AF318E4
:10B4A8009B18644A45F655161278457806FB02360D
:10B4B800E7213046F4F7ECFF0446F0B930467C212A
:10B4C800F4F7E6FF0446C0B930462521F4F7E0FF5B
:10B4D800044690B930462421F4F7DAFF044660B9EF
:10B4E80030464021F4F7D4FF044630B93046F921FC
:10B4F800F4F7CEFF0446002876D0A41B0FB14E48BF
:10B5080000E04E4831462246A619F5F719FA3046AA
:10B51800E721F4F7BDFF30B128466946652246F6B3
:10B528008243FCF709FC30467C21F4F7B1FF50B1A7
:10B53800691EC9B201EB011101F5C041684622310B
:10B54800112203F040FF30462521F4F7A1FF38B15E
:10B55800681EC0B26946652246F63E33FCF7ECFB2E
:10B568003046F921F4F794FF38B1681EC0B2694635
:10B57800652246F63E43FCF7DFFB30464021F4F7F0
:10B5880087FF50B1691EC9B201EB011101F5E04115
:10B5980068467C31112203F016FF30462421F4F767
:10B5A80077FF50B10FB1244800E02448001929461C
:10B5B8000222FCF7A9FC02340BE00FB11E4800E0A0
:10B5C8001E4800196946F5F7D7F86846F5F732F9C5
:10B5D8000419002F29D01A4B9A781C1942F002023C
:10B5E8009A700023E37116E03046F5F723F9054613
:10B5F8001FB9124831462A4615E0102810DD2A46A0
:10B608000D483146F5F79CF90D4B9A785D1942F0D3
:10B6180002029A70EC7110200146FCF7FFFB04E06F
:10B62800084831461022F5F78BF91BB0F0BD00BF72
:10B638002E6C0208F6140020831500206D1E0020D1
:10B648007C150020020200200C4B1B7813F001022D
:10B6580002D000200A4905E003F00200C0B218B188
:10B6680008491046FCF72ABC03F00403DBB20BB10F
:10B678000549F7E705480121FFF706BF48150020EF
:10B68800784C0208574C0208994C02086F150020A4
:10B6980070B5124D124C00201249FCF711FB2846D8
:10B6A800A1780222FCF730FCE81CE1780222FCF7C2
:10B6B8002BFC05F1080021790222FCF725FC05F195
:10B6C8000B0061790222FCF71FFCA17905F10E003D
:10B6D8000222BDE87040FCF717BC00BFF201002051
:10B6E8006F15002030FB01082DE9F3414F4F504CF6
:10B6F8003B689D7C237813F0010F2FD1022243F67B
:10B70800F8410DF1060003F05EFE4A4EBDF8063022
:10B718004FF0FF3033602946FFF724FE237843F0CB
:10B7280001032370444B1B7813F0030F14D1B6F9AF
:10B738000010424801EBC10101F572517A3109222A
:10B7480003F041FE3E4B1B881BB13046FFF7EEFD70
:10B7580010B90020FAF700F9FFF79AFF394E33784D
:10B76800552B0CD1DFF8D080FCF740FB98F800305F
:10B778004FF0FF306FF3410388F800300CE0442BA2
:10B788002AD1DFF8B480FCF731FB98F800300120AB
:10B798006FF3000388F800302946FFF7E3FD98F8B7
:10B7A800003013F0030F15D1224D2448B5F90010CD
:10B7B800092201EBC10101F572517A3103F003FE50
:10B7C8001F4B1B881BB12846FFF7B0FD10B900209E
:10B7D800FAF7C2F8FFF75CFFFFF736FF3378232B41
:10B7E80021D1154B1A7802F0FC026FF382021A700D
:10B7F800FCF728FC144B9A786FF341029A70134BAC
:10B808001D782DB9FCF7FEFAFCF7F0FA3D600AE066
:10B818002278013DEDB242F0060222701D700C4BF9
:10B8280053F825303B60BDE8FC8100BF10150020AF
:10B838006D15002044150020481500206F150020C4
:10B84800F0140020D81400207C1500205B1500207F
:10B858005C1500202DE9F0411646104A0F46537832
:10B868000E21C3F342034B43117803F5EC433C33F9
:10B878000B4D01F00701044603EB4101022203F0DE
:10B88800A2FDE81921780222FCF73EFB6178A8198D
:10B898000222BDE8F041FCF737BB00BF311500209C
:10B8A800F2010020044B02225978044BC1F34201F3
:10B8B80018180131FCF728BB31150020F2010020CF
:10B8C80010B5074B074C1B78074A03F0070304EB36
:10B8D80083031C88111814529B788B7010BD00BF0D
:10B8E8003115002071680208F2010020084B1B780E
:10B8F8009B0902D0012B06D102E01020054904E083
:10B908001020054901E005491020FCF7D7BA00BF0F
:10B9180031150020B7580208D8580208F95802080B
:10B928002DE9F041DFF868800F4698F80010174DB0
:10B93800C1F382010446164605F1080001310222CE
:10B94800FCF7E2FA98F80010042201F01C0101F556
:10B958000A412431204603F036FDE81921780222F5
:10B96800FCF7D2FAF81C281861780222FCF7CCFA06
:10B97800A819A1780222FCF7C7FAF01CE178281868
:10B988000222BDE8F041FCF7BFBA00BFF201002077
:10B99800F4140020064B1B7803F08003DBB233B1AC
:10B9A800435C04482021C0180222F4F7F3BC704716
:10B9B800EC230020F20100202DE9F743484D494CC3
:10B9C8002B6821789B68022203EB41010DF10600E8
:10B9D80003F0F9FCBDF806604FF46163B6FBF3F1C0
:10B9E80003FB11663C22B6B2B6FBF2F302FB136608
:10B9F8005FFA81F8DFB23A3A3B484146FCF784FAED
:10BA0800F6B2022239483946FCF77EFA0222384853
:10BA18003146FCF779FA374BA9461B7813F0010F2A
:10BA28004BD0354B354D1878232804D12B78012B72
:10BA38003FD8013305E02A2805D12B78002B38D0D0
:10BA4800013B2B7035E0A0F13003DBB2092B01D9A3
:10BA5800432828D12B7833B941461122FDF702FF3C
:10BA68005FFA80F80CE0012B05D139463B22FDF73F
:10BA7800F9FEC7B204E031463B22FDF7F3FEC6B239
:10BA88003946324640460BF092FED9F80030ADF800
:10BA980006009B6820780DF1060103EB40000222A6
:10BAA80003F08BFC05E0532803D100232B70FDF72E
:10BAB800B9FE13482978FFF76DFF65222078002327
:10BAC8001049FCF739F905200B21FCF7A7F9217873
:10BAD8000D4801310222FCF717FABDE8FE8300BFCA
:10BAE800101500202C15002002020020080200205A
:10BAF800100200206D150020D814002036150020F3
:10BB080041FB010883150020F301002073B59A4B0F
:10BB18009A4D1A7812F0010F05D12A7812F03802DE
:10BB280004BF2A706A701A78934E42F001021A70A4
:10BB38002B78924C13F038023ED191490978552957
:10BB480004D113F0070F2FD0DA1D0AE044290CD1D5
:10BB580003F0070201323D3992FBF1F1C800411AA6
:10BB6800521A62F3020323701EE053290AD1C3F369
:10BB7800C201013161F3C5032370637862F34303A3
:10BB8800637011E023290FD1FCF75CFA33787D4A02
:10BB980043F0060333701378013BDBB213707A4A23
:10BBA80052F82320794B1A6000207949FCF786F96E
:10BBB8001C20FFF785FEDDE0082A2ED175490020FC
:10BBC800FCF77CF90620FFF76DFE0C20FFF778FEE6
:10BBD8001521182201A8FFF73DFE694B1B78552B4C
:10BBE80006D1637803F0FE03C3F34202013A07E08B
:10BBF800442B0BD1637803F0FE03C3F342020132F6
:10BC080002F0030262F343036370B3E0532B28D0BE
:10BC1800232B40F0AF802378A6E0102A51D15D494C
:10BC28000020FCF74BF90620FFF73CFE0C20FFF73D
:10BC380047FE1521182201A8FFF70CFE6178564827
:10BC480001F00101FFF7A6FE4D4B1878232801D01B
:10BC58002A2804D16378DA4362F30003D4E753282F
:10BC680004D12378C3F3C202013280E0A0F130038B
:10BC7800DBB2092B01D943287CD16B7802AA03F0E7
:10BC880001033B21D41883F001024B43172606FB1E
:10BC9800023214F8041CFDF7E5FD04F8040C6B7877
:10BCA8000E22C3F342035343287803F5EC433C3395
:10BCB80000F0070003EB400001A90C3A03F07DFBFC
:10BCC80058E0182A4DD133490020FCF7F7F8062030
:10BCD800FFF7E8FD0C20FFF7F3FDFFF707FE284B01
:10BCE8001B78552B07D1237813F0C00F42D0C3F32C
:10BCF8008112013A06E0442B07D123789A09012AD8
:10BD080038DC013262F3871333E0232B04D1237824
:10BD1800C3F3C202023A2AE0532B2BD1FCF792F963
:10BD280033781E4A43F006033370164B16481978C9
:10BD380040F82120013119702378C3F3C201013181
:10BD480061F3C503C3F381112370104B11B10129AD
:10BD580004D101E01C3202E0114A00E0114A1A60E5
:10BD680008E0114A00211170C3F3C202013A62F3DC
:10BD7800C50323707CBD00BF6D1500203115002060
:10BD8800D81400205B1500205C1500201015002039
:10BD9800755802089658020844FB010848FB010838
:10BDA80080FB01089CFB01083615002073B5494B40
:10BDB800494D1A7812F0010F04D12A7812F00302C3
:10BDC80008BF2A701A78434E42F001021A702B7885
:10BDD800414C13F003022ED1404A1278552A03D160
:10BDE800C3F38202013A04E0442A06D1C3F3820273
:10BDF800013262F38403237017E0532A03D15A1CDB
:10BE080062F30103F7E7232A0FD1FCF71BF9337814
:10BE1800334A43F0060333701378013BDBB21370E7
:10BE2800304A52F82320304B1A6001A810211B22F7
:10BE3800FFF776FD4CE0012A4AD101A810211A32F9
:10BE4800FFF76EFD254B1878232804D12378C3F318
:10BE58004112013205E02A2807D12378C3F34112A1
:10BE6800013A62F3461323702CE0532804D1237857
:10BE7800DA1C62F30103F6E7A0F13003DBB2092B09
:10BE880001D943281ED12B7802AAC3F34113D41831
:10BE98000C215A1C03F001034B4302F001021F2638
:10BEA80014F8041C06FB0232FDF7DCFC04F8040C51
:10BEB800287801A900F01C0000F50A40243004226B
:10BEC80003F07BFA29780948C1F34111FFF762FDB5
:10BED8007CBD00BF6D150020F4140020D81400208C
:10BEE8005B1500205C15002010150020B8FB010828
:10BEF800064B1B7803F08003DBB233B1435C044884
:10BF08002021C0180322F4F745BA7047EC2300201B
:10BF1800F20100204328F8B504460D46174606D11D
:10BF2800104B00261A786FF3C3021A7000E00E4611
:10BF38002046FCF77FF890B10A4B303C1A780A2665
:10BF480002F00801C9B2002918BF002506FB054602
:10BF58006FF3C30236B21A70BE42A8BF3E4630B273
:10BF6800F8BD00BF6D1500202DE9F3416E4F6F4EEF
:10BF78003B7843F001033B70347844B94AF28E10A1
:10BF880003F010FA6A4B6B491860204617E0012C41
:10BF980002D10020684912E0022C02D10020674932
:10BFA8000DE0032C02D10020654908E0042C02D1E1
:10BFB8000020644903E0052C03D163490020FBF706
:10BFC8007DFF3178D9B9614B1B78312B01D1013113
:10BFD80001E0302B05D1564B4AF28E10196003F060
:10BFE800D7F95B4B1A785B4B02F08002D2B20AB1E8
:10BFF800202202E04E4A12683032DA776EE00129D8
:10C008000BD002290CD003290DD004290ED04AF2F6
:10C018008A15052918BF00250AE04AF27A1507E0B3
:10C028004AF27E1504E04AF2821501E04AF28615CA
:10C038002946042201A803F0C6F9474B474A03F1F1
:10C04800100153F8040B8B4242F8040BF9D1032278
:10C0580043489DF80410FBF757FF032241489DF819
:10C068000510FBF751FF03223F489DF80610FBF728
:10C078004BFF3E4803229DF80710FBF745FF334B63
:10C088003B4C1878232804D12378022B22D801337B
:10C0980004E02A2804D12378E3B1013B237019E096
:10C0A800A0F13003DBB2092B01D9432812D194F84F
:10C0B800008002AA904418F8041CFF22FFF72AFF08
:10C0C80008F8040C207802AA131813F8041C28187E
:10C0D80003F05EF927482178FFF70AFF1B4B1B780E
:10C0E800532B1FD1224B00221A7033780133DBB255
:10C0F800062B337004D0012B14D10D4B1B688BB168
:10C10800FDF790FB002333703B781B4A43F006038E
:10C118003B701378013BDBB21370184A52F82320A6
:10C12800174B1A60BDE8FC816D1500202C15002006
:10C1380044150020B9920208E29302080394020809
:10C14800249402084594020866940208D814002032
:10C15800EC230020F201002051B202080202002064
:10C1680003020020070200200B0200200F0200201B
:10C1780036150020BCFB01085B1500205C1500206B
:10C188001015002070B5174C0D4692220021064666
:10C198002046F4F7FFF8FF2D0AD1B10001F5D6418A
:10C1A80020463E31042203F00EF923789BB970BD76
:10C1B800FE2D01D1173E02E0FD2D02D10136267079
:10C1C80009E0B60006F5D6403E30401903F0EAF81B
:10C1D800C0B2207020B10348BDE8704011F0DABF4A
:10C1E80070BD00BF1C1700202DE9F04112F002F8C5
:10C1F80060B110208F49FBF761FE8F4B1B78432BF2
:10C2080040F0EE81BDE8F04112F016B812F004F8E3
:10C21800002826D0894C23786BB110208849FBF779
:10C228004DFE88482D211030F4F732F9002800F02F
:10C23800D781217810E010208349FBF73FFE814821
:10C248002D211030F4F724F90446002800F0C881A5
:10C2580011F0FAFF014620468222BDE8F041FBF7C3
:10C2680053BE7A4C43F6CC2223689B68934250D045
:10C27800774E744D307803EB800003F093F8032277
:10C2880001467448FBF740FE2368986846F6A243C7
:10C2980098422BD0203B984228D03378013000EBCD
:10C2A800830003F07FF80322014605F11500FBF730
:10C2B8002BFE236830789B68023303EB800003F081
:10C2C80071F80322014605F11900FBF71DFE2368EA
:10C2D80030789B68033303EB800003F063F8032294
:10C2E800014605F11D00FBF70FFE0EE02D2103228C
:10C2F8005948F4F74FF82D2103225848F4F74AF823
:10C3080057482D210322F4F745F820232B772B7665
:10C318002B75544B1B7813F0010F00F0BD80236878
:10C3280043F6CC229B68444D934261D04E4E484F11
:10C3380032783878D31803EB800003F033F84B4B8E
:10C348000146186028789846A0F13002D2B2092A2E
:10C3580001D943280FD109B2BA22FDF783FA23681D
:10C3680032789B680146C8F800003878D31803EB88
:10C37800800003F00DF82B782A2B04D1337813B101
:10C38800394A013B13702B78232B0ED13378022BBB
:10C398000BD8226846F6824192688A4205D020313D
:10C3A8008A4202D0304A013313702B78552B01D0C2
:10C3B800442B0FD1236831789B68A3F5D643B3F19A
:10C3C8003E0248BFA3F13B023B7803EBA202D0B286
:10C3D800FFF7D8FE264B1B7803F08003DBB23BB196
:10C3E8003278184B03EB820320225A749A74DA7459
:10C3F8002B78532B06D023689A6843F6CC239A42AD
:10C4080040F0EE80FBF71EFE236846F63E329B683E
:10C41800934203D10E4B0220197806E046F6A24259
:10C42800934227D10A4B002019780131BDE8F04129
:10C4380008F04ABDCE800208D814002084100020DD
:10C44800A57F0208F2010020EF80020810150020E5
:10C458002C15002003020020070200200B020020F8
:10C468000F0200206D15002036150020441500200D
:10C47800EC23002046F68242934204D1594B012016
:10C4880019780918D2E746F63E42934240F0A88050
:10C49800544B03201978C8E7236849F2EE429B6899
:10C4A80093423ED14F4E10204F49FBF707FD31789C
:10C4B8004E4D01EB011101F51441EE3110222846D1
:10C4C80002F081FF2B4605F110012A461078474FEC
:10C4D80078B94749FBF7F2FC3846E721F3F7D8FF6C
:10C4E80078B13178401B381801310322FBF70CFD75
:10C4F80007E013F8010B10B9203003F8010C8B4248
:10C50800E4D13C4D2B782A2B03D13078FD21FFF75D
:10C5180039FE2B78432B63D1307823680130C0B2C1
:10C5280059E043F6CC229342324E1AD010203249B9
:10C53800FBF7C4FC33782A2B52D1304B1B689B681D
:10C54800A3F5D643B3F13E0248BFA3F13B02254B06
:10C55800FF211B7803EBA202D0B2BDE8F041FFF740
:10C5680011BE33781F4D552B04D12B78142B01D1D4
:10C57800033B2B703378442B05D12B78122B02D137
:10C58800184B15221A702B78DFF874805901C918D6
:10C59800414401F5725100207931FBF78FFC08F511
:10C5A8006E51102071312F78FBF788FC3378112FEA
:10C5B8008CBF032700272A2B05D12878FE21C01B12
:10C5C800C0B2FFF7DFFD3378432B09D12B78173B37
:10C5D800DF1B2368F8B2997CBDE8F04111F0F2BD89
:10C5E800BDE8F0812C150020AD800208F201002082
:10C5F800A3660208D81400206B80020810150020DA
:10C60800BC44020810B50E4B1B78452B17D10D4BB7
:10C618001A7842F006021A700B4A1378012B0ED8CA
:10C628000A490B4C086844F82300013313708368E7
:10C638000B60FBF73DFBBDE81040FBF703BD10BDE9
:10C64800D81400206D1500205B150020101500205F
:10C658005C15002010B50C4B04462146D8790BF028
:10C6680068F868B1094B1B5D543BDBB2012B09D854
:10C6780020460AF055FFD0F1010038BF002010BD58
:10C68800022010BD022010BD39150020FD24002015
:10C6980008B50BF03DF8C0B208BD00002DE9F04721
:10C6A800634B644C1A78994612F0010F624D65D0BD
:10C6B8002078FFF7CFFF614A2B181178604F93F865
:10C6C800A031604E44293870336090460AD12D2B32
:10C6D80008D038B995F8A11101233B703160207852
:10C6E800FFF7D6FF98F80030552B10D133682D2B63
:10C6F8000DD03B785BB1013B514ADBB21370EB18AC
:10C7080093F8A0114F4B20781960FFF7C1FF98F8F4
:10C718000030232B19D14C4B20781B689B7C013BA4
:10C72800984212DA434B0130C0B21870FFF792FFFB
:10C738003870281890F8A0313360444B9B7803F088
:10C748000203DBB20BB1FBF75DFB98F800302A2B34
:10C7580014D1207890B1374B0138C0B21870FFF768
:10C7680079FF3870281890F8A0313360374B9B78E0
:10C7780003F00203DBB20BB1FBF744FB344EFDF7C9
:10C7880051F8237832789A4288BF337032780F3262
:10C79800934202DD2E4A0F3B1370DFF8C480002756
:10C7A80030783818C0B2FFF755FF281890F8A03134
:10C7B8000137102F08F8013F07D0254B1A78224B74
:10C7C800BA181B689B7C9A42EADB99F8003013F090
:10C7D800010F13D01F4B1A781F4B02F08002D2B200
:10C7E8002AB1227831781032521A5F2105E0227876
:10C7F80031781032521A13490968995413498B78C1
:10C8080003F00203DBB253B120780731652246F604
:10C818003E43FBF791FA05200B21FBF7FFFA21783D
:10C828000E4801310222BDE8F047FBF76DBB00BF9F
:10C838006D1500203615002020FA0108D8140020B4
:10C84800F214002044150020101500207C1500204B
:10C858002E150020EC230020F2010020F301002017
:10C86800010200202DE9F041074610460D46144606
:10C87800F3F7E0FFC3B28046B3B1AB4214D80B4E16
:10C8880020212A46F019F3F785FD2046F3F7D2FF59
:10C89800C8EB05056D08EDB2EF1902462146F019FF
:10C8A800BDE8F041F3F7CEBCBDE8F081F20100200D
:10C8B800F0B5134B1A1894781F4604B30E7800236A
:10C8C8003A1892781A4112F0010F4FF001020DD078
:10C8D800A6420D7803D09A4042EA050504E09A4042
:10C8E800C2F10F0202EA05050D7005E09A400D78C5
:10C8F800C2F10F022A400A700133042BE0D1F0BDC7
:10C9080039150020312200230178194111F0010F57
:10C9180002D00449C9188A7501330132042BD2B2F6
:10C92800F2D17047F2010020034670B50846684A04
:10C9380031B11278532A40F0C980533A1A7070BD49
:10C948001278302A24D163491C780A7822400FD003
:10C958000A78024112F0010F06D0012282401C78A9
:10C96800C2F10F0222401A7001300428F0D10CE005
:10C978000878104110F0010F04D0012090401C7875
:10C98800204318700132042AF2D1534800211AE0DA
:10C99800A2F13100C0B2032825D84E4A12780241CC
:10C9A80012F0010F00F092801C7854FA00F212F095
:10C9B800010F4FF001020BD08240C2F10F0202EAD0
:10C9C800040445481C701322BDE87040F3F7E2BC2C
:10C9D80082404149441C4C741C7822431A7010222E
:10C9E80046F682436EE0132A0BD0552A17D13B4AEC
:10C9F8003B491278122000FB0212527812F0200FE5
:10CA080064D00024344D194620466C74FFF750FF5B
:10CA1800304B9B78002B59D0204629464FE0142AEA
:10CA28000BD02A2A16D12D4A2D491278122000FB44
:10CA38000212527812F0200F48D0274C00221946D3
:10CA480062740120FFF734FF224BDB78002B3DD0C6
:10CA5800012033E0152A0BD0232A16D11F4A20497A
:10CA68001278122000FB0212527812F0200F2DD0FB
:10CA7800194C0022194662740220FFF719FF154B62
:10CA88001B79002B22D0022018E0162A0BD0442A4A
:10CA98001CD1124A12491278122000FB0212527855
:10CAA80012F0200F12D00C4C002219466274032099
:10CAB800FFF7FEFE074B5B7943B1032021461022A6
:10CAC80046F6A243BDE87040FBF736B970BD00BF1B
:10CAD800D814002039150020DA1400202F15002062
:10CAE800AF2400202DE9F04F87B09DF840508046D4
:10CAF800072D0E4605929A4637D1002427463378EB
:10CB0800234113F0010F2CD0012523B24FF0000868
:10CB18000293512029462A462B460095CDF80480D9
:10CB280002F0B4FC1B20414662194346CDF8008050
:10CB3800F5F716FB37B9112039463A462B460097C8
:10CB4800F5F70EFB534B204613F8242001276FF30B
:10CB5800000203F824201199F6F730F92046F6F779
:10CB6800FFFA0134042CCAD1F7E1012D03780CD166
:10CB78000BB90B7823B3FF2300930021464B019197
:10CB88001B780C200133029316E0022D09D10BB952
:10CB98000B78ABB10021FF2300930191029134205F
:10CBA8000AE0062D0CD10BB90B784BB10021FF23FD
:10CBB800009301910291652004220B4602F066FC65
:10CBC800BAF1010F98F800302BD13BB1334B00205C
:10CBD800D979024653460090F5F7C2FA33783BB14B
:10CBE8002E4B0120D979002203460092F5F7B8FAB6
:10CBF8000020F6F7D5F898F80030002B5BD0284BCA
:10CC08001978002957D1274B1B78002B53D0FF23C5
:10CC180000933A2001220B460191029102F036FC62
:10CC280049E063B1052D4FF0000102D100910F20BA
:10CC380001E000910B200A460123F5F791FA3378B9
:10CC480083B1052D4FF0000106D110200A460123BB
:10CC58000091F5F785FA12E00C200A4601230091AD
:10CC6800F5F77EFA022D25D0032D01D10E4B02E0F7
:10CC7800042D02D10D4B1F781DE0052D01D10C4B61
:10CC8800F9E7012D01D1044BF5E7062D0CBFFF276D
:10CC9800002710E0B41200201313002039150020DB
:10CCA800AC1200201F0E0020D01600203F2B0020C1
:10CCB800E8250020FF2798F80030002B00F09D8021
:10CCC800914C237803F02003DBB26BB18F4B1978BA
:10CCD80011F0010108D1FF230093282001220B46FF
:10CCE8000191029102F0D2FB237803F01003DBB22A
:10CCF80073B1864B197801F00201C9B241B9FF231B
:10CD08000093292001220B460191029102F0BEFBFB
:10CD1800E37813F0010F0ED07C4B197801F0040171
:10CD2800C9B241B9FF2300932A2001220B46019181
:10CD3800029102F0ABFBE37803F00203DBB273B1BC
:10CD4800724B197801F00801C9B241B9FF23009369
:10CD58002B2001220B460191029102F097FBE37808
:10CD680003F00403DBB273B1684B197801F01001CA
:10CD7800C9B241B9FF2300932C2001220B4601912F
:10CD8800029102F083FBE37803F00803DBB273B18E
:10CD98005E4B197801F02001C9B241B9FF23009315
:10CDA8002D2001220B460191029102F06FFB0CF03D
:10CDB8005FFD70B1554B197801F04001C9B241B916
:10CDC800FF230093492001220B460191029102F0B2
:10CDD8005DFBE37803F04003DBB273B14B4B19788A
:10CDE80001F08001C9B241B9FF2300934E2001220E
:10CDF8000B460191029102F049FB119B444A1978B4
:10CE0800444B51B198F80010117032781A70337889
:10CE18000BB1542005E0522003E011703278532002
:10CE28001A7002F0ADFE119B00241A783A4B1A7062
:10CE380098F80030234113F0010F2DD021460598B2
:10CE480010F030FC0122014628B923B2019000926B
:10CE58000293104605E0002123B20092019102934B
:10CE680024200B4602F012FBBAF1010F05D12B4B1F
:10CE78008020DA790521013208E0022D07F101024C
:10CE880002D18020072101E0802006212346F6F701
:10CE980081FC2046F6F738F93378234113F0010F67
:10CEA80057D000214FF0010B23B2029302205A46BB
:10CEB8000B46CDF800B0019102F0E8FADA45DFF848
:10CEC80068900CD119F8243013EA0B0334D1134AB3
:10CED8000520D1790093594404EB0B022AE019F894
:10CEE800243013F0010327D1022D1FD10C4B1B78DE
:10CEF80003F02403042B04BF0A4B83F800B000237B
:10CF08000093072014E000BFEC230020CF1300207B
:10CF1800D8120020D9120020DD1300203915002076
:10CF2800E2130020180E0020B412002000930620FF
:10CF3800791C621CF5F714F911992046F5F73EFFA4
:10CF48002046F6F70DF919F824306FF3000309F8B5
:10CF580024300134042C7FF46BAF07B0BDE8F08FA8
:10CF68002DE9F74F16469A46337804460F469DF842
:10CF780030909DF834B09DF83820DFF87C8043B1BC
:10CF880002EA03033370097898F800208A18D31A44
:10CF98000370164B00251D70217843F6ED2002F032
:10CFA800F7F9494646F2A75002F0F2F9104B31461C
:10CFB8005D7052464B463846CDF800B00194FFF7F5
:10CFC80091FD2046F8F700FD23780A480A4988F8B9
:10CFD8000030F6F771F88AF8005035703D7025700A
:10CFE80003B0BDE8F04F02F0DBBC00BF6C150020B9
:10CFF8001F0E0020D0130020AC1200202DE9F041B4
:10D0080080460E46174646F2686500243846214693
:10D0180010F048FB88B1294603220B4802F0D3F9E7
:10D028000948414610F0DCFA074810F00AFB20B91D
:10D038000123A34032781343337001340835042C9C
:10D04800E4D1BDE8F08100BFDA1300202DE9F043F8
:10D0580087B08046894604A847F25201082202F0A8
:10D06800B2F900244046214610F01CFB38B30126D3
:10D078000223A719002100933BB200250293232025
:10D088000B460422019602F001FA394632462B4635
:10D0980011200095F5F764F8042021462A46334606
:10D0A8000095F5F75DF8B9F1000F08D004A82146FE
:10D0B80010F0F8FA18B10548214610F0DDFA0134ED
:10D0C800182CCFD107B0BDE8F08300BFC9120020EB
:10D0D80010B50B4B0B4C33F8962F01469B780A483A
:10D0E8002280A37010F0A8FA2146074810F078FAB9
:10D0F800054810F0A6FAD0F1010038BF002010BD95
:10D108002C1B0020D5130020DA1300202DE9F04F46
:10D11800744B754FF0221A703B788BB00B2B7ED175
:10D12800DFF8108298F80260012E06D96F490020B6
:10D138000BB0BDE8F04FFAF7C1BE6D4D19D16D4B7C
:10D148006D4A6E496E4800241C7014700C7004708F
:10D1580088F8024000966B4E019436780296FFF7E5
:10D16800FFFEFAF76FFF2C600BB0BDE8F04FFAF73F
:10D178003DBE62496448F5F79FFF644B644E1A88C8
:10D188009B783280634AB370634B127819782B68A6
:10D19800532A9B7C09D05A1E48BF9A1DD6100136C7
:10D1A8004E4306F5CA46A8363AE05C49564810F0A0
:10D1B80017FA5548FFF78CFF044618B1052388F87D
:10D1C8000230BCE1032246F2A8514F4802F0FBF8B6
:10D1D8004D49534810F030FA032246F60A213046EA
:10D1E80002F0F1F83146484810F01BFA4648012190
:10D1F800FFF72CFF44483F49404AFFF7FFFE012351
:10D208000093404B01941B783D4802933B493A4AAE
:10D21800384BFFF7A5FEFAF715FF2C608FE10026C3
:10D22800404B334D1A78404C12F0010F00F0A280A9
:10D23800384B1A789846432A21D13B780B2B1ED1BC
:10D248003148217810F02EFAC8B13148217810F011
:10D2580029FAA0B920780FFA86F909EBD00002F074
:10D26800A1F82378012103F0070291402F4A80EAB0
:10D278000101116009EBD300C9B202F089F898F8EE
:10D288000030232B10D12A682378927C013A9342EC
:10D298000ADA254A01331370254B9B7803F0020301
:10D2A800DBB20BB1FAF7AEFD98F800302A2B0CD19F
:10D2B800237853B11C4A013B13701D4B9B7803F034
:10D2C8000203DBB20BB1FAF79DFD98F80030552B3D
:10D2D8003CD129682278897C134B08398A422BDA99
:10D2E80008322AE0791500206C15002069670208C9
:10D2F80010150020D91400206E1500207A15002082
:10D308001415002039150020DE130020C21B002050
:10D31800A8120020D81400202C150020CF120020BD
:10D32800D51200206D150020361500204415002068
:10D338007C1500201F0E002000221A70814B9B785C
:10D3480003F00203DBB20BB1FAF75CFD98F800308A
:10D35800442B0FD122787C4B072A9CBF2A68927CE9
:10D36800083A1A70774B9B7803F00203DBB20BB1D3
:10D37800FAF748FDFCF756FA744A23781178904674
:10D38800994288BF137012780F32934202DD6F4AB8
:10D398000F3B13702B684FF0000B93F81290CDF8E9
:10D3A8001CB0B9F10F0F9ABFC9F120095FFA89F9CA
:10D3B8004FF01009334638784FFA8BF20B2805D115
:10D3C80098F800105218D210614904E098F800103B
:10D3D80052186049D2108E5C98F800104FFA8BF200
:10D3E80051180B2801F0070A13D118B200EBE1001D
:10D3F8000692059301F0D6FF5449069A0978C0B2FF
:10D40800079051185448C910415C059B06EA010170
:10D418000991387898F80010089052183CE0DDF827
:10D428001CC04CFA0AF111F0010F4C490CD10898B4
:10D438000B280BD14A484FEAE20C10F80C0040FACE
:10D448000AF010F0010F01D12A2013E0DDF824C002
:10D458004CFA0AF010F0010F04D008980B2801D1FB
:10D468004D3007E046FA0AF000F0010000280CBF32
:10D47800A520DB200AF1010A5FFA8AFA01F80900FF
:10D488000BF1010B09F101090132BAF1080F5FFA3A
:10D498008BFB5FFA89F903D0B9F1200FBFD10CE0FB
:10D4A800B9F1200F09D098F800204FFA8BF18918AC
:10D4B8002A68927C9142FFF67EAF2A490B7813F0D6
:10D4C800010F17D02B68284A9B7C12780F2B02F08B
:10D4D800800298BFC3F11003D2B294BFDBB200231D
:10D4E80042B1227898F800101032521A1B49CB1812
:10D4F8005F21995413498B7803F00203DBB28BB197
:10D508000731652246F63E332078FAF715FC2B687A
:10D518009B7C102B02D905200B2101E0002007215C
:10D52800FAF77CFC2B689B7C102B08D921780F48D4
:10D53800013102220BB0BDE8F04FFAF7E5BC0BB0A1
:10D54800BDE8F08F7C150020361500202E15002030
:10D55800CF120020F8120020A8120020F2010020AB
:10D56800DE1300206D150020EC230020F3010020BD
:10D5780010B50A4CA37C4BB100200949FAF79EFC70
:10D58800084B1B78432B01D1433BA374A07C20B9E3
:10D598000549BDE81040FAF791BC10BDDA14002027
:10D5A800E5660208D8140020C4660208034B1A78FE
:10D5B80001321A7001230370704700BF6C150020F8
:10D5C8000A4A10B500241470094A0A4B14700A4A12
:10D5D8009C701470094A5C701470094A1470094AE6
:10D5E8001470FAF72FFD084B1C6010BD3915002088
:10D5F800D91400201F0E00206E1500207A15002077
:10D60800141500206C150020101500202DE9F0419C
:10D61800002386B08DF81730884B1B78012B00F05B
:10D62800EA81874C874D237843B12B78002B40F053
:10D63800A680FAF707FD08232B70A0E02A78072AAE
:10D6480000F29D80804A1278232A13D12B70FAF7B2
:10D65800F9FC7E497E4A0B7853B17E48013B047839
:10D66800DBB244F0060404700B707B4951F8233098
:10D6780013605FE2774B1A7812F0010F04D1012191
:10D688000A438DF817101A70F5F7D2F928B92B78D4
:10D698001BB90DF11700FFF789FFF5F7D7F930B976
:10D6A8002B78012B03D10DF11700FFF77FFFF5F75A
:10D6B800DBF930B92B78022B03D10DF11700FFF7F6
:10D6C80075FFF5F7DDF930B92B78032B03D10DF190
:10D6D8001700FFF76BFFF5F7E1F948B9F5F7FAF925
:10D6E80030B92B78042B03D10DF11700FFF75EFF3B
:10D6F800F5F72EFA30B92B78052B03D10DF1170069
:10D70800FFF754FFF5F718FA30B92B78062B03D139
:10D718000DF11700FFF74AFFF5F7CEF930B92B786E
:10D72800072B03D10DF11700FFF740FF9DF81730C5
:10D738002BB32B78072B1FD8DFE803F004070C0F57
:10D748001215181B0020454901E045490020FAF749
:10D75800B5FB14E000204349F9E700204249F6E709
:10D7680000204249F3E700204149F0E70020414901
:10D77800EDE700204049EAE7FAF764FCDAE12B78A4
:10D78800304F082B40F0A280324B2F4F1978984623
:10D7980011F00101394E23D113223046F2F7FAFD78
:10D7A8000123B374364A2378137003B9B374B37C76
:10D7B80013B1344B00221A70FFF7DAFE3048B17CFF
:10D7C800FFF7B2F898F8003003F0FD0343F00103C7
:10D7D80088F800302C4B1A7812B13A7000221A706F
:10D7E8003B78002B5ED0FFF7C3FE2548B17CFFF7DE
:10D7F8009BF8234B1A78984622B1002010211F4A23
:10D80800FFF730F82378387898F800401F4924EA61
:10D81800030252380A70C0B21D4A23EA04030128E1
:10D8280013703FD8002C37D1002B35D0012300933B
:10D83800184B01941B78124802931FE179150020B8
:10D84800AC1200206C150020D81400205B150020B5
:10D85800101500206D1500205C150020266B0208AD
:10D86800056B0208476B0208686B0208896B02089F
:10D87800AA6B0208CB6B0208EC6B0208DA140020D2
:10D8880014150020180E0020301500207A150020ED
:10D898006E15002039150020814B04229A702B78D0
:10D8A80001332B707F48FFF72DF8737C002B00F0B5
:10D8B80041817D4A127802F08002D2B2002A00F03B
:10D8C80039817A4AD31820225A7533E1092B31D18C
:10D8D800774806F0A3FBC6B2714C2EB3A378042B8D
:10D8E80002D10020734903E0022B04D172490020C1
:10D8F800FAF7E4FA02E00BB90433A37031460222C6
:10D908006A48FAF701FB6D4B1E78232E73D0304618
:10D91800FAF790FB002800F00D81312E40F00A81C3
:10D928002B7801332B7002E03B7801333B700823DE
:10D93800A370FFE00A2B40F0FD805D48002106F04F
:10D9480043FBC4B2002C4CD0554F7B783E466BB994
:10D958005B4BD879F7F79CFF10B90323FB704AE0BB
:10D96800BE2010F089FC7B7801337B70B3784C4A79
:10D97800092B02D90020534915E010D1504B00243F
:10D988001C709470504B514A4949464801251C70F7
:10D9980014700C7004700095019402946FE0082BC9
:10D9A80004D14B490020FAF789FA11E0062B02D17D
:10D9B80000204849F7E7042B02D100204649F2E746
:10D9C800022B02D100204549EDE70BB908339370CB
:10D9D800B378082B0BD8354821460222FAF794FA77
:10D9E80005E001230093364B01941B7842E0334F46
:10D9F8003C78232C02D1FFF7E3FD9BE02046FAF7A1
:10DA080019FB002800F09680303CE4B2631EDBB2BC
:10DA1800012B3C703AD8022C294D26D1E879F7F72A
:10DA280037FF002839D02E48FFF752FB002834D1A1
:10DA3800032246F2A8512B4801F0C5FC2849294881
:10DA48000FF0D9FD0322274946F2A85001F0B5FC92
:10DA5800244925480FF0F0FD21480121FFF7F6FA87
:10DA68001F481949124AFFF7C9FA012300240093F5
:10DA780001942B780B480E49144A0293124BFFF776
:10DA88006FFAFAF7DFFA194B1C6053E0032C51D1F7
:10DA98000B4BD879F7F7FCFE50BB0C23B37049E069
:10DAA8001F0E002014150020EC230020F201002096
:10DAB8007A150020AB670208CC670208D81400204A
:10DAC8003915002069670208D91400206E15002056
:10DAD8000667020827670208486702088A6702087B
:10DAE800DE130020A8120020D512002010150020F7
:10DAF8000024124821460FF0D5FD28B1E02010F08F
:10DB0800BBFB204610F0F2FB0134182CF1D10322A4
:10DB180046F60A200A4901F050FC0023B3702B781E
:10DB2800084A01332B70084B1A60084B1A7842F0E8
:10DB380006021A7006B0BDE8F08100BFDE130020AF
:10DB4800D5120020C4FB0108101500206D15002017
:10DB58001FB5044611B100200B4901E008460B49E6
:10DB6800FAF7ACF9217810220139C9B201EB011199
:10DB780001F5C0412231684601F025FC102001461C
:10DB88006A46FEF76FFE1FBDCC4602080E47020824
:10DB98000B4B1B78442B06D0552B037801D013B1BF
:10DBA8007047013B01E003780133037003780BB938
:10DBB800203302E0212B01D1203B0370FFF7C8BFBF
:10DBC800D81400202DE9F74FDFF8C881DFF8D4A179
:10DBD80098F80030554643F0010388F800309AF869
:10DBE8000130624C23F07F039B46D3B1002060498B
:10DBF800FAF764F95F482A21F2F74AFC18B121784C
:10DC08008222FAF781F92278002A40F0AB802B684B
:10DC180062F3CF332B60584B1A7842F003021A7024
:10DC2800A0E0DFF85491237099F800304E4603F0D5
:10DC38000202D2B20192514F002A40D013F00108DB
:10DC480013D058464E49FAF739F93B78232B20D19F
:10DC58004C4B4D4A4D481A600121FFF779FF337844
:10DC680003F0FE036BF3410312E040464849FAF71C
:10DC780025F93B78232B0CD1424B434A43481A6081
:10DC88000121FFF765FF337868F3000368F3410368
:10DC980033703B782A2B65D1337803F0FE036FF39A
:10DCA800410333702B6843F400432B600F23237028
:10DCB800364B187803B0BDE8F04F0BF099B80AF06E
:10DCC800DBFF054600282DD001213048FFF760FF13
:10DCD8003B78532B12D13378019A03F0FD0362F39A
:10DCE80000033370DAF8003043F40043CAF8003018
:10DCF8000F232370254B18780BF07AF83B78232BE9
:10DD080030D13378002203F0FD036FF30003337042
:10DD18001E4B1A70FAF796F91E4A137843F0060359
:10DD2800137015E01C49FAF7C9F83B78232B19D171
:10DD380099F8003065F3410365F3000389F8003072
:10DD4800FAF780F998F8003043F0060388F80030B5
:10DD5800124A1378013BDBB21370114A52F82320A0
:10DD6800084B1A6003B0BDE8F08F00BF4A2C0020B2
:10DD780050470208F201002070250020D814002026
:10DD88007147020810150020E0FB01083615002035
:10DD9800924702086D150020B34702085B15002062
:10DDA8005C150020EC2300202DE9FF412C4D2D4C63
:10DDB8002B7843F001032B70217801F00401C9B2DC
:10DDC80011B92948FFF7E4FE284E3378232B21D1D7
:10DDD8002378274F13F004080AD0224A6FF38203EE
:10DDE8001370244B20483B600021FFF7B1FE11E07F
:10DDF800FAF728F92B78204A43F006032B7013789A
:10DE0800013BDBB213701D4A52F823303B60164BBE
:10DE180083F800803378532B1FD12378052243F0F1
:10DE280004032370104B16491C78013CE4B204EB40
:10DE3800840000F5C840623001F0BFFA00201149A3
:10DE4800FAF73CF8FF23002100930134162004223E
:10DE58000B460191029401F019FBBDE8FF8100BF58
:10DE68006D1500207025002036150020D8140020DC
:10DE780010150020FCFB01085B1500205C15002034
:10DE880018FC01082F4702082DE9F041984B044679
:10DE98009A7812F0010F00F017811B88002B40F0D0
:10DEA8001381944D95F82030172B40F2D780012C20
:10DEB80014D1914B1B7803F00203DBB2002B00F066
:10DEC800C48095F820208B4B182A03D1013283F89F
:10DED8002020FBE0202283F82020B6E0022C03D18A
:10DEE800202385F82030B0E0844E337803F02002F8
:10DEF800D2B28AB195F82020182A0DD1032C0BD064
:10DF08007F4B804A03F1100153F8040B8B4242F80F
:10DF1800040BF9D1192395E003F01003DBB28BB1A0
:10DF280095F82030192B0DD1032C0BD0764B754A60
:10DF380003F1100153F8040B8B4242F8040BF9D19A
:10DF48001A237FE0F37813F0010F0FD095F8202003
:10DF58001A2A0BD16D4B6B4A03F1100153F8040BCD
:10DF68008B4242F8040BF9D11B236BE003F0020249
:10DF7800D2B27AB195F820201B2A0BD1644B614AA2
:10DF880003F1100153F8040B8B4242F8040BF9D14A
:10DF98001C2357E003F00402D2B27AB195F820208E
:10DFA8001C2A0BD15B4B574A03F1100153F8040BA1
:10DFB8008B4242F8040BF9D11D2343E003F0080318
:10DFC800DBB28BB195F820301D2B0DD1032C0BD073
:10DFD800514B4C4A03F1100153F8040B8B4242F8A1
:10DFE800040BF9D11E232DE00BF042FCA0B14B4BE2
:10DFF8001B788BB195F820301E2B0DD1032C0BD03C
:10E00800474B404A03F1100153F8040B8B4242F886
:10E01800040BF9D11F2315E0F37803F04003DBB2BA
:10E028009BB195F820301F2B0FD1032C0DD03D4B01
:10E03800344A03F1100153F8040B8B4242F8040BE5
:10E04800F9D1202385F8203078E095F82030013385
:10E05800DBB21F2B85F820307FF629AF95F82060BA
:10E068001F2E04D9234B002683F8206001E00136D7
:10E07800F6B206F11807FFB212E02B4831460FF04E
:10E0880011FB08B1032C04D1284B9B5D23B1032C51
:10E0980002D185F820600FE00136F6B2BE4203D007
:10E0A800172EEAD9182E07D1214B1E221A701823D1
:10E0B80085F82030BDE8F08195F8200011496522E7
:10E0C80046F63E33F9F738FE012C37D1194B0D4A85
:10E0D80003F1100153F8040B8B4242F8040BF9D1F9
:10E0E800044B93F82030172B3CD9002012493EE00E
:10E0F8007C150020F2010020AD120020EC23002046
:10E10800044E020883150020254E0208464E0208D8
:10E11800674E0208884E0208A94E020849270020C7
:10E12800CA4E02080C4F0208F8120020DB12002029
:10E1380037150020F09D0208C24D0208104BD87810
:10E1480000F02000C0B220B1022C06D000200D49FA
:10E158000DE0032C01D10C4909E00C4B93F8203059
:10E16800172B02D800200A4901E00A490020F9F7D4
:10E17800A5FE10200146BDE8F041F9F74FBE00BFEB
:10E18800EC230020DD440208E34D0208F2010020E0
:10E19800804D0208EB4E020810B5F9F753FF084B03
:10E1A8001B7803F00403DBB22BB106490020BDE85D
:10E1B8001040F9F783BE0220BDE81040FFF764BEA7
:10E1C800AD120020B24B020870B5214B06461B78F1
:10E1D800204CF3B9257819E01F4829460FF062FA58
:10E1E80078B123689D4202D9FF2E02D007E0FF2EA6
:10E1F80002D19D4208D202E036B91DB913B9256093
:10E2080012E00EB9013500E0AD19EDB2172DE3D9D2
:10E218000AE0013B2021114810222360F2F7BAF8E6
:10E2280000200F49F9F74AFEF9F7E0FD46F63E33BC
:10E2380020780C496522F9F77FFD084D216805F122
:10E24800100001310222F9F75FFE2D23AB7470BD77
:10E258002C1500204415002016150020F20100207E
:10E268005A82020883150020F8B5534BF022534810
:10E278001A700378044613F00E0518D1504A43F07B
:10E288000203156000F8013B0FF0A2F92C464D4B34
:10E29800E35C1BB14C4821460FF0EEF90134182C11
:10E2A800F5D14A4B1A7842F001021A70F8BD13F002
:10E2B8000C0543D12E46444829460FF0F3F908B11E
:10E2C8000136F6B20135182DF5D11EB9237843F081
:10E2D800040331E000253E482946EFB20FF0E2F989
:10E2E80068B1384BEB5C53B13A4B01371F700020D3
:10E2F800FFF76AFF237843F00803237002E0013533
:10E30800182DE8D1344D3A212846F2F7C1F838B132
:10E31800401BC0B20130281831460222F9F7F4FD3B
:10E328002E4B1B78532B46D12A4B00201870FFF731
:10E338004BFF237843F008032370F8BD6FF34103C4
:10E34800037003F00403DBB2244D23B100202449F9
:10E35800F9F7B4FD0DE02B78552B01D1FF2002E031
:10E36800442B02D10120FFF72FFF13200D21F9F7CD
:10E3780055FD2B78232B1ED1227802F00204D4B944
:10E388000E4902F0FB0264F3C3020A700C4A1460DF
:10E39800F9F758FE0D4B1A7842F006021A70114A26
:10E3A8001378013BDBB213700F4A52F823200F4B4E
:10E3B8001A60084B1C70F8BD79150020151500204F
:10E3C800441500202C1B0020161500206D15002078
:10E3D800AE1200202C150020F2010020D8140020D5
:10E3E800DB8E02085B1500205C150020101500204C
:10E3F800024800210922F1F7CDBF00BF49150020CE
:10E4080070B50A46002405E01B19811A2A25013433
:10E418005D54E4B20E4D0F4B295D09B19442F3D11E
:10E42800801A001918182021121BF1F7B3FF0A4BA4
:10E438001E785EB1432E04D10CB1013CE4B2002336
:10E448002B553046F9F7F6FD00B12E5570BD00BFCB
:10E4580049150020F2010020D814002038B5184CC6
:10E46800184DA07800F01000C0B250B91649F9F75D
:10E4780025FDFFF7BDFF236843F4801323600F23B6
:10E488002B702A782AB92368FF2062F3145323607B
:10E4980038BD0E48C5792DB91C200821FFF7B0FFFB
:10E4A800284638BD23680A496FF3145308222360AD
:10E4B800F2F7F0F900280CBF0120FF2038BD00BF9B
:10E4C800EC2300207B150020154C0208491500207C
:10E4D80041B10208F0B5634D85B06E7806F01006BC
:10E4E800F6B2002E3ED1604B1A78604B013A53F8D1
:10E4F80022305F4A934204D15E4B1A7842F00202FE
:10E5080007E002F11C018B4208D15A4B1A7842F0FD
:10E518000402022161F3C7021A7019E038329342EB
:10E5280016D1FFF79BFF002800F09A800128514C74
:10E5380006D12378022243F0010362F3C70306E001
:10E5480030464D49F9F7BAFC237866F3C7032370C0
:10E558004A4B1A7842F001021A702B6843F4805330
:10E568002B607DE0434E337813F0F80406D044491D
:10E57800002005B0BDE8F040F9F7A0BC13F0070F84
:10E588004FD003F00202D7B287B1214612200CF017
:10E5980095FAFF2300934320214604222346019441
:10E5A800029400F073FF0094162031E003F0040495
:10E5B800E4B2A4B1394638460CF080FA0BF0F4FC0A
:10E5C80007F01EFD0AF080FBFF2300934420394624
:10E5D80004223B460197029700F058FF1DE013F014
:10E5E800010F1AD0012143F6FA400CF067FA2046D1
:10E5F800F7F7B2F9234B45201C80FF2300932146EF
:10E60800042223460194029400F040FF0094152050
:10E61800214601222346F3F7A3FD00201A49F9F702
:10E628004DFC337803F0FA036FF341033370174B53
:10E638001B78232B14D12B686FF30C332B60F9F75D
:10E6480001FD0E4B1A7842F006021A70064A13783A
:10E65800013BDBB21370054A52F823200C4B1A60B9
:10E6680005B0F0BDEC2300205B1500205C150020F0
:10E678001CFC0108CE290020364C02086D1500202C
:10E6880056920208F014002035920208D81400208F
:10E69800101500201FB50446F7F71CFAA8B14B2047
:10E6A80001F06EFAFF2300930121FF3B019339200B
:10E6B80004220B460134029400F0E8FE064B0120C8
:10E6C8005A7842F004025A7004E0044B1888003863
:10E6D80018BF012004B010BD60250020602C002068
:10E6E800F0B51E4E0024337A0546013385B00F4637
:10E6F800337210202146012223460094F3F730FD9F
:10E7080045B9FF230093019502974F20294604221B
:10E718002B4609E0012D09D1FF23009301940297AC
:10E72800502021460422234600F0B0FE337A052B00
:10E7380011D1FA3301210024009327200B4604222B
:10E748000194029400F0A2FE044B1C7205B0BDE8CF
:10E75800F04001F0E7B905B0F0BD00BF3915002061
:10E768002DE9F04F9D4B87B01A78804699461AB12B
:10E77800012A40F0DB812AE0994B1A68994B9A42AA
:10E7880000F0D681F6F762FE974B5B7803F0200322
:10E79800DBB223B901F0ECF908B907F031FC934B6F
:10E7A8001A686FF310421A60914B1878F9F742FC17
:10E7B800002800F0BD81FFF71BFE8E4B3C221A702B
:10E7C800F9F776FA99F80030013389F80030894B67
:10E7D8001C787CB9884B08F101011A78204664F34B
:10E7E800C30264F304121A70C9B2FFF779FF89F8FB
:10E7F80000409DE1814D404607F022FCF9F702FBFD
:10E8080000207F49F9F75AFB7E4F2B78AA46FB1860
:10E8180013F8313C23B91B200621FFF7F1FD87E1EE
:10E82800754A0B21137804A8C3F3C004C3F3001678
:10E8380003F0F7036FF304131370002389F8003013
:10E84800062200F0C0FD2A78394604A8303AF1F7CC
:10E85800C7FC074620B100274FF012093D4629E0C2
:10E8680049F2DB4000F09EFD0028F4D0664D2F727F
:10E87800F6F744FF0446002840F05A81634A584B93
:10E8880021461A60FF230093019002900422082079
:10E89800234600F0FBFD012223460E20214600946A
:10E8A800F3F75EFC5A4B1A7842F004021A700123FF
:10E8B800AB713DE14946062204A800F084FD9AF8B0
:10E8C800002004A84F49303AF1F78AFC002840F0AC
:10E8D8001E812846FFF7DEFE002840F02981DFF878
:10E8E80028B101218BF808002846F6F715FF814664
:10E8F800F6F704FFDA46002840F0B280484645495A
:10E90800F1F74CFEB0B901F04BF8354B14B916B914
:10E91800414A23E036B1414A1A60414B1A786FF3F5
:10E92800410205E03F4A1A603D4B1A7866F34102FE
:10E938001A70D4E048463C49F1F730FE20B1484609
:10E948003A49F1F72BFE58B9002C40F0F180002E1F
:10E9580040F0EE8001F024F8354A214B1A60BEE001
:10E9680048463449F1F71AFE50B949F2D940012115
:10E9780000F00EFD1D4A136843F400531360E3E7EB
:10E9880048462D49F1F70AFE38B9002C40F0D080EE
:10E99800002E40F0CD80294ADFE748462849F1F7A4
:10E9A800FDFD38B9002C40F0C380002E40F0C08037
:10E9B800244AD2E748462449F1F7F0FD002840F000
:10E9C8008E8000F0EDFF002C40D0164A044B1A60F0
:10E9D800134B1A786FF34102A9E000BF0F1500200E
:10E9E8001015002070FC01086E250020EC23002083
:10E9F800D81400207B15002048150020F7140020AB
:10EA0800BC44020849150020391500208CFC010877
:10EA1800391900206BB20208BCFE01084400020844
:10EA28006D150020600002083DB2020828B40208F3
:10EA38007C00020861B2020863B20208B40002084E
:10EA4800FAB302080801020865B20208002E6FD066
:10EA5800394A3A4B1A603A4B1A7864F3410266E035
:10EA680048463849F1F79AFD064620B900F098FF64
:10EA7800002C5DD01BE048463349F1F78FFD002894
:10EA880056D048463149F1F789FD38B9002C4FD1A5
:10EA98002F4A2A4B8BF807501A6049E048462D49FF
:10EAA800F1F77CFD064650B9A4B100F079FF2A4A77
:10EAB800224B1A60224B1A7866F3410237E0484627
:10EAC8002649F1F76BFD20B148462549F1F766FD67
:10EAD80000B96CBB234A194B1A6000F061FF07F5B7
:10EAE8006A506E308AF8075000F05CFC8AF8000023
:10EAF8009AF8070000F5D440123000F053FC8AF869
:10EB080001001948F6F740FF202D11D107E0013523
:10EB1800EDB20137202D09F107097FF4CBAE08F1DA
:10EB280001010020C9B2FFF7DBFD01E000221A70E5
:10EB380007B0BDE8F08F00BF4400020810150020A0
:10EB48006D15002065B2020863B20208FAB3020824
:10EB5800080102086BB20208600002083DB2020810
:10EB680061B20208240102083915002038B51C4991
:10EB78001C4A0B6810789C7B8442144603D99D89F3
:10EB880015F0200F18D09A8912F0800F01D105E0F6
:10EB98001C3B9A8912F0400FFAD000E01C330B603E
:10EBA800002323700B689B8913F0200F06D00E4BAF
:10EBB800DA790C4B1A7001E0013010700B4A00230F
:10EBC80013700B4A13700B4A136843F48073136075
:10EBD800F9F76EF8084B1A7842F006021A7038BD39
:10EBE800101500202C15002039150020F3140020E2
:10EBF800ED140020EC2300206D15002010B51D4BEE
:10EC08001D4A1978184639B11468A48914F0200FE0
:10EC180002D1013919701AE01368998911F0400F6F
:10EC280001D106E01C33998911F0800FFAD01360E6
:10EC380002E011491C3B0B6013689A7B02709B89A8
:10EC480013F0200F03D00D4BDA790A4B1A700C4AD7
:10EC5800002313700B4A13700B4A136843F4807334
:10EC68001360F9F725F8094B1A7842F006021A7072
:10EC780010BD00BF2C1500201015002039150020EC
:10EC8800F3140020ED140020EC2300206D15002063
:10EC9800084B094A1B68934203D002F57C729342E1
:10ECA80005D1064B1878003818BF0120704700209E
:10ECB800704700BF1015002070FC0108AC1200203E
:10ECC800074B084A1B68934202D03832934205D159
:10ECD800054B1878003818BF01207047002070478E
:10ECE8001015002008010208AC1200202DE9F04F91
:10ECF8008B4B8C4D1970A0F11103DBB2012B87B03F
:10ED08000E46287020D8122804D1874B1A8842F45E
:10ED180080521A80854B00245A78214642F010020E
:10ED28005A70FF23022200933D20FE3B0194029477
:10ED380000F0ACFB4D2000F023FF1220202101221F
:10ED480023460094F3F70CFA2B78522B0DD1F3F7E6
:10ED58004BFF28B9F3F73CFF10B9F3F75DFF20B17B
:10ED6800734B1A7842F008021A70724B724C1B7877
:10ED7800002B2DD12168714A914229D0704A236015
:10ED88001370704A70481178037063F3C30163F31A
:10ED9800000163F3071111706C4A117863F30101E4
:10EDA80011706B4A117863F3C5011170694A1370C9
:10EDB800694A117863F3410163F3000163F3820147
:10EDC8001170664A116863F30C311160644A13705C
:10EDD8002368002B40F05781604F7B7803F02003B5
:10EDE800DBB273B15F4B93F80080B8F1000F08D124
:10EDF80049F2D940414600F0CBFA3B6868F34D33FD
:10EE08003B60594B187810F01E0002D0002057497B
:10EE180007E0574B93F803809946B8F1000F05D0E7
:10EE2800544907B0BDE8F04FF9F748B8524F97F882
:10EE380001B0BA46BBF1000F2BD0BBF1070F14D9B4
:10EE4800F8F7D4FF4D49B878652246F63E43F8F7FF
:10EE580073FF3878072310F003007B700EBF484912
:10EE680040464849F9F72AF80CE0BBF1020F09D8E7
:10EE7800454B5B7823B1F8F7B9FF87F8018069E261
:10EE880002237B701020014607B0BDE8F04FF8F769
:10EE9800C5BF3E4FBB795BB187F806B000F0DAFB1F
:10EEA8008E20594601225B46CDF800B0F3F758F999
:10EEB8000020F3F775FF234A21491378344843F0BB
:10EEC8000603137000230B70324923600B7032491C
:10EED80089F800300370123303FB061C9CF802C04B
:10EEE80093461CF0100F884604D130460593FFF76F
:10EEF80037FC059B03FB06835B7813F0100F04D0E7
:10EF08002A78133AD2B2032A4AD913F0200F7DD0B7
:10EF18002B78442B44D041D8232B41D02A2B3EE0D8
:10EF28002F150020D8140020E213002060250020AF
:10EF3800D21200207915002010150020C4FB01080A
:10EF48005B1500206D15002036150020F4140020F4
:10EF5800311500203815002048150020EC2300202A
:10EF680078150020AC120020492C00201F4502080B
:10EF78001F0E00200D6C0208331500208315002099
:10EF880027460208064602087C150020391500208D
:10EF9800301500202C150020AF240020552B35D12A
:10EFA8007A4B1B78002B31D1794B93F80080B8F15C
:10EFB800000F2BD143F6DB2000F0F4F9012825D10E
:10EFC8001F23FB7189F8000043F60D3000F0EAF9C1
:10EFD8003870F87900F5D440123000F0E3F9787011
:10EFE8006C48F6F7D1FC9BF80030304668F34103D3
:10EFF8008BF8003007F024F8F9F724F8664B6748D7
:10F008002360674BC3F800802B7803702B78432B61
:10F018000AD15F4B1B783BB9013389F80030614B4B
:10F028003046236007F00CF828781738C3B2072B4E
:10F0380000F290815C4908F0C3FB9AF800105B4B22
:10F0480060F301018AF8001001F00301022900F0C1
:10F0580081810122032041B1009001929B786830A0
:10F068009B1802930021033206E0009001929B78DE
:10F078006C200133029304220B4600F007FAFF23A9
:10F088008AF8013066E1474A934253D12878A0F1C3
:10F098004303DAB2122A25D8454A5BB29A4021D5F1
:10F0A800432840F05781394B1B78002B40F05281A0
:10F0B80000F080FC3F4B40B11A7803201109013160
:10F0C80091FBF0F000EB400007E01A7807201109E7
:10F0D800013191FBF0F0C400201A091A61F30712FC
:10F0E8001A7037E1F8F7A6FF002823D0314F3A7895
:10F0F80012F0F00308D163F307123A7023602E4B25
:10F108001A7842F008020EE0102B13D100F052FCDE
:10F1180080B13B786FF307133B7000232360264BC5
:10F128001A7842F0100230461A7007B0BDE8F04F66
:10F13800FFF716BB214B1E211A781E4E61F34602BB
:10F148001A70337813F0010F134B3DD022689A429E
:10F158000CD0A3F5AC639A4208D0FFF799FD28B903
:10F16800FFF7AEFD10B9AA30F3F71AFE2268144B68
:10F178009A4202D10020F3F713FE2B78522B40F06D
:10F18800AE80104B53221A70A9E000BFAC120020C9
:10F198000F15002039150020240102083015002021
:10F1A8005C15002070FC010835150020331500207F
:10F1B800002000C06D15002048150020EA15002029
:10F1C8005C010208D814002022689A420CD0A3F5EA
:10F1D800AC639A4208D0FFF75BFD28B9FFF770FDD2
:10F1E80010B9AA30F3F7DCFD2B78552B16D1FFF7B1
:10F1F80005FD3378594F43F006033370584B9B781D
:10F2080003F00203DBB24BB1F8F7F0FD236818688E
:10F21800FCF754F83B786FF341033B702B78442B91
:10F2280016D1FFF7A3FC33784C4F43F00603337035
:10F238004B4B9B7803F00203DBB24BB1F8F7D6FDDA
:10F2480023681868FCF73AF83B786FF341033B7082
:10F258002B78522B09D13378002243F00103337005
:10F26800404B1A70404B45321A70404B00271F70B4
:10F278002B78232B33D13E4B1F703E4B1F70F8F772
:10F28800B5FD33783C4943F0060333700B78334AB5
:10F29800FBB13A4A013B1770394ADBB20B7052F89E
:10F2A8002330384A23609B68934202D107F038FD27
:10F2B80015E002F59A718B4204D10120014605F050
:10F2C8003BFB0CE002F5D272934208D12E4B1F7023
:10F2D80005E0117863F30711117023603AE02B4BB6
:10F2E8001B7813B10020F3F75BFD23681F7B17F031
:10F2F8000F0702D1FDF786F91BE0012F02D1FAF7BB
:10F308003BFC16E0022F02D1FAF764FF11E0082F48
:10F3180005D84FF09C53BB4001D5FBF729FC042FBF
:10F3280003D123689B69984703E0052F01D1FBF7B8
:10F33800E7F9337803F00203DBB21BB123681868DE
:10F34800FBF7BCFF33786FF3410333702B780BB1B5
:10F35800064A137007B0BDE8F08F00BF6D15002096
:10F368007C15002036150020D8140020F514002044
:10F3780038150020781500205B1500202C1500207A
:10F388005C150020780102081A1500201F0E0020C5
:10F3980007B502AB03F8011D19460122002303F04B
:10F3A800C7FF0EBD07B5002302A901F8013D0122E0
:10F3B80004F026F89DF807000EBD08B5002303F0F9
:10F3C800B7FF002008BD034610B508461446194685
:10F3D80004F016F8E0B210BD10B5034600248454BA
:10F3E8000846194604F00CF8204610BD37B5054606
:10F3F800002400E01446012260190DF1070103F012
:10F40800FFFF9DF80730621C203BDBB25A2BF1D975
:10F4180020463EBDF8B500241949022211F83400EF
:10F4280001EBC4014000043100F571500134FFF7CD
:10F43800C4FF342CF0D143F6B6301249042200251B
:10F44800FFF7BBFF48F6D8272C4615E007EB460028
:10F4580004EB440100B259180222FFF7AEFF01364F
:10F46800F6B2094B5A199278B242EFD80134803774
:10F478000335142CBFB201D00026F2E7F8BD00BF57
:10F48800002702083FB20208A02802082DE9F34726
:10F49800044615468A46022243F6F8410DF1060055
:10F4A8001E46BDF930909DF828809DF82C70FFF716
:10F4B8008AFF2F4B2F499A78BDF906008A705A782F
:10F4C80000EBC000CA701A7900F572500A715A79B7
:10F4D8007A304A719A791B7845EAC6158A710C7098
:10F4E80081F80190CB710D7200B20922FFF765FF18
:10F4F8001EB1214B1A8801321A80BDF8063001333B
:10F508009BB2B3F57A7FADF8063002D30023ADF88D
:10F51800063002220DF1060143F6F840FFF74DFFD1
:10F52800BDF80600154B188000B200EBC00000F5CE
:10F53800725000F17A05823000B2FFF733FF10F005
:10F54800800F03D00C4B1A88013A1A8028B2002188
:10F55800FFF71EFF0A4B03F8148003EB440467709F
:10F56800BAF1000F02D00120F6F7F6F9BDE8FC87E2
:10F57800D429002052150020F0140020D81F0020A4
:10F58800911D00202DE9F743314B1D78303DEDB238
:10F59800C5F10606F6B23EB305F11207202413E0C2
:10F5A80008F101080FFA89F000215FFA88F8FFF7DF
:10F5B800EFFE09F10109B0451FFA89F9F0D1013CC4
:10F5C8000737E4B2BFB21CB1B9464FF00008E7E70D
:10F5D8000B35013428B20021E4B20135FFF7D8FE1B
:10F5E800B442ADB2F5D131E0122425B268462946BD
:10F5F8000622FFF7E8FE9DF8003043B19DF805307C
:10F608002BB99DF803308DF804308DF80530073498
:10F61800062228466946A4B2FFF7CFFEF22CE4D1B1
:10F6280068460B210622FFF7CEFE9DF8003043B155
:10F638009DF805302BB99DF803308DF804308DF80E
:10F6480005300B2069460622FFF7B7FEBDE8FE83AA
:10F65800F714002010B507F063FB09F0DDFB04F098
:10F66800B3FB04F0D9FAF3F7C9FD9C48F6F7A6F9FD
:10F6780043F6D120FFF796FE994B9A4C187043F643
:10F68800D020FFF78FFE984B187043F6DC20FFF769
:10F6980089FE964B187043F6E130FFF783FE944BD2
:10F6A800187043F6E230FFF77DFE924B187043F670
:10F6B800DA20FFF777FE904B187043F6D920FFF752
:10F6C80071FE8E4B187043F6CF20FFF76BFE8C4B04
:10F6D800187043F6CC20FFF765FE8A4B187043F686
:10F6E800D220FFF75FFE884B187043F6DF20FFF744
:10F6F80059FE864B187043F6E820FFF753FE844BFB
:10F70800187043F6DD20FFF74DFE237801280CBF63
:10F7180043F001036FF30003237043F6E020FFF783
:10F7280041FE237801280CBF43F080036FF3C71311
:10F73800237043F6E720FFF735FE764B01281A6859
:10F7480043F6EA200CBF42F000526FF35D721A6074
:10F75800FFF728FE637801280CBF43F001036FF31D
:10F76800000363706C4843F66E210822FFF72BFEF6
:10F778006A4B00241C705C706748235C312B03D1F2
:10F78800103021460DF078FF0134082CF4D12246C0
:10F7980043F6F6116048FFF716FE224643F63A2173
:10F7A8005F48FFF710FE47F2740104225D48FFF737
:10F7B8000AFE47F2780104225B48FFF704FE0AF0CC
:10F7C8006FFEF6F7CBFB43F6E120FFF7EBFD574C56
:10F7D800237860F30003237043F6E220FFF7E2FD8D
:10F7E800237860F34103237043F6E420FFF7DAFD42
:10F7F800237860F3C303237043F6E620FFF7D2FDB6
:10F80800237860F34513237043F6E920FFF7CAFD18
:10F81800237860F38613237043F6E520FFF7C2FDD3
:10F82800237860F30413237043F6EB20FFF7BAFD47
:10F83800237860F3C713237043F6E320FFF7B2FD84
:10F84800237860F3820323703948FFF7ABFD394B07
:10F8580018703948FFF7A6FD384B18703848FFF77D
:10F86800A1FD384B18703848FFF79CFD374B1870CE
:10F878003748FFF797FD374B18703748FFF792FD69
:10F88800364B18703648FFF78DFD364B18703648E2
:10F89800FFF788FD354B18703548FFF783FD354B6A
:10F8A8001870FFF76FFE3448FFF77CFD334B187074
:10F8B8003348FFF777FD334B18703348FFF772FD75
:10F8C800324B18703248FFF76DFD324B18703248D2
:10F8D800FFF768FD314B187010BD00BF0B150020F5
:10F8E8001A0E0020EA150020190E00201C0E002018
:10F8F800941200208A100020622C002000000020B2
:10F90800D8130020F61400201B0E002075240020B8
:10F9180031240020EC230020FD2400200D250020A8
:10F9280005250020FC23002012240020CF130020EE
:10F93800CE8AFFFF49270020CF8AFFFF76260020C6
:10F94800D08AFFFF46270020D18AFFFF47270020E3
:10F95800D28AFFFF78260020D48AFFFFEF250020F7
:10F96800D58AFFFFA4160020DC94FFFF0F140020A7
:10F97800DA94FFFFF714002014A2FFFFD42300201D
:10F988008FA1FFFF6B1E002091A1FFFFD61F002053
:10F9980090A1FFFFD11F0020858AFFFF7419002066
:10F9A800034B1E211A7861F346021A70704700BF94
:10F9B800EA150020024B187800F00100704700BFDC
:10F9C800EA150020014B1878C0097047EA15002095
:10F9D80008B5FFF7F7FF38B9044B1B7813F07E0F13
:10F9E8000CBF0020012008BD012008BDEA15002039
:10F9F800F8B546F6AA742046FFF7D4FC2D2803DD97
:10FA080020462D21FFF7C4FCA4F55856123E304677
:10FA1800FFF7C8FC414FC0B207EBC0000579C5F33A
:10FA28000015A5B90DE03D4B3D4953F83500F0F7F9
:10FA3800B5FD20B930462946FFF7AAFC07E0013595
:10FA4800EDB207EBC5031B7913F0080FEBD00134B7
:10FA580046F6C2739C42CED143F6C4242046FFF733
:10FA6800A1FC2D2803DD20462D21FFF791FC013450
:10FA780043F6C8239C42F1D1012143F6E120FFF768
:10FA880087FC012143F6E220FFF782FC012143F6BF
:10FA9800E420FFF77DFC012143F6E620FFF778FC20
:10FAA800012143F6E920FFF773FC012143F6E52025
:10FAB800FFF76EFC012143F6E320FFF769FC012103
:10FAC80043F6EB20FFF764FC002143F6E020FFF744
:10FAD8005FFC002143F6EA20FFF75AFC002143F6B9
:10FAE800EC20FFF755FC012143F6DC20FFF750FC22
:10FAF800002149F2DB40FFF74BFC48F64420012186
:10FB0800FFF746FC47F252042046FF21FFF740FC6E
:10FB1800013447F25A039C42F6D1F8BD080400208C
:10FB2800A69C020810B506F04BFA09F039F9074B04
:10FB38004FF416721A80012147F26200FFF728FC81
:10FB48004C20BDE8104000F01BB800BF602C00201E
:10FB580010B506F055FA09F0B7F8044B002147F242
:10FB680062001980BDE81040FFF712BC602C00202D
:10FB7800024B1888003818BF01207047602C0020FD
:10FB8800542873B5044663D83D4BDB7803F0200353
:10FB9800DBB2002B72D1172801D80EF093FB394D38
:10FBA80035F81460002E69D1E10001F5D8416846A6
:10FBB800B2310822FFF707FC334821460DF072FDE9
:10FBC80050B1F3B2072B07D0172C05D80122B24049
:10FBD800D243D2B22D4B27E01DF806300122542B18
:10FBE80008D0562B03D0532B284B1AD100E0284BB2
:10FBF800B24007E0B240254BD2B2195D42EA01019A
:10FC08001955234B195D0A431A55FFF7D3FE98B1CE
:10FC1800204B1B7883B1172C0ED81E3325F81430CF
:10FC28000AE0B240D243D2B2195D02EA0101195585
:10FC3800174B195D0A401A550136082EBCD1134BD3
:10FC48001A5D134B1B5D134318D125F8143015E0CA
:10FC5800C10001F5D8416846B2310822FFF7B3FB6D
:10FC680000231DF803202D2A05D001219940074AB9
:10FC7800105D014311550133082BF2D17CBD00BF43
:10FC8800EC230020EE150020BF1B0020891800205F
:10FC9800B11700200B1400201FB500F017FD10B994
:10FCA80000F028FD48B10021FF2300930B20042217
:10FCB8000B4601910291FFF7E9FBAD220023D9B26F
:10FCC8004D2909D0012A07D90D48002119540D489A
:10FCD80019540D4820F8131001330132552BD2B2B4
:10FCE800EDD1074B002183F85510084B08481970CF
:10FCF800084B0822197005B05DF804EBF0F74ABB11
:10FD080089180020B1170020EE15002005170020E3
:10FD1800E4160020EC15002059B1064B0C2202FB1A
:10FD28000030437AC918837A417208300BB93C33E2
:10FD380083707047F81B0020072811D9094B1B5CFA
:10FD4800022B0DD10838C0B2C308012100F007000A
:10FD580011FA00F0044A0133D15C41EA0000D054A2
:10FD6800704700BF2C1B002047240020044B0C22A6
:10FD780002FB00330C3A5A729A72FFF7DDBF00BFDC
:10FD8800F81B002010B50446FFF7F0FF034B0C22C8
:10FD980002FB0434FF23637210BD00BFF81B002070
:10FDA80070B5104D002410482146E6B20DF07AFCDB
:10FDB80098B96B7A8BB10D4AA318A25C93F83030CE
:10FDC800022A0AD0413BDAB2122A06D8084A5BB2A4
:10FDD8009A4002D53046FFF7C9FF01340C35182C7C
:10FDE800E1D170BDF81B0020D01300202C1B00208F
:10FDF8000020008810B50A4B0C2203EBD00393F8BF
:10FE08009010084B02FB00331C7A3CB900F0070045
:10FE180051FA00F010F0010F18BF1A7210BD00BFA0
:10FE28002C1B0020F81B0020044B0C2202FB003383
:10FE38001A7AFF2A01D1FF3A1A727047F81B00207C
:10FE4800104B1B7813F0010F02D10F4B187818B123
:10FE58000E4B03F590720CE00C4B03F59072197A77
:10FE68000C330139C9B2FD2998BF01209342F6D15C
:10FE78007047197A09B1FF2119720C339342F8D1EE
:10FE880000207047E21300200B140020F81B00200C
:10FE980030B504461048007800F00200C0B2C8B17E
:10FEA8000C2060430D4D285C904201D1994207D047
:10FEB800984201D1914203D0052A0BD1052B09D1D3
:10FEC8000C2303FB0455064821462B72BDE830403D
:10FED8000DF0DDBB30BD00BF15150020F81B00205C
:10FEE800161500201FB50446214614480DF0DAFB0C
:10FEF800002821D00122022300210093A318029395
:10FF08005C200B460192FFF7C1FA21460B480DF021
:10FF1800BEFB21460A480DF0BAFB214609480DF000
:10FF2800ABFB074BE40804F5CA40195DA83004B0E0
:10FF3800BDE81040FFF72CBA04B010BDC91200206C
:10FF4800D5120020D01300202DE9F7438E480DF07C
:10FF58003FFBDFF858828D4E0024E5B2284603F0B7
:10FF6800DBFF18F8019F074618F8183C13B1022B5D
:10FF78003ED10FE02846FFF7F9FE214684480DF0F0
:10FF880086FB214683480DF082FB214682480DF00E
:10FF98007EFBC9E028464946F5F764F810B12846C3
:10FFA800FFF7EEFD737AFF2B01D1FF3B7372737A73
:10FFB8004B4501D2F37A9BB1734821460DF05CFBA7
:10FFC800F37A002B40F0B080204604F0D1FA0521E6
:10FFD80028460A460B46FFF75BFF2846FFF7C6FE92
:10FFE800F37A002B40F0A0802846FFF77BFF9BE0C8
:08FFF80090B92846FFF7BAFE9C
:020000040801F1
:10000000214663480DF03CFB28463946F3F7ECFBEC
:10001000002800F086803378002B00F082803AE0E0
:10002000022814D15A4821460DF02AFB3378012BBF
:1000300001D0737A1BB928460121FFF771FE2846CB
:100040004946F5F713F800286BD0284626E0032828
:100050000FD12846FFF78EFE21464D480DF010FBCC
:1000600028460121F3F7C0FB00285AD03378032B30
:1000700010E0042815D12846FFF77CFE21464448AD
:100080000DF0FEFA28460221F3F7AEFB002848D017
:100090003378042B45D0052B43D04520FFF774FD62
:1000A0003FE001283DD1737A4B4502D32846FFF744
:1000B00061FE214638480DF0EEFA214637480DF032
:1000C000EAFA214636480DF0E6FA2846FFF7B0FE78
:1000D0003378012B25D0052B23D02846FFF706FFC8
:1000E00033780BB1032B07D12E4821460DF0DEFAF1
:1000F000B8B12046012108E0042B09D12A48214645
:100100000DF0D4FA68B120460221F2F725FA08E092
:10011000264821460DF0CAFA18B120460021F2F710
:100120004BF92846394601220223FFF7B5FE377006
:10013000214617480DF0BAFA013401462846F5F772
:10014000D7FB0C36182C7FF40CAF194D09F060FF6B
:100150002C68D4B943F6D320FFF728F9C6B29EB174
:100160004320FFF711FD2146012223460820009479
:10017000F1F7FAFF01230E20214622460094F1F701
:10018000F3FF4FF461635E432E60BDE8FE8300BF62
:1001900086180020F81B00201C1B00201F1B0020BD
:1001A000221B0020AE12002008140020E7130020BC
:1001B0000C190020431B0020324AF8B59042054636
:1001C00001D000231FE0304B1C78005D002808BFE1
:1001D000002401E00134E4B28C4207D2105D002813
:1001E000F8D02A4830F814000028F3D18C4201D10D
:1001F000002242E02649087808B9125D0A701C7096
:100200000B780EE00133DCB28C4207D2EA5C002AA4
:10021000F8D01E4A32F81320002AF3D18C422DD098
:100220002B5D002613F0010F05D10136F6B2082E22
:1002300001D05B08F6E7174F00213E7021221648D7
:1002400006EB0616F0F7AAF806F51671124801310A
:100250002022FFF7BCF8387800F046F978B93B78EF
:10026000012212FA03F3295D21EA03032B553978A1
:10027000074B8A40197821EA02021A70FF242046AF
:10028000F8BD00BFB1170020230E0020EE1500209E
:10029000EC15002009170020AA16002070B50E46A4
:1002A000C11EC9B20123002407E002FB03440A2255
:1002B00053430138A4B2C0B2DBB230B1325C303A41
:1002C000D5B2092D01D88842EFD1451C2021062244
:1002D0001648F0F763F8092CEDB204D9632C8CBFF3
:1002E0000023012309E0022307E011490135C91861
:1002F000013381F8A320DBB2EDB2052B09D8725D82
:10030000A2F13001C9B20929EFD92C2AEDD02E2A49
:10031000EBD046F60920FFF749F8844204DA55206D
:10032000BDE87040FFF730BC70BD00BF1F1A002051
:100330007C190020F0B587B00446F0F77FFA47F249
:100340006301C5B2102201A8FFF741F89DF80430FF
:100350000BB1202B03D1234B1E78022E08D9204647
:1003600001A9F0F7A3FC0746002838D001A80BE04C
:100370001D4B06EB0616F61820463146F0F796FCA4
:10038000074600282BD03046F0F758FA3F1837B30D
:100390003F1B1DE0E35D2C2B01D02E2B17D1E31961
:1003A00013F8012C303AD2B2092A10D85B78303BCE
:1003B000DBB2092B0BD80D4B1B7803F00803DBB223
:1003C00063B1013FF8B22146FFF768FF06E001374D
:1003D000FFB26B1E9F42DDDB002700E0012738469D
:1003E00007B0F0BD410E0020144402087C19002023
:1003F00008B50449F0F7D6F8D0F1010038BF002065
:1004000008BD00BFF2180020044A00231370044AFC
:100410001370044A1370044A137070474D2700206C
:1004200025190020241900200618002038B51C4B7F
:100430001C4A19781C4B19B100201870107038BD77
:1004400012789AB9194A107870B1194A117801F0E6
:100450004004E4B244B91C78844205D141F0400123
:100460001E2060F30501117000221A701C7894B1EF
:100470000F4B1D7805F04005EDB22DB943F6D520A0
:10048000FEF794FF844208D10A4B01201A7860F3EA
:1004900001021A7038BD204638BD284638BD00BF5D
:1004A00025190020061800204D270020A416002042
:1004B000482700207A26002010B5F7F79BFA084B52
:1004C00000211A68074822F002026FF382021A60C4
:1004D0001122EFF763FFBDE8104002F0D9BD00BF65
:1004E000EC230020E0180020F8B5344D07462B78A7
:1004F000A3F13002D2B2092A0CD92B2B0AD0002446
:1005000004E02E4B20221A550134E4B22B5D202B3F
:1005100002D106E0002404E0002BF2D101E0013416
:10052000E4B22E5D202EFAD0254800211122EFF7EB
:1005300035FF002E3DD0A6F13003DBB2092B02D8E7
:10054000204A00200DE02B2EFAD00020F8BD01300B
:1005500002F8013FC0B220232B5501341028E4B229
:100560000FD02B5D33B1A3F13001C9B20929EED907
:100570002B2BECD028B9F8BD104B20221A55013492
:10058000E4B22B5D202B04D0002BF5D101E0013427
:10059000E4B22B5D202BFAD00B4C0023072F2370E5
:1005A00009D807F566505830FEF700FF207001208B
:1005B000F8BD3046F8BD0120F8BD00BFAA160020E6
:1005C000E0180020DF1800209816002038B540F20F
:1005D000592500240C4829462022FEF701FF204619
:1005E000FFF782FF40B10948FFF702FF20B1012069
:1005F00010FA04F4E0B238BD0134E4B21135082C2D
:10060000E8D1002038BD00BFAA160020E018002065
:1006100070B52A4B2A4C1B7823B12A4B0020187046
:10062000207070BD2378ABB9264D2B78012B00D1FB
:1006300000BF013BDBB2012B0AD802F021FD0146CD
:100640002148F0F79DF8FFF7C1FF08B107F086F8E1
:1006500000232B701D4B587800F00200C0B2002818
:100660002AD01A6843F6D5206FF349221A60FEF7A4
:100670009DFE144DC6B22B780BB902F0E1FC0623A7
:100680009EB123702B780133DBB2B3422B7012D1B1
:100690000F4B1A786FF301021A7002F0F1FC014659
:1006A0000948F0F76DF8012070BD23702B783046B3
:1006B00001332B7070BD002070BD00BF4D2700209E
:1006C0002419002025190020F218002048190020C4
:1006D0007A2600200023074A184632F8021F11B973
:1006E0000549595C08430133572BF6D1003818BF30
:1006F00001207047EC150020891800200023074ACC
:10070000184632F8021F11B90549595C08430133F4
:10071000552BF6D1003818BF01207047EC1500208A
:10072000B117002038B50C461546F0F787F8C0B26F
:1007300007E0054B1A181B5D1219013C02F8013C39
:10074000E4B2AC42F5D838BD922A0020F8B506468E
:100750000C4608461746002110221D46EFF71EFEE4
:100760003278174B002013F8011F914206D1214621
:10077000102246F6A243F7F7E3FA12E0013004280C
:10078000F1D1002331211A463078184110F0010FC1
:1007900002D0A1540132D2B201330131042BC9B2CB
:1007A000F2D139462A462046FFF7BCFF06460548E7
:1007B000214640193246EFF749FD3046F8BD00BFEB
:1007C0000A150020922A002030B50378A121594350
:1007D00001F5387185B00131A0221248FEF700FE04
:1007E0001048F0F72BF80024C5B217E00D4B1B5D45
:1007F000242B01D10C4806E0262B01D10B4802E046
:10080000402B09D10A482A4623466946FFF79EFF36
:100810004519EDB2041900E00134E4B2AC42E5D36D
:1008200005B030BD922A0020DD130020D91200202F
:10083000D812002070B5244A03780546D31893F8DF
:100840003030542B05D121482149EFF799FF00247E
:1008500005E0462B1D480CBF1E491F49F5E72878C7
:10086000800000F5D6403E302018FEF79FFDC6B24E
:1008700046B31648EFF7E2FFC0B29F281BD8013EEF
:10088000F6B21D2E114B4FEA061108D8891901F551
:1008900014411818EE311122FEF799FD0BE00F4AB2
:1008A00089198918181801F1100351F8042B99427D
:1008B00040F8042BF9D1054809490134EFF7C8FD88
:1008C000042CCCD170BD00BF2C1B0020922A00202C
:1008D000B67D0208D77D0208957D0208139C0208A8
:1008E0005FB2020838B52C4D2B782C46012B16D060
:1008F00002D3022B4BD138E057212848FFF75CFC8C
:10090000274BFF28187045D026482749EFF738FFB6
:10091000264B1A78264B1A702B7801332B702148FE
:1009200001F098FB002836D01D480378172B02D819
:10093000FFF780FF10E0A3F15202D2B2022A02D8E0
:10094000FFF742FF08E0A121594301F5387119482A
:100950000131A022FEF744FD16481749EFF778FD54
:10096000237800200133237038BD01F093FB90B150
:100970000F4901200978002310FA01F12B70084B70
:10098000064A1B78D45C24EA0101D15438BD00200A
:10099000287038BD012038BD240E002089180020A1
:1009A000AF170020F4160020E018002009170020DF
:1009B00006170020922A002067B2020808B502F04C
:1009C00085FA18B9074B05225A7008BDF6F7E0FF03
:1009D000232804D1034B07225A70233808BD012075
:1009E00008BD00BF240E002038B50124844000213A
:1009F0000A480B22EFF7D2FCE4B20025084BEB5C6F
:100A00001C4207D0074B33F815301BB90348294661
:100A10000CF036FE0135552DF0D138BD9916002069
:100A2000B1170020EE15002070B501258540002487
:100A3000EDB20A4821460CF039FE20B1084BE25CC9
:100A400022EA0502E2540134552CF2D10348002178
:100A50000B22BDE87040EFF7A1BC00BF9916002043
:100A6000B117002010B50B4A137813F001000FD016
:100A7000094903F0FE0309780848002413F0040F25
:100A80004454137003D0FFF70BF9012010BD01206F
:100A900010BD00BF82180020A6160020E41600201A
:100AA00070B586B0F6F774FF002800F09A804E4BC0
:100AB0004E491A7888540132D2B2072A1A7001D9E5
:100AC00007221A704A4E1A783378303B9A42C0F2A5
:100AD0008580454B00221A7043F6E410FEF766FC51
:100AE000C4B214B91224002509E0FFF76FFD10EA23
:100AF0000401F7D108223D48EFF750FC70E00021D7
:100B0000072204A8EFF74AFC0622214604A8FEF7B4
:100B10005EFC327804A8303A3449EFF7BFFE10F09B
:100B2000FF0F38D12846FDF7B9FD0146002857D1FF
:100B300004A80722EFF732FC2846F4F7ADFE20B9EF
:100B40002846F4F7BFFE00284AD02A4C002108228C
:100B50002648EFF723FC0021FF2325700422009391
:100B600001350B461C2001910295FEF793FC20787D
:100B7000214D00F56A506E30FEF718FC2870207881
:100B800000F5D4401230FEF711FC68702846F4F7E7
:100B9000FFFE022025E00135EDB20734202DAED155
:100BA0000021072204A8EFF7F9FB062240F25221A8
:100BB00004A8FEF70CFC0E4B0C491A7804A8303A36
:100BC000EFF76CFE0021044608220848EFF7E6FB29
:100BD00014F0FF0F14BF0120052002E0032000E005
:100BE000012006B070BD00BF11190020EC160020D6
:100BF000F7140020D016002039150020044B054AB8
:100C00001B784FF4926101FB032318180DF0C6BA4C
:100C1000F6140020F4AB0208024800219222EFF7FC
:100C2000BDBB00BF1C17002010B504460548EFF7F8
:100C300005FE80B2912801D9013880B2014B1C54C5
:100C400010BD00BF1C1700202DE9F041FFF7E4FFA5
:100C5000A92646F642350024174821460CF026FD09
:100C6000E0B1E3B2172B16D8144BE31893F83030E9
:100C7000542B01D1FB2000E02520FFF7D5FF2F1FCB
:100C80003846FEF793FBC0B240B10137FFF7CCFF07
:100C9000AF42F5D102E03046FFF7C6FF013401361E
:100CA0000435552CF6B2D7D1FC20FFF7BDFF044820
:100CB000BDE8F0410DF072BA991600202C1B0020FF
:100CC0001C170020F0B5734C85B06378072B00F239
:100CD0007881DFE813F00800370057008500C7006F
:100CE00007013001690155216B48FFF765FA6B4B2D
:100CF000FF28187000F06A8169496A48EFF740FDE3
:100D0000694B6A4A1D78012313FA05F01178684E81
:100D100040EA01011170674A674F11786370674AB2
:100D2000735D3D70117023B943F6E010FEF73EFB92
:100D30007055634B9B7803F02003DBB213B13B7813
:100D40000122F2545C4B1878FFF74EFE5D480B21F0
:100D50000CF089FCF8B95C4B1B78002B40F0368115
:100D6000504802F073F8002800F033814D4957488D
:100D7000EFF706FD022343F6E3106370FEF716FB60
:100D8000534B18704C4B1878FFF72EFE4D480B2133
:100D90000CF069FC08B1062379E002F097F8E0B1A5
:100DA00002F0BEF8484D10B1494B1B782B702B78E0
:100DB0000BB901F027F902F0E3F8002800F00981EF
:100DC00003236370F6F716FE43F6E210FEF7EEFA21
:100DD000404B187002232B70FAE006236370F5E095
:100DE000FFF7ECFD002800F0F480374B1B78002B58
:100DF00040F0EE80304B1878FFF7F6FD364B1D784B
:100E000015F0030523D104F0C7FF002800F0E180AE
:100E100004F0A4FF002800F0DC800AF0E3FE0028C4
:100E200040F0D2802D4B93F8292093F82A1042EA03
:100E3000012193F82B2041EA0241024661F3170297
:100E4000D3F82100D3F82510032304F067FF244BC7
:100E50001A7842F014026FF345121A70FFF7F4FE8D
:100E6000042314E0FFF7AAFD002800F0B2800DF083
:100E7000C5F9002840F0AC80164B1A780AB1013A47
:100E80001A701B7873B3104B02221A70032363701D
:100E90009EE000BF240E0020B1170020AE170020F6
:100EA000E01800200B17002009170020051700206C
:100EB000E416002098160020A616002082180020B4
:100EC000EC23002099160020A9160020F21800201B
:100ED00083180020101900207A2600204C0C0020D6
:100EE000603100203C4D0DF0ABF92A78012111FA58
:100EF00002F23A4B3A4E197821EA02021A7033781C
:100F000003F00503042B01D1FEF7CAFE337813F07A
:100F1000010002D12A783349885403F00303022BDD
:100F200004D1314B1A7842F010021A7001F0CEFF52
:100F300008B90623637043F6E110FEF737FA264F2F
:100F40002A4B284A18703B78D15C09B10139D15439
:100F5000012515FA03F62649D25C087820EA060036
:100F60000870CAB91D4E3178194111F0010F10D027
:100F70005B19FF2100910192029329462B463B20E9
:100F80000332FEF787FA3B789D40337823EA050564
:100F900035703878FFF748FD0023637001F0F0FFEB
:100FA000A0B901F02FF811E00DF04AF905236370A4
:100FB000FFF758FD60B90C4B1A7842F008021A701E
:100FC00007E00020607004E0284602E0012000E015
:100FD000002005B0F0BD00BFA616002005170020B8
:100FE00082180020E416002085180020A916002091
:100FF000EC15002008B5064B4FF492611A78054BAA
:1010000001FB0231922209180348EFF71FF908BDCE
:10101000F6140020F4AB02081C17002070B53B4CFE
:101020002378032B66D8DFE803F0020A1946384B11
:1010300003221A7001232370364B033A1A70344B83
:101040001B78002B59D0344B1A7842F001021A70E9
:1010500023780022013323702E4B1A700DF0CEF846
:1010600010B12E4B0A221A702B4D2B7813F0010F62
:101070000CD00DF0C3F8064640B9FFF7BFFD2B7842
:101080000A2266F300032B70244B1A70FFF708FD49
:10109000032805D10DF0D4F82378013323702EE016
:1010A0001E4B187800282AD1194B1A78013A1A7069
:1010B0000123237070BDFFF7F3FC184B05461B7826
:1010C0000BB1012808D19220FFF798FD104B1A7838
:1010D000013A1A7001232370022D12D0052D12D16E
:1010E000FFF79AFDBF20FFF79FFD0D480DF056F862
:1010F000FEF7D6FD0020207070BD012070BD0020DD
:1011000070BD284670BD002070BD00BFA81600202D
:10111000081700201119002085180020121900203E
:101120001C1700200A4A13783BB1013BDBB2137055
:10113000084A52F82320084B1A60084B08481A78CE
:1011400000216FF300021A709222EFF727B900BF57
:10115000B017002014190020CC16002040310020C8
:101160001C1700202DE9F041394D3A4F2B7823B957
:101170000DF044F808B103233B703B78002B60D19D
:10118000354C2078002860D00DF038F800285BD16D
:101190002B78FF2B07D12E4B1870FFF7C3FF2D4A7A
:1011A000032313702370DFF8C4802C4E98F80030AE
:1011B00033B340460CF0F2FF002192224046EFF795
:1011C000EDF8274A33681146934205D0254A9342E9
:1011D00002D0FF232B7034E025781F4A0120002D18
:1011E00033D08B4204D1107001380CF033FB1CE07B
:1011F0001C498B4219D1107000200CF0F1FC14E056
:101200002B78142253433268DFF84480D1180979CF
:1012100079B9154B1B7823B14FF49270FFF7EEFCB0
:1012200001E005233B7000232B702378013B2370E2
:1012300007E0D058FFF7E2FC98F80030013388F857
:1012400000300120BDE8F0810120BDE8F08100BF41
:10125000F11800201219002081180020CC1600205F
:10126000580F0020D00F0020B01700201C170020BE
:1012700030B50F4A0F4913780D680F4C8068022B68
:1012800044F82350086001D8013313700B4B984287
:1012900004D10020BDE830400CF0DCBA084B984285
:1012A00004D10020BDE830400CF09ABC30BD00BF36
:1012B000B0170020CC16002014190020580F002071
:1012C000D00F002010B5154B1B681979022903D1E6
:1012D00013490870184617E012498B4203D1BDE844
:1012E00010400CF0C5BB10498B4203D1BDE8104043
:1012F0000CF00ABD142101FB00321379012B02D03E
:10130000032B0AD104E01046BDE81040FFF7B0BF40
:10131000034913690878117B984710BDCC1600204B
:1013200084180020580F0020D00F00201D4BF7B567
:101330001B68002504E01A7B1433954238BF15461C
:101340001A79002AF7D16846F6F768FB044608B117
:10135000F6F750FB0DF1FF3620E0134B03221A7015
:10136000124A00231370124A16F8017F13700CF012
:1013700067FF232F02D1FFF7D5FE11E0303FFFB208
:1013800037B1AF4204D8013FF8B2FFF79BFF07E047
:10139000013C4FF4DB70E4B2FFF72CFE002CDCD1F3
:1013A0000120FEBDCC16002081180020121900205B
:1013B000F118002010B5104B00241A7821466FF365
:1013C00000021A700D4B0E4A1C700E4B0E481A602C
:1013D0000822EEF7E3FFFFF71FFC0C4BFF221C7007
:1013E0000B4B1C700B4B1A700B4BFC3A1C700B4BCD
:1013F0001A700B4B1C7010BD403100208518002066
:10140000A4B10208CC160020EC160020111900200F
:1014100012190020F1180020A816002081180020C1
:10142000B017002070B5364CA378042B60D8DFE8E5
:1014300003F00320334E57000123A370314B1B7878
:1014400003F00802D2B212B12D4A0221917003F0CA
:101450001003DBB203252C4E2BB1FFF7ABFF0020AE
:10146000A570307070BDFFF7A5FF284B1D700A23D3
:101470003370254D287800282CD0F6F789FA2328D8
:1014800039D1FFF7EFFA20B10020052360702B70EF
:1014900070BD02232870A370FFF7C0FD012803D19F
:1014A0000423A370013870BD022826D1FFF7B4FBD6
:1014B000154B00251D700323A370154B1878F4F706
:1014C00001FAD8B1134A144B28461A6070BDFFF7D1
:1014D00049FE10B90423A37070BDFFF727FF0AE08F
:1014E00000F090FD0CF0ACFE0023A370012070BD55
:1014F0000020A07070BD002070BD002070BD00BF36
:10150000240E002085180020121900200817002042
:10151000D0160020F4B10208CC1600202DE9F041CD
:10152000884D894C2B6826466FF3DB632B6023784C
:101530006FF34513237001F0CFFD58B1834B1B7837
:1015400043B10220072106F05DFA237843F020031F
:10155000237010E001F0A4FD90B17D4B1B787BB9A6
:101560007A4B1B7863B10220012106F04BFA3378E5
:1015700043F0200333702B6843F000632B6010E0CE
:1015800008F07AF910B10220012108E0297801F071
:101590001001C9B211B10220014600E0022006F09C
:1015A00031FA6C4C2378082B00F21C83DFE813F02F
:1015B00009001E002B0136015A017A01E6010902D9
:1015C0000A030BF0C5FB08F00DF9FEF775FFFEF7F7
:1015D0001BFF614B00229A70012323705F4880211A
:1015E0000DF055F804F0E0FB0CF038FEFF205C4EE7
:1015F000014608F06FF9337803F00A02082A06D092
:1016000003F00502042A02D013F0300F0DD0554B21
:101610001B7803F00203DBB20BB104F0C5FB337897
:1016200003F0D3036FF304133370AB7803F00203BA
:10163000DBB24BB1082323704B484C4B3C221A7051
:10164000BDE8F0410CF0AABD494E337803F04003E9
:10165000DBB223B908F028F9002800F0C382FEF7B6
:10166000E5FE10B9FEF7D4FF70B101F0A1FC414BCB
:101670001A7842F008021A70374B00229A7005233C
:1016800023703D4B02321A706B7803F00203DBB219
:101690005BB1337803F04003DBB233B1374B1A78D8
:1016A0006FF301021A70062308E0FFF713F840B148
:1016B000337803F04003DBB21BB102232370BDE893
:1016C000F081F1F707F82E4DFF28287029D02D4B17
:1016D0001B78002B40F08682012212FA00F02A4B80
:1016E0001A781043187043F6DF30FDF75FFE274B82
:1016F0001870274808F014F8204B1B7803F00303F8
:10170000022B00F06F822978224801EB011101F5CC
:101710006C5107232E3110222370BDE8F041FDF7F4
:101720005FBEFEF7EBFF002838D01B4807F0F8FF3C
:10173000124B1B7803F00303022B00F053820323A8
:10174000BCE700BFEC2300206025002074190020B6
:101750004F2C0020E3160020240E00200010014032
:1017600060310020D723002007180020662C0020BD
:101770004819002085180020A51600207A26002090
:10178000A71600200A17002091120020071700203A
:1017900046270020E018002076260020984B994C20
:1017A0005A7860F386125A70257805F01003DBB280
:1017B000002B00F01782337803F04003DBB2002BDC
:1017C00000F01082904B1B7833B963F3041563F378
:1017D00001052570BDE8F08115F00C0540F002828E
:1017E0002946062204F1A300EEF7D8FDA01C2946E5
:1017F000A122EEF7D3FDF0236370237843F00403B6
:1018000065F304135AE70221FF2008F063F8FFF79D
:1018100069F8002800F0E68100234FE77B4B1B7836
:1018200023B17B4B5B78012B3FF448AF794B1B789E
:1018300003F00303012B02D10220FF2101E0FF206E
:10184000022108F047F8FFF73DFA002800F0CA81AE
:1018500001F096FB002800F08E806D4B00229A70FC
:10186000042323706B4B1B7803F00303012B02D17D
:101870000220FF2101E0FF20022108F02BF801F0F7
:101880007FFB20B1FFF7CEFD002800F0AB8101F017
:1018900077FB08B900F0B6FB00232370BDE8F041E8
:1018A0000CF0CEBC5B4D2B7803F00303012B02D16F
:1018B0000220FF2101E0FF20022108F00BF804F0D4
:1018C0006BFA002800F08E8104F048FA002800F03E
:1018D00089810AF087F9002840F084812D784E49EB
:1018E00005F00305012D19D191F82A2091F829302E
:1018F00043EA022391F82B2043EA024300F07F429F
:101900001A43D1F821000D23D1F8251004F006FA6E
:10191000424880212A460CF0BAFE13E091F82A20B2
:1019200091F8293043EA022391F82B2043EA02433D
:1019300000F07F421A43D1F821000323D1F825108B
:1019400004F0ECF9364B1A7842F014026FF34512AA
:101950001A702F4B00229A7001F012FB30B1314BFC
:101960001B78002B40F03E810433A7E601F038FBE2
:10197000002840F037812070BDE8F0810221FF206F
:1019800007F0A8FF284801F061FA01F041FB10B907
:10199000264B05221A7001F03BFB20B901F096FAA4
:1019A000002840F01F81214B1E78002E40F01A8144
:1019B0002B6866F349232B6000F024FB2670BDE8FA
:1019C000F081144E337803F00303012B02D102207F
:1019D000FF2101E0FF20022107F07CFF144B1F785C
:1019E00067BB144D01222878134B8240197821EAF5
:1019F00002021A70F0F7A0FE2F702770BDE8F08188
:101A0000742600207C19002074190020A9160020DB
:101A1000240E00207A2600204C0C002000100140EB
:101A200060310020A5160020D2160020D11600201B
:101A3000E0180020A7160020911200206A4B1A78A7
:101A4000984602F02002D2B29ABB337813F0030F0B
:101A50002FD104F0A1F9002800F0C48004F07EF931
:101A6000002800F0BF800AF0BDF80746002840F0CB
:101A7000B9805E4B93F8292093F82A1042EA01219D
:101A800093F82B2041EA0241024661F31702D3F892
:101A90002100D3F82510082304F040F998F800300D
:101AA00067F3041367F38203DBB243F0200388F883
:101AB00000304F4801F0CAF901F04AFA002866D117
:101AC0004C4B9B7803F01003DBB21BB9337813F057
:101AD000030F0BD0484B5B7803F00803DBB2002BFD
:101AE00055D1337803F00303012B50D101F048FAAC
:101AF000002846D098F800303B4D03F02003DBB2BD
:101B0000002B35D1337803F00303012B30D104F0DF
:101B100043F9002866D004F021F9002862D00AF0C9
:101B200061F8064600285DD1334B5B7803F0020371
:101B3000DBB2EBB12D4B93F8292093F82A1042EA3F
:101B4000012193F82B2041EA0241024661F317027A
:101B5000D3F82100D3F82510102304F0DFF82B78F8
:101B600066F3041366F38203DBB243F020032B70A9
:101B7000224B1878F0F7FEFD002833D000F042FA2F
:101B800019E001F0CDF928B11D4B1A7800E00022D0
:101B90001C4B1A701B4B1B7823BB184E3078F0F788
:101BA0003FFF00F02FFAAB7803F04003DBB213B134
:101BB0003078F0F7C1FD00232370134B0F221A7009
:101BC000BDE8F081FF20014607F084FE0F4B1B7833
:101BD00023B1054B1B7813F0010F03D10CF03EFB32
:101BE00001232370BDE8F081603100204C0C0020FF
:101BF000E01800204819002074260020A7160020B5
